:020000040800F2
:1000000000000120F5220008D1160008D3160008D0
:10001000D5160008D7160008D91600080000000001
:10002000000000000000000000000000DB160008D7
:10003000DD16000800000000DF160008E1160008C9
:100040003D2300083D2300083D230008E916000871
:100050003D230008F9160008FB16000805170008E4
:100060003D2300083D2300080F1700083D2300082A
:100070003D2300083D2300083D2300081917000810
:100080003D2300083D2300083D2300083D230008D0
:10009000291700083D2300083D2300083D230008E0
:1000A0003D2300083D2300083D2300083D230008B0
:1000B0003D2300083D230008391700083D230008B0
:1000C0003D2300083D2300083D2300083D23000890
:1000D0003D230008491700083D2300085917000870
:1000E0003D230008691700083D2300083D23000850
:1000F0003D2300083D2300083D2300083D23000860
:100100003D2300083D2300083D2300083D2300084F
:100110003D2300083D2300083D2300083D2300083F
:100120003D2300083D2300083D2300083D2300082F
:1001300000000000000000000000000000000000BF
:1001400000000000000000000000000000000000AF
:10015000000000000000000000000000000000009F
:10016000000000000000000000000000000000008F
:10017000000000000000000000000000000000007F
:10018000000000000000000000000000000000006F
:10019000000000000000000000000000000000005F
:1001A000000000000000000000000000000000004F
:1001B000000000000000000000000000000000003F
:1001C000000000000000000000000000000000002F
:1001D000000000000000000000000000000000001F
:0401E0005FF8E0F1F3
:1001E8004FF0FF0C1CEAD0521EBF1CEAD15392EA12
:1001F8000C0F93EA0C0F6FD01A4480EA010C4002EE
:1002080018BF5FEA41211ED04FF0006343EA501047
:1002180043EA5111A0FB01310CF00040B1F5000F89
:100228003EBF490041EAD3715B0040EA010062F138
:100238007F02FD2A1DD8B3F1004F40EBC25008BF22
:1002480020F00100704790F0000F0CF0004C08BF40
:1002580049024CEA502040EA51207F3AC2BFD2F10D
:10026800FF0340EAC250704740F400004FF000031B
:10027800013A5DDC12F1190FDCBF00F00040704755
:10028800C2F10002410021FA02F1C2F1200200FA93
:1002980002FC5FEA310040F1000053EA4C0308BF5A
:1002A80020EADC70704792F0000F00F0004C02BFAB
:1002B800400010F4000F013AF9D040EA0C0093F026
:1002C800000F01F0004C02BF490011F4000F013B80
:1002D800F9D041EA0C018FE70CEAD15392EA0C0FEE
:1002E80018BF93EA0C0F0AD030F0004C18BF31F059
:1002F800004CD8D180EA010000F00040704790F02F
:10030800000F17BF90F0004F084691F0000F91F0D2
:10031800004F14D092EA0C0F01D142020FD193EA98
:100328000C0F03D14B0218BF084608D180EA010020
:1003380000F0004040F0FE4040F40000704740F0FC
:10034800FE4040F44000704781F0004102E000BFE9
:1003580083F0004330B54FEA41044FEA430594EA7D
:10036800050F08BF90EA020F1FBF54EA000C55EAB8
:10037800020C7FEA645C7FEA655C00F0E2804FEA89
:100388005454D4EB5555B8BF6D420CDD2C4480EA6B
:10039800020281EA030382EA000083EA010180EA9B
:1003A800020281EA0303362D88BF30BD11F0004FE9
:1003B8004FEA01314FF4801C4CEA113102D040421F
:1003C80061EB410113F0004F4FEA03334CEA13335A
:1003D80002D0524263EB430394EA050F00F0A78072
:1003E800A4F10104D5F1200E0DDB02FA0EFC22FA6D
:1003F80005F2801841F1000103FA0EF2801843FA61
:1004080005F359410EE0A5F120050EF1200E012A51
:1004180003FA0EFC28BF4CF0020C43FA05F3C0188F
:1004280051EBE37101F0004507D54FF0000EDCF108
:10043800000C7EEB00006EEB0101B1F5801F1BD3B1
:10044800B1F5001F0CD349085FEA30004FEA3C0CB5
:1004580004F101044FEA445212F5800F80F09A80AB
:10046800BCF1004F08BF5FEA500C50F1000041EBAF
:10047800045141EA050130BD5FEA4C0C404141EBB3
:100488000101013C28BFB1F5801FE9D291F0000FAE
:1004980004BF01460020B1FA81F308BF2033A3F15D
:1004A8000B03B3F120020CDA0C3208DD02F1140C54
:1004B800C2F10C0201FA0CF021FA02F10CE002F18F
:1004C8001402D8BFC2F1200C01FA02F120FA0CFC88
:1004D800DCBF41EA0C019040E41AA2BF01EB0451D1
:1004E800294330BD6FEA04041F3C1CDA0C340EDCCF
:1004F80004F11404C4F1200220FA04F001FA02F312
:1005080040EA030021FA04F345EA030130BDC4F1CF
:100518000C04C4F1200220FA02F001FA04F340EAC4
:100528000300294630BD21FA04F0294630BD94F075
:10053800000F83F4801306BF81F480110134013D5C
:100548004EE77FEA645C18BF7FEA655C29D094EACD
:10055800050F08BF90EA020F05D054EA000C04BF4B
:100568001946104630BD91EA030F1EBF0021002036
:1005780030BD5FEA545C05D14000494128BF41F0D5
:10058800004130BD14F580043CBF01F5801130BD39
:1005980001F0004545F0FE4141F470014FF00000C4
:1005A80030BD7FEA645C1ABF194610467FEA655C75
:1005B8001CBF0B46024650EA013406BF52EA033517
:1005C80091EA030F41F4002130BD00BF90F0000F05
:1005D80004BF0021704730B54FF4806404F1320441
:1005E8004FF000054FF0000150E700BF90F0000FFA
:1005F80004BF0021704730B54FF4806404F1320421
:1006080010F0004548BF40424FF000013EE700BFF0
:1006180042004FEAE2014FEA31014FEA02701FBF80
:1006280012F07F4393F07F4F81F06051704732F0B2
:100638007F4208BF704793F07F4F04BF41F4002109
:10064800704730B54FF4607401F0004521F0004167
:100658001CE700BF50EA010208BF704730B54FF0F1
:1006680000050AE050EA010208BF704730B511F0F2
:10067800004502D5404261EB41014FF4806404F12A
:1006880032045FEA915C3FF4D8AE4FF003025FEAB0
:10069800DC0C18BF03325FEADC0C18BF033202EB34
:1006A800DC02C2F1200300FA03FC20FA02F001FA8E
:1006B80003FE40EA0E0021FA02F11444BDE600BF31
:1006C80080F0004002E000BF81F0004142001FBFFF
:1006D8005FEA410392EA030F7FEA226C7FEA236C08
:1006E8006AD04FEA1262D2EB1363C1BFD2184140FD
:1006F80048404140B8BF5B42192B88BF704710F093
:10070800004F40F4000020F07F4018BF404211F035
:10071800004F41F4000121F07F4118BF494292EA9D
:10072800030F3FD0A2F1010241FA03FC10EB0C00C9
:10073800C3F1200301FA03F100F0004302D5494256
:1007480060EB4000B0F5000F13D3B0F1807F06D303
:1007580040084FEA310102F10102FE2A51D2B1F1FB
:10076800004F40EBC25008BF20F0010040EA0300F0
:100778007047490040EB0000013A28BFB0F5000F70
:10078800EDD2B0FA80FCACF1080CB2EB0C0200FA26
:100798000CF0AABF00EBC25052421843BCBFD04075
:1007A8001843704792F0000F81F4000106BF80F4EF
:1007B80000000132013BB5E74FEA41037FEA226CB2
:1007C80018BF7FEA236C21D092EA030F04D092F07D
:1007D800000F08BF0846704790EA010F1CBF0020B1
:1007E800704712F07F4F04D1400028BF40F000400E
:1007F800704712F100723CBF00F50000704700F02E
:10080800004343F0FE4040F4000070477FEA226254
:1008180016BF08467FEA23630146420206BF5FEA25
:10082800412390EA010F40F4800070474FF0000325
:1008380004E000BF10F0004348BF40425FEA000CEC
:1008480008BF704743F0964301464FF000001CE094
:1008580050EA010208BF70474FF000030AE000BFEA
:1008680050EA010208BF704711F0004302D5404228
:1008780061EB41015FEA010C02BF8446014600209A
:1008880043F0B64308BFA3F18053A3F50003BCFAB5
:100898008CF2083AA3EBC25310DB01FA02FC634462
:1008A80000FA02FCC2F12002BCF1004F20FA02F269
:1008B80043EB020008BF20F00100704702F120025C
:1008C80001FA02FCC2F1200250EA4C0021FA02F2BD
:1008D80043EB020008BF20EADC707047844641EA17
:1008E800000313F0030349D1403A23D30B68036094
:1008F8004B6843608B688360CB68C3600B69036196
:100908004B6943618B698361CB69C3610B6A03627D
:100918004B6A43628B6A8362CB6AC3620B6B036365
:100928004B6B43638B6B8363CB6BC363403040314A
:10093800403ADBD230320BD30B6803604B6843601C
:100948008B688360CB68C36010301031103AF3D2E3
:100958000C3205D351F8043B40F8043B043AF9D271
:10096800043208D0D2071CBF11F8013B00F8013B44
:1009780001D30B8803806046704700BF082A13D351
:100988008B07B1D010F00303AED0C3F10403D21A21
:10099800DB071CBF11F8013B00F8013BA4D331F879
:1009A800023B20F8023B9FE7043AD9D3013A11F8F9
:1009B800013B00F8013BF9D20B7803704B78437088
:1009C8008B7883706046704770B54FF0FF0C4CF41D
:1009D800E06C1CEA11541DBF1CEA135594EA0C0F75
:1009E80095EA0C0F00F0DEF82C4481EA030621EAB0
:1009F8004C5123EA4C5350EA013518BF52EA0335EB
:100A080041F4801143F4801338D0A0FB02CE4FF09C
:100A18000005E1FB02E506F00042E0FB03E54FF0CC
:100A28000006E1FB03569CF0000F18BF4EF0010EC4
:100A3800A4F1FF04B6F5007F64F5407404D25FEAC0
:100A48004E0E6D4146EB060642EAC62141EA555173
:100A58004FEAC52040EA5E504FEACE2EB4F1FD0CB5
:100A680088BFBCF5E06F1ED8BEF1004F08BF5FEA33
:100A7800500E50F1000041EB045170BD06F00046E5
:100A880046EA010140EA020081EA0301B4EB5C0492
:100A9800C2BFD4EB0C0541EA045170BD41F480118A
:100AA8004FF0000E013C00F3AB8014F1360FDEBFAF
:100AB800002001F0004170BDC4F10004203C35DA8B
:100AC8000C341BDC04F11404C4F1200500FA05F30E
:100AD80020FA04F001FA05F240EA020001F00042AF
:100AE80021F0004110EBD37021FA04F642EB060125
:100AF8005EEA430E08BF20EAD37070BDC4F10C044F
:100B0800C4F1200500FA04F320FA05F001FA04F212
:100B180040EA020001F0004110EBD37041F10001FE
:100B28005EEA430E08BF20EAD37070BDC4F1200509
:100B380000FA05F24EEA020E20FA04F301FA05F271
:100B480043EA020321FA04F001F0004121FA04F219
:100B580020EA020000EBD3705EEA430E08BF20EAE9
:100B6800D37070BD94F0000F0FD101F00046400023
:100B780041EB010111F4801F08BF013CF7D041EAA5
:100B8800060195F0000F18BF704703F000465200A9
:100B980043EB030313F4801F08BF013DF7D043EA7A
:100BA8000603704794EA0C0F0CEA135518BF95EA30
:100BB8000C0F0CD050EA410618BF52EA4306D1D1B7
:100BC80081EA030101F000414FF0000070BD50EAD6
:100BD800410606BF1046194652EA430619D094EA60
:100BE8000C0F02D150EA013613D195EA0C0F05D14A
:100BF80052EA03361CBF104619460AD181EA03019E
:100C080001F0004141F0FE4141F470014FF0000055
:100C180070BD41F0FE4141F4780170BD70B54FF0F0
:100C2800FF0C4CF4E06C1CEA11541DBF1CEA135570
:100C380094EA0C0F95EA0C0F00F0A7F8A4EB050452
:100C480081EA030E52EA03354FEA013100F0888049
:100C58004FEA03334FF0805545EA131343EA126312
:100C68004FEA022245EA111545EA10654FEA0026C7
:100C78000EF000419D4208BF964244F1FD0404F580
:100C8800407402D25B084FEA3202B61A65EB0305DC
:100C98005B084FEA32024FF480104FF4002CB6EB99
:100CA800020E75EB030E22BFB61A754640EA0C0019
:100CB8005B084FEA3202B6EB020E75EB030E22BF59
:100CC800B61A754640EA5C005B084FEA3202B6EB9A
:100CD800020E75EB030E22BFB61A754640EA9C0059
:100CE8005B084FEA3202B6EB020E75EB030E22BF29
:100CF800B61A754640EADC0055EA060E18D04FEAE7
:100D0800051545EA16754FEA06164FEAC30343EA86
:100D180052734FEAC2025FEA1C1CC0D111F4801F53
:100D28000BD141EA00014FF000004FF0004CB6E74C
:100D380011F4801F04BF01430020B4F1FD0C88BFEB
:100D4800BCF5E06F3FF6AFAEB5EB030C04BFB6EBF6
:100D5800020C5FEA500C50F1000041EB045170BDE9
:100D68000EF0004E4EEA113114EB5C04C2BFD4EB16
:100D78000C0541EA045170BD41F480114FF0000E9A
:100D8800013C90E645EA060E8DE60CEA135594EA16
:100D98000C0F08BF95EA0C0F3FF43BAF94EA0C0F19
:100DA8000AD150EA01347FF434AF95EA0C0F7FF48E
:100DB80025AF104619462CE795EA0C0F06D152EAE2
:100DC80003353FF4FDAE1046194622E750EA4106C6
:100DD80018BF52EA43067FF4C5AE50EA41047FF4D7
:100DE8000DAF52EA43057FF4EBAE12E74FF0FF3C3C
:100DF80006E000BF4FF0010C02E000BF4FF0010C0D
:100E08004DF804CD4FEA410C7FEA6C5C4FEA430C85
:100E180018BF7FEA6C5C1BD001B050EA410C0CBFD4
:100E280052EA430C91EA030F02BF90EA020F002036
:100E3800704710F1000F91EA030F58BF994208BF9D
:100E480090422CBFD8176FEAE37040F0010070475A
:100E58004FEA410C7FEA6C5C02D150EA013C07D1B1
:100E68004FEA430C7FEA6C5CD6D152EA033CD3D0FC
:100E78005DF8040B704700BF8446104662468C46F6
:100E88001946634600E000BF01B5FFF7B7FF002829
:100E980048BF10F1000F01BD4DF808EDFFF7F4FF52
:100EA8000CBF012000205DF808FB00BF4DF808EDDD
:100EB800FFF7EAFF34BF012000205DF808FB00BF00
:100EC8004DF808EDFFF7E0FF94BF012000205DF822
:100ED80008FB00BF4DF808EDFFF7CEFF94BF0120D7
:100EE80000205DF808FB00BF4DF808EDFFF7C4FFD0
:100EF80034BF012000205DF808FB00BF4FEA410C19
:100F08007FEA6C5C02D150EA013C0AD14FEA430CFB
:100F18007FEA6C5C02D152EA033C02D14FF0000038
:100F280070474FF0010070474FEA410212F5001276
:100F380015D211D56FF47873B3EB625212D94FEA18
:100F4800C12343F0004343EA505311F0004F23FA02
:100F580002F018BF404270474FF00000704750EA57
:100F6800013005D111F0004008BF6FF00040704714
:100F78004FF00000704700BF0348044B834202D083
:100F8800034B03B118477047DC070020DC0700203B
:100F9800000000000548064B1B1AD90F01EBA301FE
:100FA800491002D0034B03B118477047DC070020F3
:100FB800DC0700200000000010B5064C237843B978
:100FC800FFF7DAFF044B13B10448AFF300800123A5
:100FD800237010BDDC07002000000000081D010878
:100FE80008B5054B1BB105490548AFF30080BDE8BE
:100FF8000840FFF7CFBF00BF00000000E007002057
:10100800081D010800B583B00A4B5A6942F0010275
:101018005A615B6903F001030193019B00221146A9
:101028000F2001F099FA0F2001F0A6FA03B05DF83D
:1010380004FB00BF0010024030B587B000230293C4
:10104800039304930593134B1B680BB107B030BD92
:10105800104B01221A60104B5A6942F480725A618F
:101068005B6903F480730193019B4FF680730293CD
:10107800022503950324059402A9084801F038FDC8
:101088004CF6B37302930395059402A9044801F042
:101098002FFDDBE7F8070020001002400018014090
:1010A8000014014010B588B0002201920292039208
:1010B800049205920692079216484FF02043036067
:1010C80003F5827343608260C2600261102141614E
:1010D8008261C261026242624FF480538362C262DB
:1010E8000263426382630F2301930293FF240394F4
:1010F800049305911123069301A904F0C0F930B9AE
:10110800054AD36943F48063D36108B010BD00F089
:10111800ABF8F5E7FC0700200000014008B5FFF731
:101128008BFF08BD2DE9F0478AB000240694079488
:1011380008940994474B9A6942F010029A619A6997
:1011480002F010020192019A9A6942F004029A612F
:101158009A6902F004020292029A9A6942F008021D
:101168009A619A6902F008020392039A9A6942F016
:1011780040029A619A6902F040020492049A9A69BC
:1011880042F020029A619B6903F020030593059BB6
:10119800DFF8C49001222021484601F0C5FDDFF8A0
:1011A800BC8001220421404601F0BEFD2C4F22469E
:1011B8004FF40041384601F0B7FD01260696DFF8E6
:1011C800A4A0CDF81CA00225089506A9384601F070
:1011D8008FFC12230693CDF81CA0089606A9384662
:1011E80001F086FC2023069307960894099506A922
:1011F800484601F07DFC0423069307960894099558
:1012080006A9404601F074FC4FF400430693079684
:101218000894099506A9384601F06AFC2246294631
:10122800062001F099F9062001F0A6F92246294680
:10123800072001F091F9072001F09EF9224629467E
:101248000A2001F089F90A2001F096F90AB0BDE8F0
:10125800F08700BF0010024000100140000C014060
:10126800000801400000111072B6FEE700B597B003
:10127800282200210CA808F02BFE002307930893CE
:1012880009930A930B930193029303930493059391
:10129800069309230C934FF480330D930122109287
:1012A80012920222139214934FF4E01315930CA890
:1012B80002F09CFDD8B90F2307930221089100235F
:1012C80009934FF480620A920B9307A802F0C0FFBB
:1012D80078B9112301934FF4007302930023069306
:1012E80001A803F091F830B917B05DF804FBFFF7D7
:1012F800BBFFFFF7B9FFFFF7B7FF000008B501F024
:10130800ADF8FFF7B3FF104800F022F8FFF70AFF27
:10131800FFF778FEFFF7C6FE00F060FA00F0B6FAB5
:1013280000F0F6F800F0CCFA06F01EFA08F0F8F82B
:1013380000F07EF800F040F900F054FE034808F091
:1013480083FC00F0F9FFFEE7140A0020201D0108C5
:1013580008B5054B1860054B18680023022219468A
:10136800806808F079FC08BD480800203401002096
:10137800022801D80120704708B508F04DFE09235E
:101388000360002008BD000010B5013801280AD804
:1013980014464FF0FF3392B20748006804F0EEFBA2
:1013A80040B9204610BD08F037FE092303604FF00E
:1013B800FF30F7E70520F5E748080020022801D8A4
:1013C8000020704708B508F027FE092303604FF096
:1013D800FF3008BD08B508F01FFE092303604FF071
:1013E800FF3008BD08B548B94FF0FF33012208485F
:1013F800006804F022FC40B9012008BD08F00CFE8A
:10140800092303604FF0FF30F7E70520F5E700BF39
:101418004808002008B5022804D84FF400534B6050
:10142800002008BD08F0F8FD09230360F8E7000074
:1014380000B583B00023ADF804308DF80630009372
:1014480019481A4B03604FF0FF3343604FF4807321
:10145800836003F0B1FAE8B900228DF804208DF812
:1014680005208DF8062001A90F4803F0A0F9A0B9BE
:1014780001238DF800308DF801308DF802300022FC
:101488008DF803206946084803F0F2F940B903B023
:101498005DF804FBFFF7E8FEDEE7FFF7E5FEE7E7A8
:1014A800FFF7E2FEF3E700BF4C08002000280040E9
:1014B8000268144B9A4200D0704700B583B002F01E
:1014C80079FC114BDA6942F00062DA61DB6903F0FA
:1014D80000630193019B0D4B0122C3F83C240022B9
:1014E8000321084601F038F8032001F045F80022EE
:1014F8000321292001F030F8292001F03DF803B03C
:101508005DF804FB00280040001002400000424241
:10151800054B064A1A6000225A609A60DA601A611E
:101528005A6104229A6170476008002000800140D7
:1015380030B589B000230493059306930793026896
:101548001A4B9A4201D009B030BD03F510435A69CD
:1015580042F480625A615A6902F480620192019AE7
:101568009A6942F010029A619A6902F01002029296
:10157800029A9A6942F020029A619B6903F020035B
:101588000393039B4FF48853049302250595032482
:10159800079404A9064801F0ABFA042304930595BF
:1015A800079404A9034801F0A3FACCE7008001409E
:1015B800001001400014014008B50E480E4B0360AE
:1015C8004FF48273436000238360C3600361436107
:1015D8004FF4007282610822C2610362436283622F
:1015E8000A23C36203F0F0FE00B908BDFFF73CFE12
:1015F800FBE700BFE40800200030014010B586B0CA
:10160800002302930393049305930268164B9A42AE
:1016180001D006B010BD03F560439A6942F48052C8
:101628009A619A6902F480520092009A9A6942F08B
:1016380004029A619B6903F004030193019BA023B0
:1016480002930223039303230593084C02A920461F
:1016580001F04EFA4023029300230393049302A956
:10166800204601F045FAD4E7003001400008014067
:1016780000B583B0124B9A6942F001029A619A69E7
:1016880002F001020092009ADA6942F08052DA61AF
:10169800DB6903F080530193019B0022114605206A
:1016A80000F05AFF052000F067FF064A536823F050
:1016B800E06343F00073536003B05DF804FB00BFC0
:1016C8000010024000000140FEE7FEE7FEE7FEE7EB
:1016D800FEE770477047704708B500F0D1FE08BDB7
:1016E80008B5024803F0C2F908BD00BF4C08002045
:1016F800704708B5012001F01DFB08BD08B50220A0
:1017080001F018FB08BD08B5102001F013FB08BD57
:1017180008B5024801F076F808BD00BF8809002026
:1017280008B5024802F008F908BD00BF10190020EA
:1017380008B5024803F007FF08BD00BF40090020B4
:1017480008B5024804F06AFB08BD00BF140A00206F
:1017580008B5024804F062FB08BD00BFCC090020B0
:1017680008B5024803F0F0F808BD00BF4C08002097
:101778000120704708B508F04FFC162303604FF0AE
:10178800FF3008BD08B54FF0FF31FFF7F3FFFEE764
:1017980010B503460C4A0D490D48006840B10C4885
:1017A80000680344521A934206D8094A136010BDD0
:1017B8000748084C0460F2E708F02EFC0C2303608D
:1017C8004FF0FF30F3E700BF0000012000040000E5
:1017D8003C090020181F00207047000000B587B0A2
:1017E80000230293039304930593009301931548F0
:1017F800154A026047224260836040F2E732C260C5
:101808000361836103F0A8FF90B94FF480530293FA
:1018180002A90C4803F0D8FF68B90023009301938C
:101828006946084804F050F840B907B05DF804FB71
:10183800FFF71AFDE9E7FFF717FDEEE7FFF714FDDD
:10184800F3E700BF400900200008004002680E4B83
:101858009A4200D0704700B583B003F50233DA69C5
:1018680042F00402DA61DB6903F004030193019B8F
:10187800002201211E2000F06FFE1E2000F07CFED9
:1018880003B05DF804FB00BF0008004008B50A4833
:101898000A4B03604FF4E133436000238360C36065
:1018A80003610C2242618361C36104F037F900B916
:1018B80008BDFFF7D9FCFBE7140A002000380140F7
:1018C80008B50A480A4B03604FF4E133436000232C
:1018D8008360C36003610C2242618361C36104F0C9
:1018E8001DF900B908BDFFF7BFFCFBE7CC090020D4
:1018F8000048004070B588B0002304930593069310
:1019080007930368404A934204D0404A934248D020
:1019180008B070BD04463E4B9A6942F480429A6111
:101928009A6902F480420092009A9A6942F004028D
:101938009A619B6903F004030193019B4FF40073C0
:1019480004930223059303230793324E04A93046D8
:1019580001F0CEF84FF480630493002505950695B1
:1019680004A9304601F0C4F82B482C4B03604560AD
:1019780085608023C360056145618561C56100F0AC
:101988001DFE58B9244BE3635C6200220321252025
:1019980000F0E2FD252000F0EFFDB9E7FFF764FC59
:1019A800F0E71B4BDA6942F48022DA61DA6902F463
:1019B80080220292029A9A6942F008029A619B690F
:1019C80003F008030393039B4FF4806304930223FB
:1019D800059303250795124E04A9304601F088F8AF
:1019E8004FF40063049300240594069404A9304638
:1019F80001F07EF822462946272000F0ADFD272079
:101A080000F0BAFD84E700BF0038014000480040FC
:101A180000100240000801408809002058000240D8
:101A2800000C0140034B044A1A60044B023A1A6046
:101A3800704700BF700F0020000002606C0F00208C
:101A48000B4B2A225A812B229A812C221A8100229E
:101A58009A71F0221A804FF4A0725A80054B1B68C5
:101A680036221A80044B1B6808221A80704700BF70
:101A78005C0F00206C0F0020700F002070B5174E0F
:101A88003468174DB5F80AC0A4F800C0154C4FEAE1
:101A9800102CD4F800E0AEF800C0C0B2D4F800C0F2
:101AA800ACF8000020684FEA122CA0F800C02068AB
:101AB800D2B202803268A88910802268080A108091
:101AC8002268C9B211802268190A11802268DBB223
:101AD800138033682A891A8070BD00BF6C0F0020FC
:101AE8005C0F0020700F002010B504460A4B1A88BE
:101AF8005B88013B013A9BB292B200210846FFF78E
:101B0800BDFF002303E0054A126814800133B3F5D2
:101B1800963FF8D310BD00BF5C0F0020700F002067
:101B28000020704700207047002070472DE9F843D7
:101B38008046894616461F46BDF82050BDF8244009
:101B48001EE0194A12681580013B002B08DB41FA98
:101B580003F212F0010FF4D0134A12681480F3E76D
:101B680002301F2806DC335C3218517841EA032121
:101B78000F23EAE708F110082036B8F1E00F11DC6E
:101B88003B46013FBFB26BB11FFA88F01FFA89F1DB
:101B980001F10F0300F10F029BB292B2FFF76EFF43
:101BA8000020DEE7BDE8F883700F00202DE9F84338
:101BB8008046894616461F46BDF82050BDF8244089
:101BC8001AE0174A12681580013B002B08DB41FA1E
:101BD80003F212F0010FF4D0114A12681480F3E7EF
:101BE8000130472802DC315C0723EEE708F11808CA
:101BF8004836B8F1D80F11DC3B46013FBFB26BB194
:101C08001FFA88F01FFA89F101F1170300F1170292
:101C18009BB292B2FFF732FF0020E2E7BDE8F883FB
:101C2800700F00202DE9F8438046894616461F4666
:101C3800BDF82050BDF824401AE0174A12681580F4
:101C4800013B002B08DB41FA03F212F0010FF4D03C
:101C5800114A12681480F3E701307F2802DC315CF6
:101C68000723EEE708F120088036B8F1D00F11DC21
:101C78003B46013FBFB26BB11FFA88F01FFA89F1EA
:101C880001F11F0300F11F029BB292B2FFF7F6FEAB
:101C98000020E2E7BDE8F883700F00202DE9F04747
:101CA80007468A4690461D46BDF82060104608F053
:101CB800E9F95FFA80F900242DE0B8B21FFA8AF139
:101CC800CB1D421D9BB292B2FFF7D8FE18F8040054
:101CD8002038C000002111E0144B1B681D800CF156
:101CE800FF3CBCF1010F08DD42FA0CF313F0010FC1
:101CF800F2D00E4B1B681E80F1E70131072905DC85
:101D080043180B4AD25C4FF0070CEAE70637E92F75
:101D18000ADC0134E4B24C4506D218F90430002B31
:101D2800CBDA0134E4B2F1E7BDE8F087700F0020A8
:101D3800E04F01082DE9F04F83B007468A469046E8
:101D48001C46BDF83050104608F09CF95FFA80F93F
:101D5800002633E0B8B21FFA8AF101F10F03C21D61
:101D68009BB292B2FFF78AFE18F8060020380001ED
:101D7800002116E0234B1B681C800CF1010C1FFA94
:101D88008CFCBCF1070F0AD8CCF1070342FA03F325
:101D980013F0010FEED01B4B1B681D80EDE70131DE
:101DA80089B20F2905D84318174AD25C4FF0000CA6
:101DB800E7E708370136F6B2E82F20DC4E451ED299
:101DC80008EB060118F90630002BC3DA14220F4875
:101DD800FFF7A6FE834610B90236F6B2ECE7019586
:101DE8000094C0F34F13094A51463846FFF79EFE48
:101DF80007EB5B0706EB1B1B5FFA8BF6DCE703B010
:101E0800BDE8F08F700F0020F04901085C0A00203F
:101E18002DE9F04F85B08046039191461C46BDF8E8
:101E28003850104608F02EF95FFA80FB002637E09C
:101E38001FFA88F0BDF80C1001F1170300F10B022E
:101E48009BB292B2FFF71AFE19F80630203B03EB5B
:101E58004303284F07EB0317002011E0264A1268B6
:101E68001480013B9BB2032B08D941FA03F212F00C
:101E7800010FF3D0204A12681580F2E7023080B2D1
:101E88002F2806D83B5C3A18517841EA03210F23E2
:101E9800E9E708F10C080136F6B2B8F1E40F26DCE0
:101EA8005E4524D209EB060119F90630002BBFDA8A
:101EB80014221248FFF736FE074610B90236F6B26A
:101EC800EBE70F4BA3FB003A01950094CAF30F13FD
:101ED8000A4A03994046FFF769FE0A4BA3FB0737F6
:101EE80008EB570806EBDA0A5FFA8AF6D5E705B079
:101EF800BDE8F08F50380108700F00205C0A002000
:101F0800398EE338ABAAAAAA2DE9F04F83B08046F0
:101F18008B4617461C46BDF83050104608F0B2F8FC
:101F28005FFA80F9002634E01FFA88F01FFA8BF177
:101F380001F11F0300F10F029BB292B2FFF79EFD61
:101F4800BB5D203B244A02EB831C00200FE0234AA0
:101F580012681480013B002B08DB41FA03F212F0EF
:101F6800010FF4D01D4A12681580F3E702303F28AC
:101F780008DC1CF800300CEB0002517841EA032120
:101F88000F23E8E708F110080136F6B2B8F1E40FBC
:101F98001EDC4E451CD2B919BB57002BC4DA1422DB
:101FA8000F48FFF7C1FD824610B90236F6B2EDE7D9
:101FB80001950094C0F3CF13094A59464046FFF7EC
:101FC80031FE08EB9A0806EB9A1A5FFA8AF6DDE703
:101FD80003B0BDE8F08F00BFD0200108700F0020CB
:101FE8005C0A00202DE9F04F83B0FFF71BFDA64DDA
:101FF8002B68CF221A80A54B1A68002414801A680F
:10200800C9211180196830220A802968ED200880CA
:10201800196864200880196803200880196812204C
:1020280008801968812008802968E82008801968D4
:1020380085200880196810270F8019687A20088081
:102048002968CB20088019683920088019682C2055
:10205800088019680C8019683420088019680220E3
:1020680008802968F720088019684FF02009A1F82E
:1020780000902968EA20088019680C8019680C808B
:102088002968C020088019681B2008802968C12099
:10209800088019680C802968C520088019680A809A
:1020A80019680A802A68C72111801A68B721118027
:1020B8002A684FF03608A2F800801A6808261680A9
:1020C8002A683A2111801A68552111802A68B1219D
:1020D80011801A6814801A681A2111802A68B6219A
:1020E80011801A680A2111801A68A22010802A68B3
:1020F800F22010801A6814802A68262010801A6836
:102108004FF0010EA2F800E02A68E020108018685D
:102118000F22028018684FF02A0AA0F800A0186859
:102128004FF0280CA0F800C01868068018684FF017
:102138000E0CA0F800C01868068018684FF0540C00
:10214800A0F800C018684FF0A90CA0F800C01868E3
:102158004FF0430CA0F800C01868018019680A8085
:1021680019680C8019680C8019680C8019680C8033
:102178002968E120088019680C80196815200880F2
:1021880019681720088019680720088019684FF017
:10219800110BA1F800B019680620088019684FF0E3
:1021A8002B0CA1F800C019685620088019683C203B
:1021B800088019680520088019680F8019680A8046
:1021C80018683F21018018680180186802802A6811
:1021D800A2F800C01A6814801A6814801A68A2F855
:1021E80000E01A6811802A68A2F800A01A68148012
:1021F8001A6814801A6814801B68EF221A802B68EA
:10220800A3F800B0782000F04DF92B6829221A8035
:10221800FFF716FC1E4AD36843F40043D3604FF41B
:102228007840FFF761FCC82000F03CF94FF4FC60EF
:10223800FFF75AFCC82000F035F91F20FFF754FCBF
:10224800C82000F02FF94FF6FF70FFF74DFCC820AB
:1022580000F028F94FF4784500954FF6FF730D4AC2
:1022680021462046FFF766FDDFF82CA000954FF6C3
:10227800FF7352462146A020FFF710FD4FF6FF7569
:1022880000952346524609E06C0F0020700F00208D
:1022980000080140341D01084C1D01083146A020EA
:1022A800FFF7FCFC4FF4FC6300932B460C4A3946BD
:1022B8002046FFF73FFD1F2300932B46094A494656
:1022C8002046FFF7A5FD4BF6404300932B46064AF0
:1022D80041462046FFF718FE03B0BDE8F08F00BF67
:1022E8005C1D0108741D01088C1D0108FFF774FAB4
:1022F8000B480C490C4A002302E0D458C45004335C
:10230800C4188C42F9D3094A094C002301E0136030
:102318000432A242FBD307F085FEFEF7EFFF7047B9
:1023280000000020DC070020C8550108DC07002059
:10233800141F0020FEE7704770B5A0B04FF6FF707D
:10234800FFF7D2FB2A4B1B78012B13D04FF47844AC
:1023580000944FF6FF73274A00210846FFF758FDFF
:1023680000944FF6FF73244A00210846FFF750FDFA
:1023780020B070BD4FF4FC6400944FF6FF731F4A01
:1023880000210846FFF744FD00944FF6FF731C4AEE
:1023980019210020FFF73CFD1A4E706DFEF746FA32
:1023A8000546B06DFEF742FA2946FDF719FF4FF0D2
:1023B8006A51FDF715FF4FF06A51FDF711FFFEF75F
:1023C80027F902460B46104902A807F017FD0094AA
:1023D8004FF6FF7302AA31210020FFF719FD009480
:1023E8004FF6FF73094A49210020FFF711FDBFE7A7
:1023F80044080020EC1D0108001E0108A41D010866
:10240800B81D010860080020CC1D0108DC1D01086A
:1024180010B504460E4B1A784FF47A73B3FBF2F3F7
:102428000C4A1068B0FBF3F000F0B4F868B90F2C50
:1024380001D901200AE0002221464FF0FF3000F0C8
:102448008BF8054B1C60002000E0012010BD00BF88
:1024580004000020000000200800002008B5074AFA
:10246800136843F010031360032000F063F80020A2
:10247800FFF7CEFFFFF7FCF8002008BD0020024060
:10248800034A1168034B1B780B441360704700BF65
:10249800740F002004000020014B1868704700BF2B
:1024A800740F002038B50446FFF7F6FF0546B4F16F
:1024B800FF3F02D0044B1B781C44FFF7EDFF401B85
:1024C800A042FAD338BD00BF04000020002808DB72
:1024D8000901C9B200F1604000F5614080F80013BD
:1024E800704700F00F000901C9B2014B1954704739
:1024F80014ED00E000B500F00700C0F1070CBCF1D6
:10250800040F28BF4FF0040C031D062B0FD9C31E60
:102518004FF0FF3E0EFA0CF021EA000199400EFA46
:1025280003FE22EA0E0241EA02005DF804FB0023E2
:10253800EEE70000074AD36823F4E0631B041B0C92
:10254800000200F4E060034343F0BF6343F4003348
:10255800D360704700ED00E010B50446054BD8681D
:10256800C0F30220FFF7C6FF01462046FFF7AEFF83
:1025780010BD00BF00ED00E0002807DB00F01F02DF
:10258800400901239340024A42F82030704700BFB7
:1025980000E100E00138B0F1807F0BD24FF0E0237A
:1025A8005861054AF02182F823100020986107221B
:1025B8001A6170470120704700ED00E0002838D00C
:1025C80010B4024601681C4B994227D81B4B0B4498
:1025D8001B48A0FB03031B099B001364194BD3631F
:1025E800022382F8213008686FF30D10536894684D
:1025F8002343D468234314692343546923439469C8
:102608002343D469234303430B60002090630123D1
:1026180082F8213082F8200010BC70470A4B0B4426
:102628000748A0FB03031B099B001364074BD363F4
:10263800D6E70120704700BF07040240F8FFFDBF3E
:10264800CDCCCCCC00000240F8FBFDBF000402401A
:10265800034690F82120D2B2022A06D004228263CF
:10266800002280F820200120704701680A6822F0C3
:102678000E020A6001680A6822F001020A60026C10
:10268800C06B012101FA02F2426083F82110002098
:1026980083F820007047000008B590F82130DBB2BD
:1026A800022B03D004238363012008BD026813684A
:1026B80023F00E0313600268136823F0010313600C
:1026C80003684C4A93424ED9783A934224D0143244
:1026D800934230D0143293422FD0143293422FD0E9
:1026E800143293422FD0143293422FD01432934293
:1026F8002FD002F5627293422ED0143293422DD01D
:10270800143293422CD01432934202D04FF48032C8
:1027180003E04FF4805200E00122374B5A60012356
:1027280080F82130002380F82030436B002B5ED0E6
:1027380098470020B9E71022EFE74FF48072ECE7E2
:102748004FF48052E9E74FF48032E6E74FF4801205
:10275800E3E74FF08072E0E70122DEE71022DCE7D2
:102768004FF48072D9E7254A934224D01432934219
:1027780025D01432934224D01432934224D01432F8
:10278800934224D01432934224D01432934224D05A
:1027980002F56272934223D01432934222D014324B
:1027A800934221D01432934202D04FF4803203E096
:1027B8004FF4805200E00122114B5A60AFE710221B
:1027C800FAE74FF48072F7E74FF48052F4E74FF4DA
:1027D8008032F1E74FF48012EEE74FF08072EBE7BA
:1027E8000122E9E71022E7E74FF48072E4E70020CE
:1027F8005BE700BF8000024000040240080002407E
:102808000000024038B5C36B1A6804682568016C7B
:1028180004238B40134200F09B8015F0040F00F056
:102828009780236813F0200F03D1236823F0040353
:10283800236003689A4A934246D9783A934224D04F
:102848001432934228D01432934227D01432934240
:1028580027D01432934227D01432934227D014320F
:10286800934227D002F56272934226D014329342E3
:1028780025D01432934224D01432934202D04FF41C
:10288800802203E04FF4804200E00422854B5A6026
:10289800C36A03B1984738BD4022F7E74FF4806216
:1028A800F4E74FF48042F1E74FF48022EEE74FF46B
:1028B8008002EBE74FF08062E8E70422E6E7402277
:1028C800E4E74FF48062E1E7774A934224D0143278
:1028D800934225D01432934224D01432934224D008
:1028E8001432934224D01432934224D014329342A7
:1028F80024D002F56272934223D01432934222D03C
:102908001432934221D01432934202D04FF48022E1
:1029180003E04FF4804200E00422644B5A60B7E7BA
:102928004022FAE74FF48062F7E74FF48042F4E779
:102938004FF48022F1E74FF48002EEE74FF0806217
:10294800EBE70422E9E74022E7E74FF48062E4E797
:1029580002238B40134200F0AB8015F0020F00F009
:10296800A780236813F0200F06D1236823F00A03F9
:102978002360012380F821300368494A93424BD9E8
:10298800783A934224D0143293422DD01432934291
:102998002CD0143293422CD0143293422CD01432BF
:1029A80093422CD0143293422CD002F56272934297
:1029B8002BD0143293422AD01432934229D01432A5
:1029C800934202D04FF4003203E04FF4005200E08B
:1029D8000222344B5A60002380F82030836A002B8F
:1029E8003FF459AF984756E72022F2E74FF40072B8
:1029F800EFE74FF40052ECE74FF40032E9E74FF409
:102A08000012E6E74FF00072E3E70222E1E7202236
:102A1800DFE74FF40072DCE7234A934224D01432F4
:102A2800934225D01432934224D01432934224D0B6
:102A38001432934224D01432934224D01432934255
:102A480024D002F56272934223D01432934222D0EA
:102A58001432934221D01432934202D04FF4003200
:102A680003E04FF4005200E00222104B5A60B2E734
:102A78002022FAE74FF40072F7E74FF40052F4E728
:102A88004FF40032F1E74FF40012EEE74FF0007216
:102A9800EBE70222E9E72022E7E74FF40072E4E7D8
:102AA800800002400004024008000240000002408A
:102AB80008238B4013423FF4EEAE15F0080F3FF4A5
:102AC800EAAE236823F00E032360026CC16B012376
:102AD80003FA02F24A60836380F82130002380F809
:102AE8002030036B002B3FF4D6AE9847D3E600BFE7
:102AF80070B582B00024A446ABE0854DAB4214D03B
:102B08000CD8A5F58015AB420FD005F57025AB4262
:102B18000BD0A5F58015AB4210D106E07D4DAB4238
:102B280003D005F58035AB4208D18B68002B5AD00D
:102B3800012B53D04261082400E0CC68BEF1FF0F9E
:102B480053D806464FEA8C0233680F25954023EA8E
:102B5800050304FA02F2134333604B6813F0805FF5
:102B680075D06D4B9A6942F001029A619B6903F036
:102B780001030193019B4FEA9C02951C674B53F894
:102B880025600CF00305AD000F23AB4026EA0306D1
:102B9800634B984230D003F58063984200F09680EA
:102BA80003F58063984200F0938003F580639842B0
:102BB80000F0908003F58063984200F08D8003F563
:102BC8008063984216D0062317E0CC680434B5E732
:102BD800CC680834B2E7CC680C34AFE7026108244B
:102BE800ACE70024AAE70424A8E7061DACF1080214
:102BF8009200A9E7052300E00023AB4033430232EB
:102C0800464D45F822304B6813F4801F66D0454A7C
:102C1800936843EA0E0393604B6813F4001F63D074
:102C2800404AD36843EA0E03D3604B6813F4003F6D
:102C380060D03C4A536843EA0E0353604B6813F470
:102C4800803F5DD0374A136843EA0E0313600CF1E6
:102C5800010C0B6833FA0CF258D0012202FA0CF27C
:102C680003EA020E32EA0303F1D14B68122B3FF656
:102C780044AF122B3FF662AF01A555F823F000BF11
:102C8800332B0008432B0008D92B0008EB2B000836
:102C9800452B0008452B0008452B0008452B00084C
:102CA800452B0008452B0008452B0008452B00083C
:102CB800452B0008452B0008452B0008452B00082C
:102CC800452B0008D32B0008DF2B0008012394E7CD
:102CD800022392E7032390E704238EE7114A9368BF
:102CE80023EA0E03936097E70E4AD36823EA0E039C
:102CF800D3609AE70B4A536823EA0E0353609DE7B3
:102D0800084A136823EA0E031360A0E702B070BDF7
:102D180000002210000031100010024000000140A5
:102D280000080140000401400AB10161704709042C
:102D38000161704708B5054B5B69034200D108BDC6
:102D4800024B5861FFF7F7FAF9E700BF00040140AA
:102D580038B512F4804F44D00468B4F850309BB2B0
:102D680091F800C003EBCC03023304EB4304B4F83E
:102D78000044C4F309048B69A34228D31B1B8B614D
:102D88008B697BB9056835F82C309BB223F48043F6
:102D980023F0700383F4005343F4004343F08003AB
:102DA80025F82C3012F0400F0ED002680D7832F85A
:102DB80025309BB223F4E04323F0700343F400432F
:102DC80043F0C00322F8253024B9204638BD00233B
:102DD8008B61D5E723460A894969006804F0ACFC91
:102DE800F3E70468B4F850309BB291F800C003EBE5
:102DF800CC03063304EB4304B4F80044C4F30904D9
:102E08008B69A3422FD31B1B8B618B697BB9056828
:102E180035F82C309BB223F4804323F0700383F4FD
:102E2800005343F4004343F0800325F82C3012F09C
:102E3800400F0FD1026891F800C032F82C309BB2D5
:102E480023F4E04323F0700343F4004343F0C0034A
:102E580022F82C30002CB8D023464A8949690068EA
:102E680004F06AFCB1E700238B61CEE770B586B049
:102E7800002800F08180044690F8A932EBB10323C2
:102E880084F8A932206803F0E6FC254655F8106B53
:102E9800EC460FCDACE80F002B68CCF80030231DB2
:102EA8000ECB304603F0C7FC054658B1022384F820
:102EB800A9320125284606B070BD80F8A83206F070
:102EC8005DFCDCE70021206803F0CFFC2B4616E010
:102ED8005A1C02EB820104EBC1010120487002EB8D
:102EE800820104F8313004EBC1000021C17003EB0A
:102EF800830004EBC0008163C1630164D3B26168DD
:102F08008B42E5D316E005EB850304EBC3030022EF
:102F180083F8692183F8685183F86B21C3F8782115
:102F2800C3F87C2105EB850304EBC303C3F88021B8
:102F38000135EDB2A942E6D8254655F8106BEC46A6
:102F48000FCDACE80F002B68CCF80030231D0ECB5A
:102F5800304603F08CFC054620B1022384F8A932E0
:102F68000125A7E7002384F82430012384F8A93237
:102F7800206803F0DFFF9DE701259BE738B590F84F
:102F8800A832012B11D00446012580F8A852006808
:102F980003F058FC2946204606F005FD206803F09A
:102FA800C7FF002084F8A80238BD0220FCE770B5EE
:102FB80005460C46164612F0400F00F00E810268D6
:102FC800B2F850309BB2097803EBC103023302EB2D
:102FD8004302B2F80024C2F30902A36993424ED90E
:102FE8009B1AA361A369002B66D16378002B49D192
:102FF8002B68B3F8502092B2134403EB0113B3F8D3
:103008000424C2F30902A3F80424B3F804246FEAE1
:1030180042426FEA524292B2A3F804242B686278C3
:10302800002A3CD1B3F8502092B21344227803EB23
:103038000213B3F80C24C2F30902A3F80C24B3F862
:103048000C246FEA42426FEA524292B2A3F80C246F
:103058002178284606F0C6FB16F4804F41D02A682E
:10306800217832F821309BB223F4E04323F0700337
:1030780043F4404343F0800322F8213031E0002339
:10308800A361AFE7012BC9D12B68B3F8502092B2E6
:10309800134403EB01130022A3F80424BEE7012A1A
:1030A800D6D1B3F8502092B21344227803EB02131E
:1030B8000022A3F80C24CBE716F4804F0DD0286823
:1030C80030F821309BB223F4E04323F0700343F43B
:1030D800404343F0800320F8213094F82430012B3A
:1030E80012D02A68217832F821309BB223F4E043C9
:1030F80023F0400383F0300343F4004343F080039C
:1031080022F82130002070BD636913446361E369CC
:103118001344E361216A2369994224D3C91A2162BD
:103128006278002A44D12A68B2F8501089B20A4459
:10313800217802EB0112B2F80414C1F30901A2F8D4
:1031480004143E2B1BD9580913F01F0F00D1013866
:10315800B2F8041489B2800280B2014341F40041FC
:10316800A2F8041426E021B9002384F82430134679
:10317800D6E7002384F8243023620B46D0E74BB906
:10318800B2F804146FEA41416FEA514189B2A2F8DA
:1031980004140FE0590813F0010F00D00131B2F800
:1031A800040480B2890289B20143A2F8041401E040
:1031B800012A06D09BB222896169286803F0C2FE01
:1031C8008FE72A68B2F8501089B20A44217802EBD6
:1031D800011299B2A2F80414ECE70268B2F8503070
:1031E8009BB2097803EBC103063302EB4302B2F842
:1031F8000024C2F30902A36993424FD39B1AA36127
:10320800A369002B67D16378002B4AD12B68B3F8E8
:10321800502092B2134403EB0113B3F80424C2F311
:103228000902A3F80424B3F804246FEA42426FEABF
:10323800524292B2A3F804242B686278002A3DD146
:10324800B3F8502092B21344227803EB0213B3F878
:103258000C24C2F30902A3F80C24B3F80C246FEA77
:1032680042426FEA524292B2A3F80C2421782846CF
:1032780006F0B8FA16F4804F7FF433AF2A68217845
:1032880032F821309BB223F4E04323F0700343F477
:10329800404343F0800322F8213022E70023A36152
:1032A800AEE7012BC8D12B68B3F8502092B2134473
:1032B80003EB01130022A3F80424BDE7012AD5D1AA
:1032C800B3F8502092B21344227803EB0213002281
:1032D800A3F80C24CAE716F4804F0DD1286830F8FB
:1032E80021309BB223F4E04323F0700343F44043BE
:1032F80043F0800320F8213094F82430012B7FF428
:10330800F0AE636913446361E3691344E361216ABE
:103318002369994224D3C91A21622A68617800294D
:1033280043D1B2F8501089B20A44217802EB011255
:10333800B2F80C14C1F30901A2F80C143E2B1BD9E6
:10334800580913F01F0F00D10138B2F80C1489B2D4
:10335800800280B2014341F40041A2F80C1426E037
:1033680021B9002384F824301346D6E700232362CA
:1033780084F824300B46D0E74BB9B2F80C146FEA46
:1033880041416FEA514189B2A2F80C140FE0590883
:1033980013F0010F00D00131B2F80C0480B2890299
:1033A80089B20143A2F80C1401E0012906D09BB2AE
:1033B80062896169286803F0C5FD92E6B2F8501089
:1033C80089B20A44217802EB011299B2A2F80C14CE
:1033D800EDE72DE9F04105462868B0F8443013F4CC
:1033E800004F00F09282B0F84440A3B214F00F04EA
:1033F80040F0E28013F0100F6BD003889AB213F4F8
:10340800006F40F09D8012F4004FE5D0038823F050
:1034180070031B051B0D43F0800303802868B0F878
:1034280050309BB295F8682103EBC203063300EBDA
:103438004303B3F80034C3F30903C5F884318BB1EF
:10344800D5F87C1171B1B5F86E2104F075F9D5F88D
:103458007C31D5F884211344C5F87C3100212846F5
:1034680006F0B4F92A68138899B213F4006FB3D13F
:1034780001F44051B1F5405FAED0B2F850309BB284
:103488001A44B2F80C34C3F30903A2F80C34D5F883
:1034980078313E2B77D9590913F01F0F00D1013924
:1034A800B2F80C349BB2890289B20B4343F400434F
:1034B800A2F80C342A6813889BB223F4804323F0C3
:1034C800700383F4405343F4004343F080031380B4
:1034D80082E703889BB223F4E14323F070036FEA89
:1034E80043436FEA53439BB203802A68B2F85030D3
:1034F8009BB295F8281003EBC103023302EB430299
:10350800B2F80034C3F309036B64EA6B1A44EA6344
:103518000021284606F066F995F82430002B3FF480
:103528005BAF2B6C002B7FF457AF95F824302A68DB
:1035380043F08003A2F84C30002385F824304BE791
:10354800B0F850309BB295F8682103EBC2030633FC
:1035580000EB4303B3F80034C3F30903C5F884311F
:10356800B5F86E2105F52C7104F0E6F82A68138881
:1035780023F070031B051B0D43F0800313802846BE
:1035880006F01CF928E74BB9B2F80C346FEA43434C
:103598006FEA53439BB2A2F80C348BE7590813F037
:1035A800010F00D00131B2F80C3498B28B029BB2F3
:1035B8000343A2F80C347DE730F824309EB213F4AC
:1035C800004F4CD116F0800F3FF406AF621C02EB9F
:1035D800820105EBC101286830F824309BB223F43E
:1035E800E14323F070036FEA43436FEA53439BB20E
:1035F80020F82430CB78012B00F0F28016F4807F7D
:1036080040F07E812868B0F850309BB2621C02EB13
:10361800820215F8326003EBC603023300EB430362
:10362800B3F80034C3F3090304EB840205EBC202C8
:10363800126C9A4240F24C8104EB840705EBC707F1
:10364800D21A3A6404EB840205EBC202126C002A17
:1036580040F045813146284606F0C4F8BCE630F80B
:10366800243023F070031B051B0D43F0800320F862
:10367800243004EB8401C90001F5B47105EB01089D
:1036880004EB840305EBC30393F87431002B42D198
:103698002868B0F850309BB204EB840205EBC202F4
:1036A80092F8682103EBC203063300EB4303B3F837
:1036B8000074C7F3090717BB04EB840305EBC303C6
:1036C800D3F884213A44C3F88421D3F87C213A44BE
:1036D800C3F87C21D3F880313BB104EB840305EBBC
:1036E800C303D3F878319F4275D204EB840305EB0A
:1036F800C30393F86811284606F068F862E704EBFC
:10370800840105EBC1013B46B1F86E21D1F87C116B
:1037180004F012F8D0E704EB840305EBC30393F835
:103728006B31022B35D0296804EB840205EBC20209
:1037380092F8680131F820309BB223F4E04323F07B
:10374800700343F4004343F0C00321F82030286895
:1037580092F8682130F8223013F4804F20D0B0F866
:1037680050309BB203EBC203023300EB4303B3F8C0
:103778000074C7F30907002F9ED004EB840105EB02
:10378800C1013B46B1F87021D1F87C1103F0D4FF98
:1037980092E7324641462846FFF7DAFA07468BE7B2
:1037A800B0F850309BB203EBC203063300EB43037F
:1037B800B3F80074C7F30907002F3FF47DAF04EB9B
:1037C800840105EBC1013B46B1F87221D1F87C11A7
:1037D80003F0B2FF70E74146286803F0C6FBF1E644
:1037E80004EB840305EBC30300221A6493F8343016
:1037F800FBB116F0400F37D04B781BBB2B68B3F8E2
:10380800502092B21344621C02EB820215F8322057
:1038180003EB0213B3F80424C2F30902A3F8042447
:10382800B3F804246FEA42426FEA524292B2A3F814
:103838000424013404EB840415F83410284605F0F8
:10384800D1FFC9E5012BF4D12B68B3F8502092B20F
:103858001344621C02EB820215F8322003EB0213B8
:103868000022A3F80424E4E72A68631C03EB83031B
:1038780005EBC3035B78D3B9B2F850309BB213445D
:10388800621C02EB820215F8322003EB0213B3F834
:103898000C24C2F30902A3F80C24B3F80C246FEA31
:1038A80042426FEA524292B2A3F80C24C1E7012BBC
:1038B800BFD1B2F850309BB21344621C02EB8202B3
:1038C80015F8322003EB02130022A3F80C24B0E70A
:1038D80004EB840205EBC20200271764B2E604EB8E
:1038E800840205EBC202D66B1E44D663526C04EB0D
:1038F800840405EBC4041344636403F036FB6BE5EE
:1039080032462846FFF753FB66E50020BDE8F08104
:1039180090F8A832012B0DD010B50446012380F889
:10392800A83280F82410006803F0FCFA002084F81C
:10393800A80210BD0220704710B584B00446006884
:1039480003F0FAFA10F4004F20D110F4806F21D15F
:1039580010F4804F2FD110F4005F37D110F4805F3E
:103968003ED110F4006F40F0878010F4007F40F0E3
:10397800AE8010F4807F27D02268B2F844309BB222
:1039880023F480739BB2A2F844301DE02046FFF771
:1039980020FD19E02268B2F844309BB223F480631A
:1039A8009BB2A2F84430204605F02DFF00212046A6
:1039B800FFF7AEFF08E02268B2F844309BB223F468
:1039C80080439BB2A2F8443004B010BD2268B2F81C
:1039D80044309BB223F400539BB2A2F84430F3E77F
:1039E8002268B2F840309BB223F004039BB2A2F8DD
:1039F80040302268B2F840309BB223F008039BB2F3
:103A0800A2F84030204605F021FF2268B2F8443081
:103A18009BB223F480539BB2A2F84430D4E72268C7
:103A280032F8231004AA02EB430222F8101C0133D7
:103A3800DBB2072BF3D92268B2F840309BB243F0CF
:103A48000103A2F840302268B2F840309BB223F05C
:103A580001039BB2A2F840302368B3F8442012F463
:103A6800806FF9D0B3F8442092B222F4806292B207
:103A7800A3F8442000230BE00023DAE7226804A916
:103A880001EB430131F8101C22F823100133DBB29B
:103A9800072BF3D92268B2F840309BB243F00803F1
:103AA800A2F840302268B2F844309BB223F4006395
:103AB8009BB2A2F844302268B2F840309BB243F07F
:103AC8000403A2F84030204605F0B0FE7CE72268E7
:103AD800B2F844309BB223F400739BB2A2F844308E
:103AE800204605F08AFE6FE710B50446084611F037
:103AF800800F25D101F0070C0CEB8C01C90001F5F2
:103B0800B47E04EB0E010CEB8C0C04EBCC0C4FF0E8
:103B1800000E8CF869E100F0070008700A61CB70AC
:103B2800022B1AD094F8A832012B19D0012384F85B
:103B3800A832206802F0B0FE002084F8A80210BD68
:103B480001F0070C0CF1010C0CEB8C0104EBC1012A
:103B58004FF0010E81F801E0DDE700230B71E1E78A
:103B68000220ECE710B504460B4611F0800F1FD178
:103B780001F0070202EB8201C90001F5B4710144AA
:103B880002EB820200EBC202002082F8690103F016
:103B980007030B7094F8A832012B13D0012384F883
:103BA800A832206803F05DF8002084F8A80210BD50
:103BB80001F00702013202EB820100EBC101012092
:103BC8004870E4E70220F2E710B501F0070C0CEBAF
:103BD8008C01C90001F5B4710CEB8C0E00EBCE0E14
:103BE800CEF87C21CEF880310024CEF884418EF8BE
:103BF80069418EF868C10144006803F0B6F92046AF
:103C080010BD01F0070101EB810100EBC100D0F804
:103C18008401704738B501F0070404F1010C0CEB7E
:103C28008C0104EB840E00EBCE0ECEF83C20CEF8CF
:103C3800403001228EF84C20CEF848300025CEF8CE
:103C4800445000EBC1035A7000F83140194600682F
:103C580003F08BF9284638BD38B501F007054268EE
:103C6800954231D804460B4611F0800F1ED101EB66
:103C78008101C90001F5B471014403EB830300EB32
:103C8800C303002283F8692101238B700D7094F817
:103C9800A832012B1AD0012384F8A832206803F037
:103CA800CBF85DB1002084F8A80238BD6B1C03EB8B
:103CB800830100EBC10101224A70E5E704F52C718C
:103CC800206803F03DF9EDE70120EEE70220ECE77C
:103CD8000B4601F00F014268914230D810B50446F6
:103CE80013F0800F21D103F0070202EB8201C90013
:103CF80001F5B471014402EB820200EBC20200201C
:103D080082F8690100228A7003F007030B7094F8A7
:103D1800A832012B15D0012384F8A832206803F0BB
:103D2800B0F8002084F8A80210BD03F007020132A1
:103D380002EB820100EBC10101204870E2E701209B
:103D480070470220F0E790F8A832012B14D010B584
:103D58000446012380F8A83211F0800F06D10068CC
:103D680002F098FD002084F8A80210BD01F00701B8
:103D7800006802F08DFDF5E70220704711F0800F12
:103D88000BD001F00701013101EB810100EBC1000B
:103D980052B90273C3800020704701EB8101C9004A
:103DA80001F5B4710844F3E70122027303811B0C87
:103DB8004381F0E7014B01221A62704700000E426E
:103DC80082B0084B1B68084AA2FB03235B0A00FB6E
:103DD80003F3019300BF019B5A1E0192002BF9D1F6
:103DE80002B0704700000020D34D6210002800F098
:103DF800F18170B582B00446036813F0010F2CD02E
:103E0800994B5B6803F00C03042B1DD0964B5B6841
:103E180003F00C03082B12D06368B3F5803F41D040
:103E2800002B55D103F1804303F504331A6822F4BB
:103E380080321A601A6822F480221A6037E08A4BAE
:103E48005B6813F4803FE7D0874B1B6813F4003F8F
:103E580003D06368002B00F0BF81236813F0020FC2
:103E680075D0814B5B6813F00C0F5FD07E4B5B689D
:103E780003F00C03082B54D02369002B00F08A8030
:103E88007A4B01221A60FEF707FB0546764B1B6842
:103E980013F0020F75D1FEF7FFFA401B0228F5D97F
:103EA80003209EE1704A136843F48033136063680B
:103EB80043B3FEF7F1FA05466B4B1B6813F4003F5A
:103EC800CBD1FEF7E9FA401B6428F5D9032088E135
:103ED800B3F5A02F09D0644B1A6822F480321A6017
:103EE8001A6822F480221A60E1E703F18043A3F5FF
:103EF8003C331A6842F480221A601A6842F480320D
:103F08001A60D4E7FEF7C8FA0546574B1B6813F446
:103F1800003FA2D0FEF7C0FA401B6428F5D9032061
:103F28005FE1514B5B6813F4803FA5D14E4B1B6892
:103F380013F0020F03D02369012B40F04F814A4A46
:103F4800136823F0F803616943EAC1031360236827
:103F580013F0080F33D0A369002B5CD0434B012228
:103F6800C3F88024FEF798FA05463F4B5B6A13F0C6
:103F7800020F21D1FEF790FA401B0228F5D9032041
:103F88002FE1394A136823F0F803616943EAC10352
:103F98001360DCE7354B00221A60FEF77DFA054610
:103FA800314B1B6813F0020FD1D0FEF775FA401B96
:103FB8000228F5D9032014E10120FFF701FF236847
:103FC80013F0040F00F09680274BDB6913F0805F35
:103FD80034D1254BDA6942F08052DA61DB6903F0AB
:103FE80080530193019B0125214B1B6813F4807FAB
:103FF80026D0E368012B3DD0002B53D103F1804339
:1040080003F504331A6A22F001021A621A6A22F0CE
:1040180004021A6233E0154B0022C3F88024FEF72D
:104028003BFA0546104B5B6A13F0020FC7D0FEF748
:1040380033FA401B0228F5D90320D2E00025D3E744
:104048000B4A136843F480731360FEF725FA06469B
:10405800074B1B6813F4807FCBD1FEF71DFA801B3A
:104068006428F5D90320BCE0001002400000424259
:10407800007000405F4A136A43F001031362E3686B
:1040880033B3FEF709FA06465A4B1B6A13F0020FC0
:104098002FD1FEF701FA801B41F288339842F3D9F9
:1040A80003209EE0052B09D0524B1A6A22F0010228
:1040B8001A621A6A22F004021A62E0E74D4B1A6A81
:1040C80042F004021A621A6A42F001021A62D6E742
:1040D800FEF7E2F90646474B1B6A13F0020F08D0B9
:1040E800FEF7DAF9801B41F288339842F3D90320AE
:1040F80077E0E5B9E369002B72D03E4A526802F0D6
:104108000C02082A56D0022B17D03B4B00221A6605
:10411800FEF7C2F90446374B1B6813F0007F47D0FF
:10412800FEF7BAF9001B0228F5D9032059E0314AF5
:10413800D36923F08053D361DCE72F4B00221A6642
:10414800FEF7AAF905462B4B1B6813F0007F06D033
:10415800FEF7A2F9401B0228F5D9032041E0236AA3
:10416800B3F5803F1AD023494B6823F47413226AAD
:10417800606A024313434B601F4B01221A66FEF725
:104188008BF904461B4B1B6813F0007F0ED1FEF71A
:1041980083F9001B0228F5D9032022E0154A536849
:1041A80023F40033A1680B435360DCE7002018E0D8
:1041B800002016E0012B16D00E4B5B6803F480310B
:1041C800226A914211D103F47013626A93420ED1AC
:1041D800002006E001207047012002E0012000E0F5
:1041E800002002B070BD0120FBE70120F9E70120A3
:1041F800F7E700BF00100240000042420F4B5B6827
:1042080003F00C02082A01D00D487047C3F383421B
:104218000C49885C13F4803F0BD0084B5B68C3F3F0
:104228004043094AD35C064A02FB00F0B0FBF3F0B6
:104238007047064B03FB00F0704700BF00100240B8
:1042480000127A00DC520108D852010800093D002A
:10425800002800F0A08070B50D460446524B1B683C
:1042680003F007038B420BD24F4A136823F007036E
:104278000B431360136803F007038B4240F08D80F3
:10428800236813F0020F17D013F0040F04D0474A25
:10429800536843F4E0635360236813F0080F04D0B5
:1042A800424A536843F460535360404A536823F0CA
:1042B800F003A1680B435360236813F0010F31D05A
:1042C8006368012B20D0022B25D0384A126812F0DF
:1042D800020F64D035494A6822F0030213434B6049
:1042E800FEF7DAF80646314B5B6803F00C036268A8
:1042F800B3EB820F16D0FEF7CFF8801B41F288335C
:104308009842F0D9032045E0284A126812F4003F89
:10431800E0D101203EE0254A126812F0007FD9D191
:10432800012037E0204B1B6803F00703AB420AD992
:104338001D4A136823F007032B431360136803F027
:104348000703AB422DD1236813F0040F06D0174A98
:10435800536823F4E063E1680B435360236813F068
:10436800080F07D0114A536823F46053216943EAC0
:10437800C1035360FFF742FF0C4B5B68C3F30313A1
:104388000B4AD35CD8400B4B18600B4B1868FEF7F0
:104398003FF8002070BD012070470120FAE7012096
:1043A800F8E70120F6E700BF0020024000100240B5
:1043B800C02001080000002008000020014B1868F8
:1043C800704700BF0000002008B5FFF7F7FF044B57
:1043D8005B68C3F30223034AD35CD84008BD00BF1F
:1043E80000100240B820010808B5FFF7E7FF044BAA
:1043F8005B68C3F3C223034AD35CD84008BD00BF3F
:1044080000100240B820010870B582B00446036865
:1044180013F0010F36D03F4BDB6913F0805F49D1B1
:104428003C4BDA6942F08052DA61DB6903F0805371
:104438000193019B0125384B1B6813F4807F3BD007
:10444800344B1B6A13F4407313D0626802F4407251
:104458009A420ED02F4A136A23F440702F4901263E
:10446800C1F840640026C1F84064106213F0010FDF
:1044780036D1284A136A23F4407361680B431362E8
:10448800002D3ED1236813F0020F06D0214A53684D
:1044980023F44043A1680B435360236813F0100FC3
:1044A80034D01C4A536823F4800361690B4353607A
:1044B80000202CE00025BEE7174A136843F48073F8
:1044C8001360FDF7E9FF0646134B1B6813F4807F62
:1044D800B6D1FDF7E1FF801B6428F5D9032016E06B
:1044E800FDF7DAFF06460B4B1B6A13F0020FC0D12B
:1044F800FDF7D2FF801B41F288339842F3D903209D
:1045080005E0D36923F08053D361BBE7002002B0F4
:1045180070BD00BF00100240007000400000424221
:1045280008B501380F2863D8DFE800F03557622F47
:104538006262623262626262626262082F4B5A6829
:10454800186810F0807054D0C2F383432C49C85CBB
:1045580012F4803F15D0294B5B68C3F34043294AC6
:10456800D25C294BB3FBF2F303FB00F0234B5B68EF
:1045780013F4800F3DD14000244BA3FB00304008CA
:1045880037E0234B03FB00F0F0E7FFF737FE30E09E
:10459800FFF734FE2DE0194B1B6A40F202321A4035
:1045A800B2F5817F26D003F44073B3F5007F04D0C1
:1045B800B3F5407F09D000201BE0104A526A12F080
:1045C800020FF5D049F6404013E00C4B186810F480
:1045D80000300ED04FF224400BE0FFF705FF074BE9
:1045E8005B68C3F3813301335B00B0FBF3F000E099
:1045F800002008BD4FF40040FBE700BF0010024058
:10460800F0520108EC52010800127A00ABAAAAAADB
:1046180000093D0000B5036899691FFA81FED86951
:104628009A691FFA82FCE64505D0D86980B240EA4B
:1046380002405DF804FB80B240EA0140F9E70368F4
:10464800186A5B6A9BB243EA00407047030903EBB0
:10465800830300F00F0000EB4300C0B27047000076
:1046680000F5FA6C022921D801EB4103C1EBC30123
:104678001E4BA3FB013102EB5103634400F2CF70E0
:1046880003EB90031A4AA2FB0020A3EB501303EBA1
:10469800D01304331748A0FB03201A1A00EB52006A
:1046A8008008C0EBC000181AC0B2704701EB410384
:1046B800C1EBC3010D4BA3FB013102EB5103634472
:1046C80003EB9C030A4AA2FB0C12A3EB521303EB65
:1046D800D21302330748A0FB03201A1A00EB52003A
:1046E8008008C0EBC000181ADEE700BF398EE33837
:1046F8001F85EB512549922438B50446FDF7CCFEB9
:10470800054623685A6812F0200F07D1FDF7C4FE4A
:10471800401BB0F57A7FF4D9032004E05A6842F0D0
:1047280010025A60002038BD38B504460268536844
:1047380023F010035360FDF7AFFE054623685B685E
:1047480013F0200F07D1FDF7A7FE401BB0F57A7FC5
:10475800F4D9032000E0002038BD38B505460C46E2
:10476800FFF7CAFF08B1012038BD2B68220C9A61F7
:104778002B68A4B2DC612846FFF7D6FF0028F3D0E7
:104788000120F1E738B505460C46FFF7B5FF08B13B
:10479800012038BD2B68220C1A622B68A4B25C6217
:1047A8002846FFF7C1FF0028F3D00120F1E770B5D4
:1047B800002857D00D460646002955D0037C012B0A
:1047C80054D00123037402234374BAB90B784C788C
:1047D800C4EB0414A4004FF4616202FB03448B7819
:1047E8001C4421463046FFF7B8FF0546C8B10423EC
:1047F8007374002333740125284670BD0878FFF7C9
:1048080025FF4FF4616303FB00F46878FFF71EFF90
:10481800C0EB001004EB8004A878FFF717FF0444EE
:10482800DFE73268536823F0050353603046FFF72B
:1048380006FFB0F1FF3F01D0844204D8012373740E
:1048480000233374D8E700F5A83101F5C07130466C
:10485800FFF798FF0028F1D0042373740023337402
:104868000125C9E70125C7E70125C5E70225C3E7F3
:1048780000285AD038B50D460446002957D0037C85
:10488800012B56D00123037402234374BAB9CB78A1
:10489800C3734B7843738B788373A27B617BE07B14
:1048A800FFF7DEFE207328702046FFF7B3FE224B89
:1048B800984211D8012363740020207438BDC87849
:1048C800FFF7C4FEE0736878FFF7C0FE6073A8784E
:1048D800FFF7BCFEA073E0E7184DA5FB00352D0CD3
:1048E800174B03FB150529462046FFF736FF28B16D
:1048F80004236374002323740120DFE72046FFF7B5
:104908009EFEB0F1FF3FD5D08542D3D900F5A8313E
:1049180001F5C0712046FFF735FF0028CAD00423EF
:104928006374002323740120C8E701207047012025
:10493800C4E70220C2E700BF8F5F010007452EC20F
:10494800805101007047000010B5044603681A68DA
:1049580012F0020F03D05B6813F0020F06D1074B69
:104968004FF400325A610123637410BDFFF7EAFF68
:104978002268536823F002035360F0E70004014003
:10498800C0B138B505460268536823F00803536080
:10499800FDF782FD04462B685B6813F0080F07D10A
:1049A800FDF77AFD001BB0F57A7FF4D9032000E00B
:1049B800002038BD01207047002850D010B50446AB
:1049C800437C4BB1022363742046FFF7D9FF38B10B
:1049D80004236374012010BD0374FCF769FDF1E73B
:1049E8002046FFF789FE28BB2268536823F0070397
:1049F8005360A36823B11B4A136B23F001031363AD
:104A0800184AD36A23F46073A1680B43D3626368BE
:104A1800B3F1FF3F12D02268C3F3034191602268CB
:104A28009BB2D3602046FFF77FFE88B104236374EE
:104A38000120D0E7042363740120CCE70120FFF7AD
:104A48006FFD08B1431EE6E7042363740120C2E743
:104A58000023E37301236373A3736374BBE701202B
:104A6800704700BF006C00407047704703681A68C1
:104A780012F0010F1CD010B504465A6812F0010F4D
:104A880010D05B6813F0040F0DD0FFF7EEFF23681A
:104A98006FF004025A60042363742268536823F099
:104AA8000103536010BDFFF7DFFF01236374F4E7D0
:104AB8007047000070B582B0044600230193006877
:104AC80001F0D9FB054610B1284602B070BD206838
:104AD80001F09AFE38B90123A364A36C012B0BD013
:104AE8002E46284614E00023A364206801F0C3FB87
:104AF8000028F2D00546E7E70021206801F022FDF2
:104B08000028EDD04FF08055DEE7019B013301937B
:104B1800019A4FF6FE739A4213D896B9002120687D
:104B280001F010FDE0B91249206801F0B9FD064610
:104B3800C0B90021206801F089FBC30FE5D01E46EB
:104B4800E3E7019A4FF6FE739A420ED810F08043BD
:104B580002D001236364B7E7002262641D46B3E70D
:104B68000546B1E74FF08055AEE74FF08075ABE7EB
:104B7800000010C170B581B104460E46016D0904EC
:104B8800006801F0F7FC054608B1284670BD002111
:104B9800206801F05BFB3060F7E74FF00065F4E751
:104BA8002DE9F04F87B005460C4616469B46DDF8C2
:104BB80040A0FDF771FC002C36D0814695F8347082
:104BC800FFB2012F40F005810023AB6306EB0B0316
:104BD800EA6D93422ED8032385F834302B680022DF
:104BE800DA626B6C012B00D076024FF0FF33009332
:104BF8004FEA4B230193902302930223039300234C
:104C08000493012305936946286801F022FBBBF150
:104C1800010F14D902232B633146286801F018FCD0
:104C2800A0B9DDF8048038E0AB6B43F00063AB63F8
:104C38000127D3E0AB6B43F00073AB63CEE00123F5
:104C48002B633146286801F0EBFBE9E72B68654ADE
:104C58009A63AB6B0343AB63012385F834300023BD
:104C68002B63BBE0286801F0CEFA2070C0F307235D
:104C78006370C0F30743A370000EE0700434A8F11A
:104C880004080136072EEDD9FDF706FCA0EB090054
:104C9800504510D2BAF1000F0DD02868466B40F28B
:104CA8002A331E4015D1436B13F4004FECD0B8F1F2
:104CB800000FE9D0E6E72B684A4A9A63AB6B43F0EA
:104CC8000043AB63012385F8343000232B630327AB
:104CD80084E0436B13F4807F05D0BBF1010F02D948
:104CE8006B6C032B38D12B685A6B12F0080F44D128
:104CF8005A6B12F0020F4CD15A6B12F0200F54D19C
:104D08002868436B13F4001F5BD0B8F1000F58D02C
:104D180001F079FA2070C0F307236370C0F30743EA
:104D2800A370000EE0700434A8F10408FDF7B4FB8A
:104D3800A0EB0900504502D2BAF1000FE0D12B6870
:104D4800284A9A63AB6B43F00043AB63012385F8B1
:104D5800343000232B6341E001F0C2FB03460028F6
:104D6800C1D02A681F499163AA6B1343AB6301231F
:104D780085F8343000232B6330E01A4A9A63AB6B12
:104D880043F00803AB63012385F8343000232B6319
:104D980024E0144A9A63AB6B43F00203AB6301232C
:104DA80085F8343000232B6318E00E4A9A63AB6B06
:104DB80043F02003AB63012385F8343000232B63D1
:104DC8000CE040F23A538363012385F8343000271E
:104DD80004E0AB6B43F00053AB630127384607B0E0
:104DE800BDE8F08FFF0540002DE9F04F8BB0054678
:104DF8000C4616469B46DDF850A0FDF74DFB002CEF
:104E080037D0804695F83470FFB2012F40F0E28029
:104E18000023AB6306EB0B03EA6D93422FD8032301
:104E280085F834302B680022DA626B6C012B00D0D5
:104E380076024FF0FF3304934FEA4B2305939023F8
:104E480006930023079308930123099304A928686C
:104E580001F0FFF9BBF1010F16D920232B6331466E
:104E6800286801F025FB0190019BABB9DDF814908F
:104E780040E0AB6B43F00063AB630127AFE0AB6B83
:104E880043F00073AB63AAE010232B633146286814
:104E980001F0F6FA0190E7E72B68534A9A63AB6B87
:104EA800019A1343AB63012385F8343000232B6345
:104EB80095E023780393627843EA02230393A27868
:104EC80043EA02430393E27843EA02630393043418
:104ED800A9F1040903A9286801F098F90136072EF9
:104EE800E7D9FDF7D9FAA0EB0800504510D2BAF17E
:104EF800000F0DD02868466B40F21A331E4015D1BA
:104F0800436B13F4804FECD0B9F1000FE9D0E6E71A
:104F18002B68354A9A63AB6B019A1343AB63012341
:104F280085F8343000232B63032758E0436B13F4D0
:104F3800807F05D0BBF1010F02D96B6C032B18D110
:104F48002B685A6B12F0080F24D15A6B12F0020F1B
:104F58002CD15A6B12F0100F34D0234A9A63AB6BE2
:104F680043F01003AB63012385F8343000232B632F
:104F780035E001F0B5FA03460028E1D02A681A495D
:104F88009163AA6B1343AB63012385F83430002384
:104F98002B6324E0144A9A63AB6B43F00803AB63BA
:104FA800012385F8343000232B6318E00E4A9A63F6
:104FB800AB6B43F00203AB63012385F83430002365
:104FC8002B630CE040F23A529A63012385F834309F
:104FD800002704E0AB6B43F00053AB63012738466E
:104FE8000BB0BDE8F08F00BFFF0540000346426EDE
:104FF800920F0A70426EC2F383624A7090F867207B
:1050080002F003028A7090F86620CA7090F8652052
:105018000A7190F864204A71826E120DCA80B0F845
:105028006A2002F00F020A72826EC2F3C0324A721C
:10503800826EC2F380328A72826EC2F34032CA72C2
:10504800826EC2F300320A7300224A73426C002A4D
:1050580040F08680806E40F6FC7202EA8002D86ECC
:1050680042EA90720A61DA6EC2F3C2620A7593F874
:105078006F2002F007024A75DA6EC2F342528A754F
:10508800DA6EC2F38242CA75DA6EC2F3C2320A76A7
:105098000A6901325A65087E00F007000230824032
:1050A8005A6591F808C00CF00F0C012000FA0CF0BA
:1050B8009865400A00FB02F2DA654FF400721A663E
:1050C800DA6EC2F380324A76DA6EC2F3C6128A7694
:1050D800DA6E02F07F02CA761A6FD20F0A771A6F59
:1050E800C2F341724A771A6FC2F382628A771A6FE3
:1050F800C2F38352CA771A6FC2F3405281F8202054
:10510800002081F82100B3F8722002F0010281F832
:1051180022201A6FC2F3C03281F823201A6FC2F31B
:10512800803281F824201A6FC2F3403281F825209A
:105138001A6FC2F3003281F826201A6FC2F3812257
:1051480081F827201A6FC2F3012281F828201B6FEB
:10515800C3F3460381F82930012381F82A307047C8
:10516800012A11D1826E120402F47C12B0F86E008A
:1051780002430A610A69013292025A65DA654FF4FC
:1051880000729A651A669BE7026805499163826B0B
:1051980042F080528263012083F83400704700BFD8
:1051A800FF05400070B590B004460123ADF81230F9
:1051B800006801F034F800286CD0636C032B45D1EB
:1051C800636C032B5DD1636C032B1DD0BDF81210EB
:1051D80021650904206801F028FA054600285BD1FA
:1051E8000021206801F032F860660421206801F08F
:1051F8002DF8A0660821206801F028F8E0660C2147
:10520800206801F023F820670421206801F01EF8C7
:10521800000DE06405A92046FFF7E8FE00283ED10E
:10522800226D12040023206801F074F9054698BB2A
:10523800234653F8106B93E807008DE80700043401
:1052480094E80E00304600F0C5FF25E0206801F024
:10525800D7F9054600BB0021206800F0F7FF60671A
:105268000421206800F0F2FFA0670821206800F000
:10527800EDFFE0670C21206800F0E8FFC4F880002B
:105288009EE70DF11201206801F074FA0546002826
:1052980099D001E04FF08065284610B070BD4FF0FE
:1052A8008055F9E770B58AB0044600230493059346
:1052B800069307930893762309930AAB13E907002B
:1052C8008DE8070004AB0ECB206800F083FF18B10F
:1052D800012528460AB070BD05461A4E0023C6F8B7
:1052E800A030206800F097FF0123C6F8A030022004
:1052F800FDF7D8F82046FFF7DDFB30B1012584F82B
:105308003450A36B0343A363E3E72046FFF74AFF48
:1053180030B1012584F83450A36B0343A363D8E765
:105328004FF40071206801F063F80028D1D0236899
:1053380005499963A36B0343A363012584F834509B
:10534800C7E700BF00003042FF054000A8B110B514
:10535800044690F8343063B1032384F8343020468F
:10536800FFF7A0FF58B9A0632063012384F8343005
:1053780010BD0377FCF7DCF8EEE701207047012049
:10538800F6E7436C0B60836C4B60C36C8B60036DFA
:10539800CB60436D0B61836D4B61C36D8B61036E95
:1053A800CB610020704710B582B0044600230193FA
:1053B80001A9FFF7DFFB10B1A36B0343A3630198B7
:1053C800C0F3432002B010BD002856D010B50446E3
:1053D800436A33B94368B3F5827F05D00023C361BC
:1053E80002E00023036143610023A36294F8513073
:1053F800002B3CD0022384F851302268136823F034
:1054080040031360636803F48273A26802F40442E1
:105418001343E26802F400621343226902F00202B5
:105428001343626902F001021343A26902F4007295
:105438001343E26902F038021343226A02F0800241
:105448001343A26A02F40052216813430B60638B72
:10545800226803F0040353602268D36923F40063CD
:10546800D36100206065012384F8513010BD84F8B1
:1054780050302046FCF7C2F8BCE70120704760B303
:1054880070B50E46154604468369B3F5807F26D06D
:1054980090F84130E3B1214651F8080B00F000FEC6
:1054A800A2683146206800F02FFE236BA2682946C7
:1054B800606800F051FE2268A16852F8213043F07C
:1054C800010342F82130012384F84130002070BDE7
:1054D80080F84030FBF722FEDDE70120704701200D
:1054E800F5E710B4036A046A24F0010404628469CD
:1054F80024F0F00C4CEA021223F00A030B438261F9
:10550800036210BC704710B4036A046A24F01004E4
:105518000462846924F4704C4CEA023223F0A0033C
:1055280043EA01138261036210BC7047836823F069
:1055380070030B4343F0070383607047704770475D
:1055480070477047704710B5044603681A6912F02F
:10555800020F11D0DA6812F0020F0DD06FF00202BC
:105568001A610123037703689B6913F0030F70D056
:10557800FFF7E6FF0023237723681A6912F0040F68
:1055880012D0DA6812F0040F0ED06FF004021A611C
:105598000223237723689B6913F4407F5FD020465A
:1055A800FFF7CEFF0023237723681A6912F0080F4C
:1055B80012D0DA6812F0080F0ED06FF008021A61E4
:1055C800042323772368DB6913F0030F4ED02046AA
:1055D800FFF7B6FF0023237723681A6912F0100F2C
:1055E80012D0DA6812F0100F0ED06FF010021A61A4
:1055F800082323772368DB6913F4407F3DD02046D6
:10560800FFF79EFF0023237723681A6912F0010F22
:1056180003D0DA6812F0010F36D123681A6912F044
:10562800800F03D0DA6812F0800F34D123681A692A
:1056380012F0400F03D0DA6812F0400F32D123681D
:105648001A6912F0200F03D0DA6812F0200F30D157
:1056580010BDFFF774FF2046FFF773FF8AE7204667
:10566800FFF76DFF2046FFF76CFF9BE72046FFF72B
:1056780066FF2046FFF765FFACE72046FFF75FFFB0
:105688002046FFF75EFFBDE76FF001021A61204672
:10569800FFF754FFC1E76FF080021A61204600F05F
:1056A80052F9C3E76FF040021A612046FFF74AFF3C
:1056B800C5E76FF020021A61204600F043F9C7E7FA
:1056C8000368244A904212D002F5006290420ED03C
:1056D800B0F1804F0BD0A2F59832904207D002F576
:1056E8008062904203D002F58062904203D123F099
:1056F80070034A681343174A904212D002F50062B9
:1057080090420ED0B0F1804F0BD0A2F59832904263
:1057180007D002F58062904203D002F58062904281
:1057280003D123F44073CA68134323F080034A6902
:10573800134303608B68C3620B688362054B98420E
:1057480003D003F50063984201D10B690363012379
:1057580043617047002C014040B310B5044690F8EF
:105768003D30F3B1022384F83D30214651F8040B53
:10577800FFF7A6FF012384F8463084F83E3084F80A
:105788003F3084F8403084F8413084F8423084F85F
:10579800433084F8443084F8453084F83D300020A4
:1057A80010BD80F83C30FCF751F8DBE7012070476A
:1057B80010B4846824F47F4C42EA03220A4342EA84
:1057C8000C02826010BC704790F83C30012B78D0F6
:1057D80010B50446012380F83C30022380F83D30A0
:1057E8000268936823F47F4323F0770393600B6880
:1057F800602B4CD023D8402B54D011D8202B03D069
:105808000AD80BB1102B05D119462068FFF78EFE78
:10581800002028E0012026E0302BF5D0012022E0EE
:10582800502B0AD1CA6849680068FFF75AFE502110
:105838002068FFF77BFE002015E0012013E0B3F598
:10584800805F3AD0B3F5005F14D0702B37D1CB68A6
:105858004A6889680068FFF7ABFF2268936843F0DD
:10586800770393600020012384F83D30002384F8F7
:105878003C3010BDCB684A6889680068FFF798FF1C
:105888002268936843F4804393600020EBE7CA687A
:1058980049680068FFF737FE60212068FFF746FE79
:1058A8000020E0E7CA6849680068FFF71AFE40214F
:1058B8002068FFF73BFE0020D5E70020D3E7012052
:1058C800D1E702207047000090F83C20012A34D02C
:1058D80010B40346012280F83C20022280F83D20C3
:1058E80002685068946820F0700C086840EA0C0060
:1058F80050601A681248824212D000F50060824255
:105908000ED0B2F1804F0BD0A0F59830824207D06C
:1059180000F58060824203D000F58060824204D1A5
:1059280024F08004496821439160012283F83D20D6
:10593800002083F83C0010BC70470220704700BF6D
:10594800002C014070477047026802F10C0353E8CD
:10595800003F23F490730C3242E800310029F3D160
:10596800026802F1140353E8003F23F001031432E4
:1059780042E800310029F3D1036B012B05D0202325
:1059880080F84230002303637047026802F10C0379
:1059980053E8003F23F010030C3242E8003100299D
:1059A800F3D1ECE790F84130DBB2212B01D0022093
:1059B80070478368B3F5805F17D0036A5A1C026288
:1059C8001A7803685A60C38C9BB2013B9BB2C384AC
:1059D8004BB90268D36823F08003D3600268D368A8
:1059E80043F04003D360002070470369002BE4D1E3
:1059F800036A1B880268C3F308035360036A02330F
:105A08000362E0E710B504460268136923F44053C3
:105A1800C1680B43136183680269134342691A43DF
:105A28000168CB6823F4B05323F00C031343CB6015
:105A38000268536923F4407381690B435361026818
:105A4800134B9A4220D0FEF7BFFC024602EB8202BB
:105A580002EB820263689B00B2FBF3F20D48A0FBE5
:105A680002314909642303FB11231B013233A0FBD4
:105A780003035B0903F0F00202EB011203F00F03CA
:105A8800216813448B6010BDFEF7AEFC0246DDE7CB
:105A9800003801401F85EB512DE9F84305460F46B4
:105AA80016469946DDF820802B681C6837EA0404FE
:105AB8000CBF01240024B4422DD1B8F1FF3FF3D02C
:105AC800B8F1000F05D0FCF7E7FCA0EB0900404552
:105AD800EAD92A6802F10C0353E8003F23F4D07393
:105AE8000C3242E800310029F3D12A6802F114038C
:105AF80053E8003F23F00103143242E80031002943
:105B0800F3D1202385F8413085F84230002385F809
:105B18004030032000E00020BDE8F88360B310B5F2
:105B2800044690F8413013B3242384F841302268A6
:105B3800D36823F40053D3602046FFF763FF22683D
:105B4800136923F4904313612268536923F02A03ED
:105B580053612268D36843F40053D3600020606423
:105B6800202384F8413084F84230606310BD80F807
:105B78004030FBF7BFFED7E7012070472DE9F04121
:105B880082B01E4690F84130DBB2202B4BD1044640
:105B98000D46904600294AD00AB9012044E0002366
:105BA8004364212380F84130FCF776FC0746A4F8CB
:105BB8002480A4F82680A368B3F5805F02D04FF054
:105BC80000080FE02369FBB14FF000080AE038F83D
:105BD800023B2268C3F308035360E28C92B2013A95
:105BE80092B2E284E38C9BB28BB100963B460022D2
:105BF80080212046FFF750FFD8B9002DE7D015F8CF
:105C0800012B23685A60E8E7A8460025EAE70096D2
:105C18003B46002240212046FFF73EFF58B920238B
:105C280084F8413000E0022002B0BDE8F081012094
:105C3800FAE70320F8E70320F6E72DE9F04182B000
:105C48001E4690F84230DBB2202B53D104460D4655
:105C58009046002952D00AB901204CE00023436441
:105C6800222280F842200363FCF716FC0746A4F8BA
:105C78002C80A4F82E80A368B3F5805F02D04FF083
:105C8800000817E0236913B14FF0000812E0A84696
:105C980000250FE023685B68C3F3080328F8023B7C
:105CA80003E023685B682B700135E28D92B2013AFC
:105CB80092B2E285E38D9BB2BBB100963B460022CF
:105CC80020212046FFF7E8FED0B9002DE2D0A368D6
:105CD800B3F5805FE5D013B92369002BE1D02368C1
:105CE8005B6803F07F032B70DEE7202384F84230E3
:105CF800002000E0022002B0BDE8F0810120FAE7B0
:105D08000320F8E7704708B50168CA6822F0400226
:105D1800CA60202280F84120FFF7F4FF002008BD68
:105D28007047704708B5406A0023C385C384FFF7EE
:105D3800F8FF08BD704790F84230DBB2222B69D1DA
:105D48008368B3F5805F4FD0826AB3F5805F04D073
:105D5800002B56D10369002B53D103685B6813707D
:105D6800836A01338362C38D9BB2013B9BB2C385B7
:105D7800002B51D100B583B00268D36823F020030B
:105D8800D3600268D36823F48073D36002685369D0
:105D980023F001035361202380F84230002343633A
:105DA800036B012B33D100230363026802F10C0358
:105DB80053E8003F23F010030C3242E80031002979
:105DC800F3D103681A6812F0100F06D0002201926E
:105DD8001A6801925B680193019B818DFFF7AAFF06
:105DE800002003B05DF804FB0269002AACD1826A86
:105DF80003685B68C3F308031380836A0233836212
:105E0800B1E703685B6803F07F031370A8E7FFF747
:105E180087FFE5E7022070470020704710B582B081
:105E2800044602681368D068516913F00F0F09D14E
:105E380013F0200F0CD010F0200F09D02046FFF7E8
:105E48007AFF16E011F0010115D110F4907F12D1FC
:105E5800216B012979D013F0800F03D010F0800F47
:105E680040F0138113F0400F03D010F0400F40F0C2
:105E7800108102B010BD13F0010F06D010F4807F1E
:105E880003D0626C42F00102626413F0040F04D084
:105E980019B1626C42F00202626413F0020F04D07E
:105EA80019B1626C42F00402626413F0080F07D063
:105EB80010F0200F00D119B1626C42F00802626440
:105EC800626C002AD5D013F0200F02D010F0200FFA
:105ED80029D123685B6903F04003626C12F0080F54
:105EE80000D163B32046FFF72FFD23685B6913F0E9
:105EF800400F20D0226802F1140353E8003F23F03A
:105F08004003143242E800310029F3D1E36B73B146
:105F1800624A5A63E06BFCF7BFFB0028A9D0E06B2C
:105F2800436B9847A5E72046FFF705FFD1E72046D2
:105F3800FFF7F7FE9DE72046FFF7F3FE99E72046B7
:105F4800FFF7EFFE0023636493E713F0100F82D08E
:105F580010F0100F3FF47FAF0023019313680193F3
:105F680053680193019B536913F0400F51D0E26BC2
:105F780013685B689BB2002B3FF47BAFA18D9942FD
:105F88007FF677AFE3859369202B37D0226802F13B
:105F98000C0353E8003F23F480730C3242E80031CD
:105FA8000029F3D1226802F1140353E8003F23F0DB
:105FB8000103143242E800310029F3D1226802F1CA
:105FC800140353E8003F23F04003143242E8003141
:105FD8000029F3D1202384F8423000232363226868
:105FE80002F10C0353E8003F23F010030C3242E89F
:105FF80000310029F3D1E06BFCF72AFB022363632D
:10600800A18DE38D9BB2C91A89B22046FFF792FE93
:106018002FE7A18DE38D9BB2C91A89B2E38D9BB29C
:10602800002B3FF426AF00293FF423AF226802F18A
:106038000C0353E8003F23F490730C3242E800301D
:106048000028F3D1226802F1140353E8003F23F03B
:106058000103143242E800300028F3D1202384F8E9
:10606800423000232363226802F10C0353E8003F07
:1060780023F010030C3242E800300028F3D1022349
:1060880063632046FFF756FEF3E62046FFF78AFCD7
:10609800EFE62046FFF737FEEBE600BF2D5D000870
:1060A80010B40A6850F8223023F0010340F8223077
:1060B8008B68082B24D000244A6822431343CA68FB
:1060C80013430A6913434A691343CA6913430A6AA3
:1060D80013434A6A13438A6A1343CA6A13430A6B0F
:1060E80013438A691A434B6B1A43096850F82140D5
:1060F800044B2340134340F82130002010BC704764
:106108004024D9E78000F0FF00B5013250F8223072
:1061180003F0404C0B68D1F804E043EA0E13D1F8C1
:1061280008E043EA0E23D1F80CE043EA0E43D1F825
:1061380010E00EF1FF3E43EA0E53D1F814E0AEF141
:10614800020E43EA0E6389690B434CEA030340F8E5
:10615800223000205DF804FBB3F5804F05D06FF0C6
:10616800704340F822300020704730B450F8223095
:10617800094C1C400B684D6843EA05138D6843EAD7
:1061880005238D692B43C96843EA01431C4340F842
:106198002240002030BC70470000F0CF0B4B1B683A
:1061A8000B4AA2FB03235B0A41F2883202FB03F38A
:1061B8001A46013B3AB1426B12F0800FF8D0C52362
:1061C8008363002070474FF00040704700000020B4
:1061D800D34D621084B00DF1040C8CE80E000B4610
:1061E8001343039A1343049A1343059A1343069AD5
:1061F8001343426822F4FD4222F07F0213434360B6
:10620800002004B07047D0F8800070470B68C0F8D1
:106218008030002070470323036000207047006827
:1062280000F0030070470B6883604B688A6813436B
:10623800CA6813430A691343C2686FF30B02134316
:10624800C360002070470069C0B2704714304058DE
:1062580070470B6843624B6883628B68CA68134354
:106268000A6913434A691343C26A22F0F7021343C7
:10627800C3620020704710B586B00446002301931E
:106288000293039304934FF48063059301A9FFF7E6
:10629800CAFF2046FFF782FF06B010BD38B5044696
:1062A8000D46504B1B685049A1FB03135B0A03FBC7
:1062B80002F21346013A002B5DD0636B13F0450FD1
:1062C800F7D013F4006FF4D1636B13F0040F06D109
:1062D800636B13F0010F05D00120A0634DE004208B
:1062E800A0634AE0C523A3632046FFF7ACFFA8429A
:1062F80001D0012041E000212046FFF7A7FF034617
:106308003A481840C8B3002B38DB13F0804F38D117
:1063180013F0005F37D113F0805F36D113F0006FB0
:1063280036D113F0806F36D113F0807F36D113F455
:10633800000F36D113F4800F36D113F4001F36D175
:1063480013F4801F36D113F4802F36D113F4003F95
:1063580036D113F4803F36D113F4004F36D113F4FD
:10636800804F36D113F4005F36D113F0080F36D0C2
:106378004FF4000001E04FF0004038BD4FF00070CE
:10638800FBE74020F9E78020F7E74FF48070F4E757
:106398004FF40070F1E74FF48060EEE74FF40060CF
:1063A800EBE74FF48050E8E74FF40050E5E74FF48F
:1063B8008040E2E74FF40040DFE74FF40030DCE7CD
:1063C8004FF48020D9E74FF40020D6E74FF480102F
:1063D800D3E74FF40010D0E74FF48000CDE74FF437
:1063E8008030CAE700000020D34D621008E0FFFDAE
:1063F80030B587B0044601911025029540230393D8
:10640800002304934FF48063059301A9FFF70BFF62
:1064180041F2883229462046FFF740FF07B030BDD9
:1064280030B587B0044601911125029540230393A6
:10643800002304934FF48063059301A9FFF7F3FE4B
:1064480041F2883229462046FFF728FF07B030BDC1
:1064580030B587B004460191122502954023039375
:10646800002304934FF48063059301A9FFF7DBFE33
:1064780041F2883229462046FFF710FF07B030BDA9
:1064880030B587B00446019118250295402303933F
:10649800002304934FF48063059301A9FFF7C3FE1B
:1064A80041F2883229462046FFF7F8FE07B030BD92
:1064B80030B587B00446019119250295402303930E
:1064C800002304934FF48063059301A9FFF7ABFE03
:1064D80041F2883229462046FFF7E0FE07B030BD7A
:1064E80030B587B00446002301930C25029540225D
:1064F800039204934FF48063059301A9FFF793FE79
:10650800034A29462046FFF7C9FE07B030BD00BF41
:1065180000E1F50530B587B00446019207250295DC
:1065280040230393002304934FF48063059301A948
:10653800FFF779FE41F2883229462046FFF7AEFE82
:1065480007B030BD30B587B00446019137250295B4
:1065580040230393002304934FF48063059301A918
:10656800FFF761FE41F2883229462046FFF796FE82
:1065780007B030BD30B587B0044601910D250295AE
:1065880040230393002304934FF48063059301A9E8
:10659800FFF749FE41F2883229462046FFF77EFE82
:1065A80007B030BD0146144B1B68144AA2FB0323F5
:1065B8005B0A41F2883202FB03F31A46013BBAB187
:1065C8004A6B12F0450FF8D012F4006FF5D14B6BFF
:1065D80013F0040F06D1486B10F0010005D1C52354
:1065E8008B63704704208863704701208863704775
:1065F8004FF00040704700BF00000020D34D6210EC
:1066080010B586B004460023019302220292C022EC
:10661800039204934FF48063059301A9FFF703FEE7
:106628002046FFF7BFFF06B010BD10B586B0044680
:10663800019109230293C0230393002304934FF489
:106648008063059301A9FFF7EEFD2046FFF7AAFF37
:1066580006B010BD0146104B1B68104AA2FB03236D
:106668005B0A41F2883202FB03F31A46013B82B10E
:106678004A6B12F0450FF8D012F4006FF5D1486B51
:1066880010F0040002D1C5238B637047042088638F
:1066980070474FF00040704700000020D34D621053
:1066A80010B586B0044641F0004141F480110191D3
:1066B8002923029340230393002304934FF4806318
:1066C800059301A9FFF7AFFD2046FFF7C3FF06B00A
:1066D80010BD0000F8B505460E461746234B1B684B
:1066E800234AA2FB03235B0A41F2883202FB03F32D
:1066F8001A46013B8AB36C6B14F0450FF8D014F4BA
:10670800006FF5D16B6B13F0040F06D16B6B13F0B0
:10671800010F05D00120A86321E00420A8631EE032
:106728002846FFF790FDB04201D0012017E0C523AD
:10673800AB6300212846FFF789FD034610F460404B
:1067480008D013F4804F0BD113F4004F0BD04FF443
:10675800805004E01B0C3B8001E04FF00040F8BD86
:106768004FF40050FBE74FF48030F8E700000020BA
:10677800D34D621070B586B004460D4600230193D0
:10678800032602964022039204934FF480630593F4
:1067980001A9FFF748FD2A4631462046FFF79AFF30
:1067A80006B070BD0146164B1B68164AA2FB0323B0
:1067B8005B0A41F2883202FB03F31A46013BE2B15D
:1067C8004A6B12F0450FF8D012F4006FF5D14B6BFD
:1067D80013F0040F0BD14B6B13F001030AD1486B74
:1067E80010F040000BD040228A63184670470420FE
:1067F800886370470120886370474FF000407047F6
:1068080000000020D34D621010B586B004464FF446
:10681800D573019308230293402303930023049321
:106828004FF48063059301A9FFF7FDFC2046FFF7AD
:10683800B9FF06B010BD84B001A880E80E000020A2
:1068480004B0704703460020A3F844004FF43F42C9
:10685800A3F840207047B0F8403023F47C535B0421
:106868005B0CA0F84030002070470020704784B0CF
:10687800844601A880E80E000123ACF840300020CF
:10688800ACF84000ACF84400ACF8500004B07047D5
:10689800002070470020704710B5034691F800C0EB
:1068A80030F82C2092B222F4EC4222F0700292B21C
:1068B800C878032861D8DFE800F0555C025800204A
:1068C80048F2800E42EA0E0223F82C2091F800C00C
:1068D80033F82C2092B222F4E04222F0700242EA0D
:1068E8000C0242EA0E0223F82C200A7B002A40F010
:1068F800DC804A78002A51D0B3F8502092B21A446A
:106908000C7802EB0412B1F806C04FEA5C0C4FEAAF
:106918004C0CA2F800C40C7833F8242012F0400F75
:106928000CD033F8242092B222F4E04222F0700214
:1069380042F4004242F0C00223F82420CA78012A17
:106948001DD0097833F8212092B222F4E04222F0D7
:10695800400282F0200242F4004242F0800223F812
:10696800212017E142F40072AAE742F4C062002035
:10697800A6E742F480620020A2E70120A0E7097898
:1069880033F8212092B222F4E04222F0400242F48D
:10699800004242F0800223F82120FBE0B3F85020A7
:1069A80092B21A440C7802EB0412B1F806C04FEA0E
:1069B8005C0C4FEA4C0CA2F808C4B3F8502092B211
:1069C8001A440C7802EB0412B2F80CC4CCF3090C8C
:1069D800A2F80CC40C693E2C39D94FEA541E14F0A5
:1069E8001F0F01D10EF1FF3EB2F80CC41FFA8CFC48
:1069F8004FEA8E2E1FFA8EFE4CEA0E0C4CF4004C19
:106A0800A2F80CC40C7833F8242012F4804F0CD070
:106A180033F8242092B222F4E04222F0700242F4C9
:106A2800404242F0800223F82420097869BB33F8F9
:106A3800212092B222F4804222F0700282F4405265
:106A480042F4004242F0800223F82120A2E04CB92F
:106A5800B2F80C446FEA44446FEA5444A4B2A2F872
:106A68000C44CFE74FEA540C14F0010F01D00CF19D
:106A7800010CB2F80C44A4B24FEA8C2C1FFA8CFC1F
:106A880044EA0C04A2F80C44BCE733F8212092B283
:106A980022F4804222F0700282F4005242F4004252
:106AA80042F0800223F8212074E0CA78022A72D0CA
:106AB8000C7833F8242092B222F4E24222F07002D9
:106AC80042F4004242F0800223F82420B3F8502018
:106AD80092B21A4491F800C002EB0C12B1F808C047
:106AE8004FEA5C0C4FEA4C0CA2F800C4B3F85020F3
:106AF80092B21A4491F800C002EB0C12B1F80AC025
:106B08004FEA5C0C4FEA4C0CA2F808C44A78002AF9
:106B180050D10C7833F8242012F4804F0CD033F87D
:106B2800242092B222F4E04222F0700242F4404261
:106B380042F0800223F824200C7833F8242012F045
:106B4800400F0CD033F8242092B222F4E04222F015
:106B5800700242F4004242F0C00223F8242091F867
:106B680000C033F82C2092B222F4804222F0700246
:106B780082F4405248F28004224323F82C200978FA
:106B880033F8212092B222F4E04222F0400222435C
:106B980023F8212010BD0C7833F8242092B222F477
:106BA800E04222F0700242F4014242F0800223F8EF
:106BB80024208BE70C7833F8242012F4804F0CD073
:106BC80033F8242092B222F4E04222F0700242F418
:106BD800404242F0800223F824200C7833F8242025
:106BE80012F0400F0CD033F8242092B222F4E04285
:106BF80022F0700242F4004242F0C00223F824203E
:106C0800CA78012A1ED00C7833F8242092B222F4D4
:106C1800E04222F0400282F0200242F4004242F0B8
:106C2800800223F82420097833F8212092B222F434
:106C3800804222F0700242F4004242F0800223F8BF
:106C48002120A7E70C7833F8242092B222F4E042FE
:106C580022F0400242F4004242F0800223F824204D
:106C6800E1E70B7B002B46D14B7813B30A7830F859
:106C7800223013F0400F0CD030F822309BB223F4AE
:106C8800E04323F0700343F4004343F0C00320F8CB
:106C980022300A7830F822309BB223F4E04323F004
:106CA800400343F4004343F0800320F822300020DF
:106CB80070470A7830F8223013F4804F0CD030F83F
:106CC80022309BB223F4E04323F0700343F44043A3
:106CD80043F0800320F822300A7830F822309BB243
:106CE80023F4804323F0700343F4004343F080030C
:106CF80020F82230DBE74B78002B4ED10A7830F8A9
:106D0800223013F4804F0CD030F822309BB223F499
:106D1800E04323F0700343F4404343F0800320F83A
:106D280022300A7830F8223013F0400F0CD030F8B7
:106D380022309BB223F4E04323F0700343F4004372
:106D480043F0C00320F822300A7830F822309BB292
:106D580023F4E04323F0700343F4004343F0C003FB
:106D680020F822300A7830F822309BB223F480438E
:106D780023F0700348F2800C43EA0C0320F8223019
:106D88000A7830F822309BB223F4E04323F0400322
:106D980043EA0C0320F8223089E70A7830F82230D9
:106DA80013F4804F0CD030F822309BB223F4E04328
:106DB80023F0700343F4404343F0800320F822306B
:106DC8000A7830F8223013F0400F0CD030F8223017
:106DD8009BB223F4E04323F0700343F4004343F0F1
:106DE800C00320F822300A7830F822309BB223F40E
:106DF800E04323F0700343F4404343F0800320F85A
:106E080022300A7830F822309BB223F4E04323F092
:106E1800400348F2800C43EA0C0320F822300A7839
:106E280030F822309BB223F4804323F0700343EA06
:106E38000C0320F822303AE74B788BB10A7830F807
:106E480022309BB223F4E04323F0400383F0100385
:106E580043F4004343F0800320F8223000207047B9
:106E68000A7830F822309BB223F4804323F0700371
:106E780083F4805343F4004343F0800320F8223026
:106E8800ECE70B7B002B4BD14B7833B30A7830F807
:106E9800223013F0400F0CD030F822309BB223F48C
:106EA800E04323F0700343F4004343F0C00320F8A9
:106EB8002230CB78012B33D00A7830F822309BB2BD
:106EC80023F4E04323F0400383F0200343F400431A
:106ED80043F0800320F8223022E00A7830F822308C
:106EE80013F4804F0CD030F822309BB223F4E043E7
:106EF80023F0700343F4404343F0800320F822302A
:106F08000A7830F822309BB223F4804323F07003D0
:106F180083F4405343F4004343F0800320F82230C5
:106F28000020704711B98023A0F84C30002070472A
:106F38000020704700207047B0F8440080B27047C6
:106F48000020704701335B0800EB420000F58060C9
:106F580008E00A7891F801C042EA0C2220F8042BD4
:106F68000231013B002BF4D1704770B505460C4641
:106F78004A78012A3BD00B7B002B40F0A6828B6914
:106F88000A69934240F284829B1A8B61B5F85030AB
:106F98009BB22B44217803EB0113B3F80C14C1F313
:106FA8000901A3F80C143E2A40F27682510912F026
:106FB8001F0F00D10139B3F80C2492B2890289B2AB
:106FC8000A4342F40042A3F80C24227835F8223010
:106FD8009BB223F4804323F0700383F4405343F4BB
:106FE800004343F0800325F82230002070BD8E69ED
:106FF80009698E4200D90E46237B73B3E378022BCE
:107008004DD0236A9B1B2362217835F8213013F079
:10701800400F00F0F581002A40F0E281B5F85030C9
:107028009BB22B4403EB0113B3F80C24C2F30902FF
:10703800A3F80C243E2E40F2BA81710916F01F0FF6
:1070480000D10139B3F80C2492B2890289B20A43FB
:1070580042F40042A3F80C24CBE1B6B23346E288EE
:1070680061692846FFF76EFFB5F850309BB22B4494
:10707800227803EB0213A3F80464227835F822304F
:107088009BB223F4E04323F0400383F0300343F43E
:10709800004343F0800325F822300020A6E7236A46
:1070A800994280F06681227835F822309BB223F429
:1070B800E04323F0700343F4014343F0800325F8D1
:1070C8002230236A9B1B2362227835F8223013F082
:1070D800400F00F0A7806378B3BBB5F850309BB27F
:1070E8002B4403EB0213B3F80C24C2F30902A3F8F0
:1070F8000C243E2E0FD9710916F01F0F00D101394B
:10710800B3F80C2492B2890289B20A4342F40042CD
:10711800A3F80C241AE04EB9B3F80C246FEA4242E3
:107128006FEA524292B2A3F80C240FE0720816F0EC
:10713800010F00D00132B3F80C1489B2920292B256
:107148000A43A3F80C2401E0012B30D0B3B26289C2
:1071580061692846FFF7F6FE636933446361236A71
:10716800226993422DD99B1B23626378002B45D15A
:10717800B5F850309BB22B44227803EB0213B3F8D6
:107188000424C2F30902A3F804243E2E1DD9710970
:1071980016F01F0F00D10139B3F8042492B2890206
:1071A80089B20A4342F40042A3F8042428E0B5F85F
:1071B80050309BB22B4403EB0213B2B2A3F80C2459
:1071C800C4E7002222621E46CFE74EB9B3F8042472
:1071D8006FEA42426FEA524292B2A3F804240FE0E7
:1071E800720816F0010F00D00132B3F8041489B206
:1071F800920292B20A43A3F8042401E0012B06D0BC
:10720800B3B2228961692846FFF79CFE35E7B5F8D5
:1072180050309BB22B44227803EB0213B2B2A3F88E
:107228000424EDE76378B3BBB5F850309BB22B4428
:1072380003EB0213B3F80424C2F30902A3F80424ED
:107248003E2E0FD9710916F01F0F00D10139B3F87E
:10725800042492B2890289B20A4342F40042A3F894
:1072680004241AE04EB9B3F804246FEA42426FEAE4
:10727800524292B2A3F804240FE0720816F0010FEC
:1072880000D00132B3F8041489B2920292B20A43D0
:10729800A3F8042401E0012B30D0B3B2228961693C
:1072A8002846FFF74FFE636933446361236A226906
:1072B80093422DD99B1B23626378002B45D1B5F8E7
:1072C80050309BB22B44227803EB0213B3F80C2402
:1072D800C2F30902A3F80C243E2E1DD9710916F039
:1072E8001F0F00D10139B3F80C2492B2890289B278
:1072F8000A4342F40042A3F80C2428E0B5F85030C1
:107308009BB22B4403EB0213B2B2A3F80424C4E7E4
:10731800002222621E46CFE74EB9B3F80C246FEA6A
:1073280042426FEA524292B2A3F80C240FE072086C
:1073380016F0010F00D00132B3F80C1489B2920292
:1073480092B20A43A3F80C2401E0012B06D0B3B291
:10735800628961692846FFF7F5FD8EE6B5F8503079
:107368009BB22B44227803EB0213B2B2A3F80C248D
:10737800EDE7217835F8212092B222F4E24222F09A
:10738800700242F4004242F0800225F82120B5F84C
:10739800502092B22A44217802EB01129BB2A2F843
:1073A8000434228961692846FFF7CCFD65E64EB9A9
:1073B800B3F80C246FEA42426FEA524292B2A3F841
:1073C8000C2416E0720816F0010F00D00132B3F851
:1073D8000C1489B2920292B20A43A3F80C2408E072
:1073E800B5F850309BB22B4403EB0113B2B2A3F8AB
:1073F8000C24B3B2628961692846FFF7A3FD3CE615
:10740800B2BBB5F850309BB22B4403EB0113B3F871
:107418000424C2F30902A3F804243E2E0FD97109EB
:1074280016F01F0F00D10139B3F8042492B2890273
:1074380089B20A4342F40042A3F8042421E04EB979
:10744800B3F804246FEA42426FEA524292B2A3F8B8
:10745800042416E0720816F0010F00D00132B3F8C8
:10746800041489B2920292B20A43A3F8042408E0F1
:10747800B5F850309BB22B4403EB0113B2B2A3F81A
:107488000424B3B2228961692846FFF75BFDF4E55D
:1074980000228A611A4679E54AB9B3F80C246FEAE2
:1074A80042426FEA524292B2A3F80C248DE5510889
:1074B80012F0010F00D00131B3F80C2492B2890206
:1074C80089B20A43A3F80C247FE5CB78022B4DD070
:1074D800012B40F02F8189692369994240F2E680A7
:1074E800C91AA161F2B9B5F8502092B22A4421789C
:1074F80002EB0112B2F80414C1F30901A2F8041452
:107508003E2B40F2D780580913F01F0F00D10138E5
:10751800B2F8041489B2800280B2014341F40041F8
:10752800A2F804146278002A40F0F680B5F85020DA
:1075380092B22A44217802EB0112B2F80C14C1F37A
:107548000901A2F80C143E2B40F2CD80590913F022
:107558001F0F00D10139B2F80C349BB2890289B2ED
:107568000B4343F40043A2F80C342EE5F2B9B0F80B
:1075780050309BB203440A7803EB0213B3F8042497
:10758800C2F30902A3F804240A693E2A31D9510931
:1075980012F01F0F00D10139B3F8042492B2890206
:1075A80089B20A4342F40042A3F804246378002B0A
:1075B80051D1B5F850309BB22B44227803EB02131B
:1075C800B3F80C24C2F30902A3F80C2422693E2A5A
:1075D80028D9510912F01F0F00D10139B3F80C2432
:1075E80092B2890289B20A4342F40042A3F80C24F9
:1075F80033E04AB9B3F804246FEA42426FEA5242D0
:1076080092B2A3F80424D1E7510812F0010F00D078
:107618000131B3F8042490B28A0292B20243A3F86B
:107628000424C3E74AB9B3F80C246FEA42426FEA6C
:10763800524292B2A3F80C240FE0510812F0010F45
:1076480000D00131B3F80C2490B28A0292B20243FE
:10765800A3F80C2401E0012B1DD0E369002B3FF4B3
:10766800B4AC227835F8221044F2400303EA010052
:107678008B4302D000287FF4A8AC35F822309BB2A7
:1076880023F4E04323F0700343F4004343F0C003C2
:1076980025F8223099E4B5F850309BB22B44227873
:1076A80003EB0213228AA3F80C24D6E70023A36174
:1076B8000B4617E74BB9B2F804146FEA41416FEA79
:1076C800514189B2A2F804142CE7590813F0010FAC
:1076D80000D00131B2F8040480B2890289B20143B2
:1076E800A2F804141EE74BB9B2F80C346FEA43430E
:1076F8006FEA53439BB2A2F80C3466E4590813F0BE
:10770800010F00D00131B2F80C3498B28B029BB251
:107718000343A2F80C3458E4012A7FF456ACB5F8B8
:10772800502092B22A44217802EB01129BB2A2F8AF
:107738000C344AE4012059E410B45C0800EB420020
:1077480000F5806007E030F8042B0A70C2F30722C6
:107758004A700231013C002CF5D113F0010F01D021
:1077680003880B7010BC704738B51D4C21461D4866
:1077780001F0D0FE1C4B1870012221461B4801F075
:107788006FFE1B4B187018BB1A4802F05DFA1A48B6
:1077980002F05AFA194D686DF9F748F80446A86DD1
:1077A800F9F744F82146F8F71BFD4FF06A51F8F74E
:1077B80017FD4FF06A51F8F713FDF8F729FF024655
:1077C8000B460F4802F0E0F90E4B01221A7038BD43
:1077D8000D4802F039FA0B4B00221A70F7E700BF88
:1077E800A811002018530108AC110020780F0020C0
:1077F8000C0000205C1E0108141E0108600800200F
:10780800281E010844080020481E010800B583B05E
:10781800009313460A4601460348FDF7C1F900B133
:10782800012003B05DF804FB6008002000B583B0B8
:10783800009313460A4601460348FDF7D5FA00B1FE
:10784800012003B05DF804FB6008002008B5034878
:10785800FDF7A9FD043818BF012008BD6008002005
:1078680008B501460148FDF78CFD08BD60080020F9
:1078780082B001238DF807309DF8070002B07047E9
:1078880008B5FFF7F5FF012801D0012008BD02481F
:10789800FDF75CFDFAE700BF6008002020230380A5
:1078A800004870475C000020202303800048704790
:1078B8003C00002020230380004870471C00002063
:1078C8000A230380004870471000002038B504469A
:1078D800037CE3B94FF400730222012101F0FEFF9B
:1078E8000125C4F86C514FF400730222812120460F
:1078F80001F0F4FFE5624FF41B7002F04FF8C4F892
:10790800B802A0B1204600F042F9002038BD40235B
:107918000222012101F0E2FF0125C4F86C51402345
:1079280002228121204601F0D9FFE562E3E7022027
:10793800ECE738B50446012101F0DBFF0025C4F867
:107948006C518121204601F0D4FFE562204600F009
:107958004AF9D4F8B80218B102F024F8C4F8B852B9
:10796800002038BD2DE9F04182B006460C46D0F81B
:10797800B8720023ADF806300B7813F0600536D0E6
:10798800202D40F0B4804A78FE2A05D0FF2A1DD069
:1079980000F0B1FE0225ADE04A8812B9CA88012A72
:1079A80005D02146304600F0A6FE0225A2E013F0DD
:1079B800800FF6D0D0F8BC329B6998473860012216
:1079C8003946304601F0A4F9002593E04A8842B9C7
:1079D800CA8832B913F0800F03D100F0F7F80025F8
:1079E80088E02146304600F086FE022582E091F8C4
:1079F8000180B8F10B0F76D8DFE808F0062D757511
:107A0800757575757575152290F89C32032B03D022
:107A180000F071FE02256DE002220DF1060101F071
:107A280077F9454666E090F89C32032B03D000F0C6
:107A380062FE02255EE00122391D01F069F959E074
:107A480090F89C32032B02D18B787B6052E000F0D7
:107A580052FE02254EE0097901F053FF21793046A4
:107A680001F047FFA38894F90420002A19DB03F0EA
:107A78000F0303EB830306EB83030022C3F85821AB
:107A8800337C4BBB4FF4007302220121304601F0D6
:107A980025FF0123C6F86C312179304600F04EF9F4
:107AA80028E003F00F0303EB830306EB83030022B4
:107AB8009A61337C4BB94FF400730222812130461E
:107AC80001F00CFF0123F362E6E740230222812143
:107AD800304601F003FFF5E740230222012130463A
:107AE80001F0FCFED5E700F006FE022502E000F0FA
:107AF80002FE0225284602B0BDE8F08108B500F074
:107B080093F8002008BD08B500F000F9002008BD72
:107B180009B1C0F8BC120020704710B51346D0F860
:107B2800B842D4F814229C469A4200D293B2D4F8B0
:107B38003422A2EB0C02C4F83422002284F8382242
:107B4800042222720A46812101F012FF10BD38B5C5
:107B58000446D0F8B85295F8183223B9D5F814323B
:107B68000BB16B7A3BB18121204601F0D2FE6B7AD2
:107B7800022B04D038BD012101F0CBFEF3E71F230F
:107B880005F503720121204601F0FAFEF2E738B547
:107B98000446D0F8B85200202872687285F85D0251
:107BA80085F85C02D4F8BC321B689847012120464E
:107BB80001F0A7FE8121204601F0A3FE1F2305F551
:107BC80003720121204601F0DBFE38BD08B5D0F86C
:107BD800B82200231372012151721F2302F5037288
:107BE80001F0CEFE08BDD0F8B83200221A727047F4
:107BF80038B50546D0F8B8420A4BC4F82C3284F898
:107C08003812002323720D2304F50B72812101F031
:107C1800AFFE1F2304F503720121284601F0B0FED0
:107C280038BD00BF5553425310B50446D0F8B812BA
:107C38000B7A022B08D006D3033BDBB2012B02D808
:107C48000021FFF7D5FF10BD01F21B2291F8191290
:107C580000F060FB0028F6DA01212046FFF7C8FF94
:107C6800F1E7000038B50546D0F8B842D4F810322C
:107C7800C4F83032D4F81432C4F83432012101F097
:107C880087FE1F2804D1D4F80C221F4B9A420CD02F
:107C98002023052294F81912284600F0EFF8022351
:107CA80063722846FFF753FF38BD94F8191201296B
:107CB800EED894F81A32002BEAD0102BE8D804F248
:107CC8001B22284600F026FB00280CDB237A013B08
:107CD800DBB2022BE8D962898AB104F10C0128468B
:107CE800FFF71BFFE0E7237A052B03D02846FFF7B1
:107CF8002EFFD9E701212846FFF77AFFD4E70021B4
:107D08002846FFF775FFCFE75553424310B50446A1
:107D1800D0F8B8321A7A72B1012A0ED103F21B22B6
:107D280093F8191200F0F6FA002806DA0121204625
:107D3800FFF75EFF01E0FFF795FF10BD10B5D0F823
:107D4800B842637A022B08D011F0800F04D0012BBF
:107D580002D00121FFF74CFF10BD812101F0D9FDB0
:107D680000236372F8E7000010B4D0F8B8425378E3
:107D780013F0010F0DD00723638105E0013B9BB28F
:107D88000F4AD15CE2181173002BF7D1002010BC08
:107D98007047D0F8BC32D86901EBC10100EB810013
:107DA8000179053113798B4200D90B46638104E0D0
:107DB800013B9BB2C15CE2181173002BF8D1E5E7D7
:107DC80010530108D0F8B8020823438105E0013BAD
:107DD8009BB2044AD15CC2181173002BF7D1002062
:107DE800704700BF08530108D0F8B8020823438140
:107DF80005E0013B9BB2044AD15CC2181173002B09
:107E0800F7D10020704700BF0053010810B4D0F824
:107E1800B842002304E0E118002008730133DBB204
:107E2800112BF8D9702323730C23E37494F85C3274
:107E380094F85D128B420FD003F1470104EBC101A6
:107E48000879A073487A2076097A61760133DBB223
:107E580084F85C32042B08D0122363811379122B27
:107E680000D86381002010BC7047002384F85C327E
:107E7800F2E7D0F8B832002058817047D0F8B8023D
:107E880090F85D3203F1470100EBC1010A7100224D
:107E98000A720133DBB280F85D32042B00D07047E0
:107EA80080F85D22FBE770B50446D0F8B862D6F8D2
:107EB80014324BB90D46D0F8BC329B680846984737
:107EC80058B90023738170BD2023052296F8191232
:107ED800FFF7D4FF4FF0FF30F5E73A230222294697
:107EE8002046FFF7CBFF052333724FF0FF30EAE758
:107EF80070B582B005460E46D0F8B842002306E0B9
:107F0800E2184FF0000C82F80CC001339BB20B2B27
:107F1800F6D9D5F8BC325B680DF1060269463046E1
:107F28009847D0B90823E373009A531E190E217499
:107F3800C3F307416174C3F30723A374013AE274DE
:107F480002232375BDF80630002262751A0AA2754D
:107F5800E3750C23638102B070BD3A2302223146D7
:107F68002846FFF78BFF4FF0FF30F4E770B5054662
:107F78000E46D0F8B842D0F8BC325B6804F25E22F4
:107F880004F5187130469847B8B9D4F86022531EE2
:107F9800190E2173C3F307416173C3F30723A37356
:107FA800013AE273B4F85E320022227462741A0A4B
:107FB800A274E3740823638170BD3A230222314618
:107FC8002846FFF75BFF4FF0FF30F5E708B51A4486
:107FD800D0F8B832D3F860329A4201D8002008BDF0
:107FE80021230522FFF74AFF4FF0FF30F7E72DE97D
:107FF800F84306460F46D0F8B842D4F86852B4F8A9
:108008005E3203FB05F5B5F5007F28BF4FF4007518
:10801800D0F8BC22D2F8109004F10C08B5FBF3F3A9
:108028009BB2D4F8642241463846C84700281DDB75
:10803800ABB242468121304601F09AFCD4F8643252
:10804800B4F85E22B5FBF2F21344C4F86432D4F8F3
:1080580068329B1AC4F86832D4F83422521BC4F828
:10806800342263B903232372002009E01123042278
:1080780039463046FFF702FF4FF0FF3000E000209E
:10808800BDE8F883F8B506460F46D0F8B842237A1B
:1080980073BB154694F91832002B31DAD0F8BC328C
:1080A8009B6808469847A0BBAA78EB781B0443EA6C
:1080B80002632A7943EA02236A791A43C4F86422DC
:1080C800E9792B7A43EA0123C4F868323946304605
:1080D800FFF77CFF00282FDB02232372D4F8142239
:1080E800D4F86832B4F85E1201FB03F39A4219D14E
:1080F8004FF40073638139463046FFF778FFF8BDC7
:108108002023052294F81912FFF7B8FE4FF0FF302C
:10811800F5E73A23022239463046FFF7AFFE4FF023
:10812800FF30ECE72023052294F819123046FFF7B8
:10813800A5FE4FF0FF30E2E74FF0FF30DFE72DE913
:10814800F84306468846D0F8B842D4F86852B4F8DE
:108158005E3203FB05F5B5F5007F28BF4FF40075C7
:10816800D0F8BC22D2F8149004F10C07B5FBF3F355
:108178009BB2D4F8642239464046C84700281ADB27
:10818800D4F86422B4F85E32B5FBF3F10A44C4F8BB
:108198006422D4F86822521AC4F86822D4F8341237
:1081A800491BC4F834127AB900213046FFF720FD84
:1081B8000020BDE8F8830323042241463046FFF738
:1081C8005DFE4FF0FF30F4E702FB03F3B3F5007FE9
:1081D80028BF4FF400739BB23A460121304601F0A4
:1081E800CFFB0020E5E72DE9F04106460F46D0F821
:1081F800B842237A002B6AD1154694F91832002B1D
:1082080040DBD0F8BC329B6808469847002842D12A
:10821800D6F8BC32DB68384698478046002843D1F8
:10822800AA78EB781B0443EA02632A7943EA02231B
:108238006A791A43C4F86422E9792B7A43EA01235C
:10824800C4F8683239463046FFF7C0FE002842DBE2
:10825800D4F86832B4F85E2202FB03F3D4F814228F
:108268009A422AD1B3F5007F28BF4FF40073012149
:1082780021729BB204F10C02304601F081FB4046AA
:10828800BDE8F0812023052294F81912FFF7F6FDC6
:108298004FF0FF38F3E73A23022239463046FFF71A
:1082A800EDFD4FF0FF38EAE7272302223946304632
:1082B800FFF7E4FD4FF0FF38E1E72023052294F8AB
:1082C80019123046FFF7DAFD4FF0FF38D7E7FFF70E
:1082D80036FF8046D3E74FF0FF38D0E710B5D0F827
:1082E800B842537813F0020F0AD1D4F86832D4F8A0
:1082F8006422FFF76BFE002809DB0020608110BDB7
:1083080024230522FFF7BAFD4FF0FF30F7E74FF0BF
:10831800FF30F4E708B513785A2B5FD8DFE803F08D
:108328002E5E5E325E5E5E5E5E5E5E5E5E5E5E5EC1
:108338005E5E365E5E5E5E5E5E5E423A5E5E3E5EDD
:108348005E5E5E4A5E4E5E5E525E565E5E5E5E5A81
:108358005E5E5E5E5E5E5E5E5E5E5E5E5E5E5E5E35
:108368005E5E5E5E5E5E5E5E5E5E5E5E5E5E5E5E25
:108378005E5E5E5E5E5E5E5E5E5E4600FFF793FD7D
:10838800002008BDFFF742FD0020FAE7FFF7ECFCEC
:108398000020F6E7FFF76DFD0020F2E7FFF769FD23
:1083A8000020EEE7FFF70EFD0020EAE7FFF71CFDCF
:1083B8000020E6E7FFF79CFD0020E2E7FFF7D6FD87
:1083C8000020DEE7FFF75EFE0020DAE7FFF70BFF8D
:1083D8000020D6E7FFF782FF0020D2E720230522FE
:1083E800FFF74CFD4FF0FF30CBE798B108B50346D7
:1083F800D0F8B40210B10020C3F8B40209B1C3F830
:10840800B012012183F89C121A70184601F024FA60
:10841800002008BD0220704719B1C0F8B41200202E
:1084280070470220704708B501F050FA002008BDD7
:1084380008B5D0F8B4322BB11B68984700B908BD0D
:108448000220FCE70220FAE708B5D0F8B4325B68EE
:108458009847002008BD38B5044600F52A75284617
:1084680000F035F90123C4F89432B4F8AE32C4F8F8
:10847800983294F8A81201F01F03012B08D0022BA0
:108488000BD07BB92946204600F0D0FA002038BD31
:108498002946204600F0FEFAF8E72946204600F073
:1084A80029FBF3E701F08001204601F032FAEDE7FD
:1084B80038B504460D4691BB1346D0F89422032ADA
:1084C80003D0052A24D0084633E0D0F86011D0F84C
:1084D800642191420DD9891AC0F860118A4206D9DF
:1084E8008AB21946204600F028FC284621E092B2BC
:1084F800F7E7D0F8B4321B691BB190F89C22032A25
:1085080004D0204600F021FC284612E09847F8E7FE
:108518000021C0F8941201F0FCF9284609E0D0F8CF
:10852800B4329B6933B190F89C22032A04D198474E
:10853800002038BD0220FCE70220FAE738B50446DF
:108548000D46002953D11346D0F89422022A0CD0A4
:10855800042A00D01AB98021204601F0DAF994F8EB
:10856800A032012B3ED0284638BD026A416A8A42B1
:108578001BD8C269B2FBF1F301FB13232BB991425B
:1085880003D8D0F898329A421CD3D4F8B432DB68B6
:108598001BB194F89C22032A21D08021204601F0A7
:1085A800B8F9204600F0DCFBD9E7521A026292B211
:1085B800194600F0BAFB00231A461946204601F076
:1085C800DFF9CCE70022114600F0AFFB0021C4F828
:1085D80098120B460A46204601F0D2F9BFE720461A
:1085E8009847DAE7002384F8A0322846BCE7D0F899
:1085F800B4325B6933B190F89C22032A04D19847BE
:108608000020B1E70220AFE70220ADE770B50446CD
:1086180040230022114601F061F90125C4F85851A0
:108628004026C4F86461334600228021204601F0C8
:1086380055F9A561666284F89C520023C4F8943207
:108648006360C4F8A432D4F8B8322BB1D4F8B43289
:108658005B68002120469847002070BD0174002007
:10866800704790F89C3280F89D32042380F89C3241
:108678000020704790F89C32042B01D000207047EE
:1086880090F89D3280F89C32F8E708B590F89C3253
:10869800032B01D0002008BDD0F8B432DB69002BD1
:1086A800F8D09847F6E70346002002E00130C0B250
:1086B80001331A78002AF9D1704708B54B88012B85
:1086C80000D008BDC0F8A43200F03FFBF9E70B78F2
:1086D80003704B7843708B78CA7803EB022343808E
:1086E8000B794A7903EB022383808B79CA7903EBF0
:1086F8000223C380704710B50446802101F009F9B0
:108708000021204601F005F910BD30B583B00546BB
:108718000C460023ADF806304A88130A013B062BA5
:1087280000F2A480DFE803F004182CA2A2869300CC
:10873800D0F8B0321B680DF10601007C9847BDF8EF
:1087480006201AB1E388002B40F09480E388002BC0
:1087580000F09A8003B030BD037C43B9D0F8B4323E
:108768009B6A0DF10600984702234370E7E7D0F8AB
:10877800B432DB6A0DF10600984702234370DEE746
:10878800D2B2052A52D8DFE802F003101D2A374476
:10879800D0F8B0325B6823B10DF10601007C984730
:1087A800CDE72146FFF7A7FFD4E7D0F8B0329B68A2
:1087B80023B10DF10601007C9847C0E72146FFF779
:1087C8009AFFC7E7D0F8B032DB6823B10DF1060194
:1087D800007C9847B3E72146FFF78DFFBAE7D0F84A
:1087E800B0321B6923B10DF10601007C9847A6E75A
:1087F8002146FFF780FFADE7D0F8B0325B6923B1BF
:108808000DF10601007C984799E72146FFF773FFB1
:10881800A0E7D0F8B0329B6923B10DF10601007CC6
:1088280098478CE72146FFF766FF93E72146FFF755
:1088380062FF8FE7037C33B9D0F8B4325B6B0DF17C
:10884800060098477BE72146FFF755FF82E7037C40
:1088580043B9D0F8B4321B6B0DF1060098470723D3
:1088680043706CE72146FFF746FF73E72146FFF7A1
:1088780042FF6FE79A4228BF1A46ADF80620014624
:10888800284600F045FA61E7284600F05EFA61E7FD
:1088980038B504468B88F3B9CB88E3B94B887F2B6E
:1088A80019D803F07F0590F89C32032B0CD080F880
:1088B8009E52294601F054F8204600F046FA35B198
:1088C800022384F89C3209E0FFF715FF06E0012334
:1088D80084F89C3202E02046FFF70DFF38BD000007
:1088E80038B504460D468978284B197001290ED8E9
:1088F80090F89C32022B0ED0032B21D02946FFF78B
:10890800FAFE224B19782046FFF79EFD02E0294621
:10891800FFF7F1FE38BD81B14160032380F89C3236
:10892800FFF786FD022803D0204600F00EFAF1E793
:1089380029462046FFF7DFFEECE700F006FAE9E7F4
:1089480089B1436899421DD0D9B2FFF77DFD0F4B1D
:10895800197861602046FFF76BFD02280DD020468C
:1089680000F0F3F9D6E7022380F89C324160FFF764
:108978006BFD204600F0E9F9CCE729462046FFF7D1
:10898800BAFEC7E700F0E1F9C4E700BFAD11002067
:1089980008B5CB88012B0AD190F89C32022B09D953
:1089A800032B11D10122011D00F0B2F901E0FFF7FC
:1089B800A2FE08BD5BB23BB10146002341F8083F67
:1089C800012200F0A5F9F4E7FFF795FEF1E708B5F5
:1089D80090F89C32013B022B12D8CB88022B0CD189
:1089E8000123C360D0F8A4320BB10323C360022271
:1089F80000F10C0100F08CF908BDFFF77CFEFBE7E5
:108A0800FFF779FEF8E708B590F89C32013B022B96
:108A180009D84B88012B00D008BD0023C0F8A43228
:108A280000F093F9F8E7FFF766FEF5E708B50B786D
:108A380003F06003202B05D0402B03D043B1FFF790
:108A48005AFE03E0D0F8B4329B689847002008BD6E
:108A58004B78092B1BD8DFE803F011171A141A08F2
:108A6800051A0E0BFFF751FEF0E7FFF711FFEDE7D0
:108A7800FFF736FFEAE7FFF78BFFE7E7FFF7A7FF08
:108A8800E4E7FFF71AFEE1E7FFF7BDFFDEE7FFF7D0
:108A980032FEDBE738B505460C460B7803F0600379
:108AA800202B06D0402B04D01BB1FFF724FE00205A
:108AB80038BD95F89C32013B022B16D82379012B3F
:108AC8000ED8D5F8B4329B68214628469847E388E3
:108AD800002BECD10028EAD1284600F036F9E6E769
:108AE80021462846FFF707FEE1E721462846FFF71B
:108AF80002FEDCE770B505468B880C7804F060044C
:108B0800202C07D0DAB2402C04D05CB1FFF7F3FD7B
:108B1800002405E0D5F8B4329B682846984700241D
:108B2800204670BD202C09D04E78012E33D0032E5C
:108B38000AD0002E55D0FFF7DEFDF1E7D0F8B432A9
:108B48009B6898470446EBE790F89C32022B04D0C8
:108B5800032B11D0FFF7CFFDE2E70AB1802A03D13A
:108B68002846FFF7C8FDDBE7114600F0D2FE80215A
:108B7800284600F0CEFED3E74B8823B91AB1802AE5
:108B880001D0CB881BB1284600F0DFF8C8E71146B2
:108B980000F0BFFEF7E790F89C32022B04D0032BBD
:108BA80011D0FFF7A8FDBBE70AB1802A03D12846F8
:108BB800FFF7A1FDB4E7114600F0ABFE802128467F
:108BC80000F0A7FEACE74B88002BA9D112F07F0F6D
:108BD80003D1284600F0B9F8A2E7114600F0A1FE3B
:108BE800F7E790F89C02022806D0032829D02846E7
:108BF800FFF781FD344693E70AB1802A13D113F0B9
:108C0800800F15D102F07F0202EB8202910001F57C
:108C1800A8712944043100230B600222284600F081
:108C280077F834467CE72846FFF765FD344677E752
:108C380002F07F0202EB82029100103129440431D4
:108C4800E9E75BB2002B1FDB02F00F0000EB8000AE
:108C580005EB8000D0F8580120B3002B27DB02F089
:108C68007F0303EB83039C0004F5A8742C440434AD
:108C78000AB1802A24D100232360022221462846F3
:108C880000F046F834464BE702F00F0000EB800096
:108C980005EB800080690028DFD12846FFF72BFD0F
:108CA80034463DE72846FFF726FD344638E702F00C
:108CB8007F0303EB83039C0010342C440434D7E770
:108CC8001146284600F035FE10B101232360D4E791
:108CD80000232360D1E7D0B170B50D46164604468F
:108CE800FFF7E1FC431C5B009BB233802B7003232E
:108CF8006B70022307E001345A1CD2B2E8540233E5
:108D0800DBB20021A95420780028F4D170BD704747
:108D180008B513460222C0F89422C36103620A46CA
:108D2800002100F025FE002008BD08B513460A46BC
:108D3800002100F01DFE002008BD08B513460A46B4
:108D4800002100F01DFE002008BD08B50423C0F86E
:108D5800943200231A46194600F00AFE002008BD86
:108D680008B50523C0F8943200231A46194600F0C6
:108D780007FE002008BD000008B5044B03EB800285
:108D8800526852680344187A904708BDD0110020F1
:108D980008B5084B1B5C53B9064B01221A5403EB68
:108DA8008002526812680344187A904708BD002070
:108DB800FCE700BFD011002038B5044C04EB800557
:108DC8006D68AD680444207AA84738BDD0110020EA
:108DD80038B5044C04EB80056D68ED680444207ACE
:108DE800A84738BDD011002008B5074B01221A70DA
:108DF800FEF746FD20B9044A137803F0FE0313700A
:108E0800014B187808BD00BFB400002008B5074B17
:108E180001221A70FEF71AFD20B9044A137803F0EC
:108E2800FE031370014B187808BD00BFB400002082
:108E380010B5084611461A46094BFEF7E7FC10B173
:108E48000123184610BD074CFEF700FD0346002815
:108E5800F7D0631E0CB11C46F6E70123F1E700BF0B
:108E680000E1F505A086010010B5084611461A462E
:108E7800094BFEF7DBFC10B10123184610BD074C67
:108E8800FEF7E4FC03460028F7D0631E0CB11C462D
:108E9800F6E70123F1E700BF00E1F505A086010030
:108EA80030B589B0124B187810F001041AD1154664
:108EB80003291BD8DFE801F002040A100C4612E06F
:108EC8006846FEF7CDFC069B2B600CE06846FEF773
:108ED800C7FC079B2B8006E06846FEF7C1FC079B92
:108EE8002B6000E00324204609B030BD0424FAE7D3
:108EF800B4000020002302E010BC70470133012BAE
:108F080017D803EB43020B4951F822208242F5D1CE
:108F180010B403EB4302920000248C500133012B60
:108F2800EAD803EB4302034951F822208242F5D1E3
:108F3800EFE77047B01100200146006838B10246DB
:108F48001378202B06D93A2B04D00132F8E74FF0DA
:108F5800FF3070473A2B01D00020704710B4034609
:108F680013F8010B3038092808D89A4202D04FF07C
:108F7800FF3005E030B901320A6001E04FF0FF3000
:108F880010BC70474FF0FF30FAE7F8B590F804527C
:108F98000DB92846F8BD0446D0F82C7201233A468C
:108FA800014690F80102FFF713FF0546D0B90023E8
:108FB80084F80432D4F82032FB1AD4F818229342E9
:108FC800E7D294F803620AE0D4F818321F44012368
:108FD8003A46214694F80102FFF7FAFE013E012EB7
:108FE800F2D8D6E70125D4E770B5D0F82C328B42F9
:108FF80002D10026304670BD04460D46FFF7C5FF76
:1090080006460028F6D101232A46214694F8010293
:10901800FFF7D2FE10B101264FF0FF35C4F82C52ED
:10902800E8E7000010B50446002380F804324FF04A
:10903800FF33C0F82C32FFF7D7FF98BB024694F8ED
:10904800FF1194F8FE3143EA01231BB217498B4202
:109058002AD194F8391094F838301B0443EA016394
:1090680094F8371043EA012394F836100B4323F0A1
:109078007F430F498B4213D094F8551094F854301D
:109088001B0443EA016394F8531043EA012394F85C
:1090980052100B4323F07F4305498B4200D0012235
:1090A800104610BD0322FBE70222F9E755AAFFFF8D
:1090B800464154002DE9F04385B005461746002384
:1090C80003600846FFF738FF061EC0F29E819F4BDB
:1090D80053F82640002C00F09D812C6094F8003253
:1090E8007BB194F80102FFF747FE10F0010508D1A3
:1090F800002F00F08B8110F0040F00F087810A2503
:1091080084E1002384F80032F0B284F80102FFF70A
:109118003FFE10F0010F40F07F811FB110F0040FE7
:1091280040F07C8100212046FFF77CFF054601289E
:1091380000F095800027032D00F07281002D40F08B
:109148007181227BE37A43EA02231BB2B3F5007FE5
:1091580040F06A81E27DA37D53EA02230DD194F8A1
:10916800272094F826301B0443EA026394F825204C
:1091780043EA022394F824201343C4F81832217CCC
:1091880084F803124A1ED2B2012A00F24F8103FB6F
:1091980001F1607B84F80202002800F04981421E38
:1091A800104240F04781A67C627C42EA06221646BD
:1091B800A4F8082212F00F0F40F03E8194F814C072
:1091C800E27C52EA0C220ED194F823C094F82220B3
:1091D800120442EA0C6294F821C042EA0C2294F884
:1091E80020C042EA0C0294F80FE094F80EC05CEA42
:1091F8000E2C00F023810CEB010909EB16194A45E6
:10920800C0F01E81A2EB0902B2FBF0FE8242C0F060
:10921800198140F6F57296453AD94FF6F57296459A
:1092280077D84FF0020835E0002304AA02EB810248
:1092380042F8103C0131032913D80B0103F5DF7301
:1092480023441A79002AEFD0D87A9A7A120442EA8B
:109258000062587A42EA00221B7A1343E5E70021AC
:10926800E9E700260BE039462046FFF7DBFE054616
:1092780000283FF460AF0136032E3FF65CAF04AB25
:1092880003EB860353F8107C002FECD10225F2E79C
:109298004FF001080EF1020EC4F814E2C4F81C7273
:1092A8000CEB0702C4F8202207EB0900C4F82802D7
:1092B800B8F1030F30D0002E00F0C8800A44C4F87B
:1092C8002422B8F1020F3DD00EEB4E010EF0010240
:1092D80002EB510202F2FF12B3EB522FC0F0B8803A
:1092E8004FF0FF33C4F81032C4F80C32802384F8EE
:1092F8000532B8F1030F2DD084F80082144A138880
:1093080001339BB21380A4F806322046FFF7F2FD22
:109318007CE04FF00308BDE7002E40F0958094F8FC
:109328002F1094F82E20120442EA016294F82D10AE
:1093380042EA012294F82C100A43C4F824224FEA86
:109348008E02C7E74FEA4E02C4E700BFCC110020E7
:10935800C811002094F8312094F8303043EA0223F1
:109368001BB2012BC8D1791C2046FFF73DFE00280F
:10937800C2D1002384F8053294F8FF2194F8FE3115
:1093880043EA02231BB2334A9342B5D1E278A37869
:109398001B0443EA0263627843EA022322781343F8
:1093A8002D4A9342A8D194F8E72194F8E6311B049A
:1093B80043EA026394F8E52143EA022394F8E4219E
:1093C8001343264A934297D194F8EB2194F8EA3153
:1093D8001B0443EA026394F8E92143EA022394F860
:1093E800E8211343C4F8103294F8EF2194F8EE31D1
:1093F8001B0443EA026394F8ED2143EA022394F83C
:10940800EC211343C4F80C3276E70B25284605B047
:10941800BDE8F0830C25F9E70325F7E70A25F5E70A
:109428000125F3E70D25F1E70D25EFE70D25EDE71C
:109438000D25EBE70D25E9E70D25E7E70D25E5E720
:109448000D25E3E70D25E1E70D25DFE70D25DDE730
:109458000D25DBE755AAFFFF525261417272416147
:1094680070B584B0019000911646039103A8FFF7E8
:1094780063FD041E1DDB114B53F824502DB1284603
:10948800FFF738FD002385F80032019B13B1002255
:1094980083F80022094A42F8243063B1012E02D031
:1094A800002004B070BD0022694601A8FFF702FE43
:1094B800F7E70B20F5E70020F3E700BFCC11002009
:1094C800134B5B7ADBB2012B01D90120704710B432
:1094D80004460F4B93F809C05FFA8CFC002003F890
:1094E8000C0093F809C003EB8C0CCCF804405C7AB0
:1094F8001C4422725A7A541CE4B25C7230320A70EC
:109508003A234B702F238B70C87010BC704700BF74
:10951800D011002008B50022FFF7D2FF08BD0000D7
:1095280008B500220F491048FEF75FFF70B90F49D0
:109538000D48FEF771FF60B90D490B48FEF7E8FAD0
:1095480050B90948FEF76FFF48B908BDF7F78CFE18
:10955800EDE7F7F789FEEFE7F7F786FEF1E7F7F7AC
:1095680083FEF2E7EC000020DC1100207C000020E4
:109578000801002012230B8000487047D800002003
:1095880004230B8000487047D40000200023934236
:109598001ED200B510E00CF1370C01F813C0000121
:1095A8004FEA430C0CF1010C4FF0000E01F80CE0EF
:1095B8000133DBB2934209D24FEA107CB0F1204F5D
:1095C800E9D20CF1300C01F813C0E8E75DF804FBB0
:1095D8007047000038B50B4BD3F8E807D3F8EC47D1
:1095E800D3F8F037C01800D138BD074D08222946F6
:1095F800FFF7CCFF042205F110012046FFF7C6FF54
:10960800F2E700BF00F0FF1FBA00002008B51A23D8
:109618000B80FFF7DFFF014808BD00BFB80000203E
:1096280008B50A4628B905490548FFF754FB034819
:1096380008BD02490248FFF74EFBF8E7A0140020D6
:10964800601E010810B50A46034C21460348FFF77F
:1096580042FB204610BD00BFA0140020741E010864
:1096680008B50A4628B905490548FFF734FB0348F9
:1096780008BD02490248FFF72EFBF8E7A0140020B6
:10968800881E010808B50A4628B905490548FFF7A4
:1096980022FB034808BD02490248FFF71CFBF8E714
:1096A800A0140020941E0108034B586D08609B6DA0
:1096B80013800020704700BF60080020002070471A
:1096C800002070470020704770B5084615461E46B2
:1096D8000B4B32462946FEF7A9F838B9094CFEF774
:1096E800B5F818B1601E44B10446F8E73246294679
:1096F800054800F049FA002070BD0220FCE700BFD1
:1097080000E1F505A0860100A41E010870B5084611
:1097180015461E460B4B32462946FEF777F838B9F0
:10972800094CFEF793F818B1601E44B10446F8E7F7
:1097380032462946054800F027FA002070BD02206D
:10974800FCE700BF00E1F505A0860100D01E010876
:1097580008B5044800F078FAFEF792F800B908BD99
:109768000220FCE7FC1E0108022805D8DFE800F00B
:1097780005040200012070470220704702680E4B62
:109788009A4200D0704700B583B003F5DA33DA693E
:1097980042F40002DA61DB6903F400030193019BE0
:1097A800002203211420F8F7D7FE1420F8F7E4FE6E
:1097B80003B05DF804FB00BF005C004008B500F58D
:1097C8002C71D0F8EC02FEF746FE08BD08B501EB97
:1097D800810300EBC303D3F87C21D0F8EC02FEF739
:1097E80067FE08BD08B501EB810300EBC303DA6B24
:1097F800D0F8EC02FEF7A2FE08BD08B5D0F8EC02DE
:10980800FEF743FF08BD10B504468368022B09D153
:109818000121D4F8EC02FEF721FFD4F8EC02FEF7A0
:10982800F5FE10BDF7F720FDF2E7000010B504467D
:10983800D0F8EC02FEF715FFA36923B1024A1369B9
:1098480043F00603136110BD00ED00E008B5D0F841
:10985800EC02FEF70FFF08BD10B504461948C0F822
:10986800EC42C4F8C002184B03600823436002238B
:10987800836000238361C3610362F9F7F7FAE8B9EB
:10988800182300221146D4F8C002FAF777FA5823B1
:1098980000228021D4F8C002FAF770FA9823002237
:1098A8008121D4F8C002FAF769FAD82300220121ED
:1098B800D4F8C002FAF762FA002010BDF7F7D4FC1A
:1098C800DEE700BF10190020005C004008B5D0F8A2
:1098D800C002F9F753FBFFF747FF08BD08B59446E8
:1098E8001A466346D0F8C002FAF7FEF8FFF73CFFC5
:1098F80008BD08B5D0F8C002FAF734F9FFF734FF0D
:1099080008BD08B5D0F8C002FAF71DFAFFF72CFF1A
:1099180008BD08B5D0F8C002FAF79EF9FFF724FF92
:1099280008BD08B5D0F8C002FAF7D2F9FFF71CFF56
:1099380008BDD0F8C03211F0800F08D101F07F01C6
:1099480001EB810103EBC10393F86A01704701F051
:109958007F01013101EB810103EBC1039878704766
:1099680008B5D0F8C002F9F7D3FFFFF7FDFE08BD30
:1099780008B5D0F8C002FAF74DF9FFF7F5FE08BDB3
:1099880008B5D0F8C002FAF71FF9FFF7EDFE08BDD9
:1099980008B5D0F8C002FAF734F908BD0048704796
:1099A800A016002070477047024A0349034800F098
:1099B800C9B800BF28010020D9F1000838010020EB
:1099C8000C4B416810B59942044601D005F000FCE3
:1099D800A168094B994202D0204605F0F9FBE168DD
:1099E800064B994204D02046BDE8104005F0F0BB74
:1099F80010BD00BF001C0020681C0020D01C0020E7
:109A08002DE9F84300250423304C314A3149DFF869
:109A1800C890DFF8C880324F324E116004F15C0004
:109A280029460822C4E90335C4E90055C4E90555A7
:109A3800A560656600F04CFA04F15800C4E90749CE
:109A4800C4E90987E66200F015FB274B294608227E
:109A580004F1C4006367C4E91A55C4E91E552567B3
:109A6800C4F8CC50C4F8805000F032FA04F168030E
:109A780004F1C000C4F88430C4E92298C4E924760B
:109A880000F0F8FA194B294604F596700822C4F834
:109A9800DC30C4E93455C4E93855C4F8D850C4F8A2
:109AA8003451C4F8E85000F013FA04F1D003C4E9C3
:109AB8003D87C4F8F09004F59470C4F8FC60C4F8CD
:109AC800EC30BDE8F84300F0D5BA00BF001C002018
:109AD800381D0020B1990008499E00086D9E0008B5
:109AE800AD9E0008D19E0008090001001200020086
:109AF80010B504460A4800F0C1FA636B23B9094B54
:109B0800094A1B68626323B1BDE81040044800F0AD
:109B1800B7BAFFF775FFBDE81040014800F0B0BACA
:109B2800481D0020381D0020C9990008014800F090
:109B3800A5BA00BF481D0020014800F0A1BA00BF27
:109B4800481D00202DE9F8434FF0000980460F46D4
:109B58001646D6E90154013D10D4A389012B08D932
:109B6800B4F90E30013304D021464046B84749EADB
:109B78000009013D6B1C04F16804EED13668002E23
:109B8800E7D14846BDE8F8830FB400B5074A83B06B
:109B980004AB106853F8042B8168019302F066FC4B
:109BA80003B05DF804EB04B0704700BF3401002037
:109BB80030B5054689B008460C4600F063FA012323
:109BC8000222204907936B6B0691029204A9421C5A
:109BD80004940191AC6805900392002B2ED0626E1C
:109BE800B4F90C30D20701D4980521D5990406D4CC
:109BF800626E43F4005322F40052A3816266284641
:109C080001AA214605F002FC636E00280CBF0A2554
:109C18004FF0FF35DA0702D4A3899B0502D5284601
:109C280009B030BDA06D00F02BFA284609B030BD50
:109C3800A06D00F023FAB4F90C30D7E72846FFF7F7
:109C480057FFCCE70C1F0108024B01461868FFF7C5
:109C5800AFBF00BF340100202DE9F043664C0E462B
:109C6800D4F80080174604461D4683B0B8F1000FAB
:109C780004D0D8F83430002B00F0A680022F05D08D
:109C8800012F00F2A580002DC0F2A280636EDA07D2
:109C980051D52146404605F08FFB216B41B104F1B7
:109CA8004003994202D0404600F086FA002323631D
:109CB8000023B4F90CC0A3611CF0800F63605DD170
:109CC8002CF44A6C2CF0030C022FA4F80CC063D0BF
:109CD80001AB214640466A4605F07CFDA38918433E
:109CE800A081002D2ED0002E2DD0D8F83430002B96
:109CF80037D0009AB4F90C30AA421CBF43F4006371
:109D0800A381012F04BF43F00103A38113F00802CC
:109D1800C4E90465266028D0D90753D50022A2607B
:109D2800626E6D42D207A56123D49B0521D4A06D34
:109D380000F0A6F91DE0A3899B05AAD4A06D00F048
:109D48009DF9A6E7009D284600F032FB064600284C
:109D580041D0A38943F08003A381D8F83430002B85
:109D6800C7D14046FFF7C4FEC3E7A260626ED207C0
:109D7800DBD50025284603B0BDE8F08340462169BD
:109D880000F01AFAB4F90CC0022F2CF44A6C2CF02B
:109D9800030CA4F80CC09BD100250021012204F17A
:109DA800430323602361636E4CF00200A081D8074F
:109DB800A1606261DED41CF4007FDBD1A06D00F0ED
:109DC8005FF9D7E7A560D1E74046FFF791FE55E771
:109DD8004FF0FF35CEE7DDF80090A94506D048469C
:109DE80000F0E6FA064608B14D46B2E74FF0FF35F7
:109DF800B4F90CC0D1E700BF340100200EB430B56F
:109E080004466FF000459CB00B4A1FAB0B49059206
:109E180053F8042B086802A9CDE901340495079585
:109E2800069400F08DFD0022029B1A701CB0BDE85C
:109E3800304003B0704700BF0802FFFF3401002024
:109E480010B50C46B1F90E1000F0BAF8002803DB83
:109E5800236D0344236510BDA38923F48053A38194
:109E680010BD00BF2DE9F0410C46B1F90C101F469A
:109E7800CB05054616460BD421F48051A1813B46FB
:109E880032462846B4F90E10BDE8F04100F0AEB8ED
:109E9800B4F90E100223002200F07CF8B4F90C107B
:109EA800EAE700BF10B50C46B1F90E1000F072F8E1
:109EB800B4F90C30421C0EBF23F4805343F4805392
:109EC8002065A38110BD00BFB1F90E1000F050B895
:109ED80070B5860747D0541E002A3ED00346CAB242
:109EE80001E0013C39D303F8012B9D07F9D1032C7C
:109EF8002CD9CDB205EB05250F2C1A4605EB0545E7
:109F080034D9A4F1100C2CF00F0603F1100EB6444E
:109F18004FEA1C1CC2E90055C2E9025510327245CD
:109F2800F8D10CF1010214F00C0F03EB021204F04B
:109F38000F0C13D0ACF1040323F0030304331344D0
:109F480042F8045B9342FBD10CF003042CB1C9B274
:109F58001C4403F8011BA342FBD170BD64461346A1
:109F6800002CF4D1F9E703461446C0E7A446E1E71C
:109F7800002238B5064D044608462A60F7F71EFA4F
:109F8800431C00D038BD2B68002BFBD0236038BDA4
:109F98003C1D002038B50C46114600228446074D6A
:109FA80020462A601A466446F7F714FA431C00D084
:109FB80038BD2B68002BFBD0236038BD3C1D00202A
:109FC80038B50C46114600228446074D20462A60C3
:109FD8001A466446F7F706FA431C00D038BD2B68CA
:109FE800002BFBD0236038BD3C1D002038B50C4643
:109FF800114600228446074D20462A601A466446C8
:10A00800F7F7C2F9431C00D038BD2B68002BFBD0F2
:10A01800236038BD3C1D0020014B1868704700BF05
:10A028003401002070B50F4B0F4DAB42A3EB050672
:10A0380007D00024B61055F8043B01349847A642CF
:10A04800F9D807F05DFE094D094B5E1BAB424FEA9C
:10A05800A60606D0002455F8043B01349847A642CA
:10A06800F9D870BDBC550108BC550108BC5501089C
:10A07800C4550108704700BF704700BF704700BF54
:10A08800704700BF20F0030110F00300C0F100008A
:10A0980051F8043B00F1040C4FEACC0C6FF00002BD
:10A0A8001CBF22FA0CF213434FF0010C4CEA0C2CA3
:10A0B8004CEA0C4CA3EB0C0222EA030212EACC1283
:10A0C80004BF51F8043B0430F4D0C2F1000102EAA5
:10A0D8000102B2FA82F2C2F11F0200EBD20070470D
:10A0E800024B13B1024800F005B8704700000000A9
:10A0F800C9FB0008002301461A46184605F004BEAD
:10A108002DE9F84306460820894605F06DFD054609
:10A11800DFF89880304600F007FCD8F808305F6810
:10A1280027F00307A7F11104A4EB09042C44B4FB9E
:10A13800F5F4013C05FB04F4A54208DC0021304697
:10A1480005F02CFDD8F808303B44984205D030463D
:10A1580000F0F0FB0020BDE8F8833046614205F0CE
:10A168001DFD01300FD0124AD8F808303F1B47F0C8
:10A1780001075F60136830461B1B136000F0DAFBB1
:10A188000120BDE8F8830021304605F007FDD8F826
:10A198000820831A0F2BDADD43F001035360054BC7
:10A1A80003491B68C01A0860D1E700BF6802002095
:10A1B800501D00205C02002000297CD0F8B50C4618
:10A1C800064600F0B1FB54F8043C764FA4F10805AC
:10A1D80023F001016818D7F808C04268844522F0C6
:10A1E800030200F08380DB07426000EB020C33D4EB
:10A1F80054F8084CDCF804302D1B2144AC6807F1F6
:10A20800080C644503F0010364D0D5F80CE0C4F8E9
:10A218000CE0CEF80840002B00F0818041F00103EB
:10A228006B600160B1F5007F22D20122CB08490999
:10A238008A40796801330A437A6057F8331007EB8C
:10A24800C302083AC5E9021247F83350CD603046D8
:10A25800BDE8F84000F06EBBDCF80430DB072BD516
:10A2680041F00103B1F5007F44F8043C0160DCD300
:10A27800B1F5206F4FEA512353D28B0903F139000E
:10A2880003F13802C300F818FB580838984203D184
:10A2980061E09B68984204D05A6822F003028A421F
:10A2A800F7D8D868C5E9023085603046DD60BDE87A
:10A2B800F84000F03FBB7047114407F1080C836871
:10A2C80063453FD0C268DA60936041F001036B6078
:10A2D8006950A7E7002B5FD10A44D0E90213CB608D
:10A2E800996042F001036B60AA50B0E70A44D907AD
:10A2F80007D454F8083CED1A1A44D5E90213CB6088
:10A30800996042F001036B60274BBD601B68934264
:10A318009DD8264B30461968FFF7F2FE97E711449F
:10A32800CDE7142B08D9542B1DD80B0B03F16F0064
:10A3380003F16E02C300A6E703F15C0003F15B02C0
:10A34800C300A0E741F00103C7E90455C5E902CC01
:10A358006B6069507BE70121921001FA02F279687B
:10A368000A437A609EE7B3F5AA7F06D8CB0B03F1C0
:10A37800780003F17702C30085E740F25452934214
:10A3880006D88B0C03F17D0003F17C02C3007AE749
:10A398004FF47E737E2276E741F001036B60016023
:10A3A80055E700BF6802002060020020801D0020E1
:10A3B800024B0146186800F003B800BF34010020C2
:10A3C8002DE9F04F01F10B05162D064683B024D870
:10A3D800102900F2AD8000F0A7FA102518234FF0DD
:10A3E800020CB84F3B445C68A3F10802944200F0A9
:10A3F8001D8130466368E268A16823F00303CA60E0
:10A40800234491605A68083442F001025A6000F00F
:10A4180091FA204603B0BDE8F08F35F0070500F14A
:10A428008780A94200F2848000F07EFAB5F5FC7FAF
:10A43800C0F06F816B0A7FD0042B00F21E81AB093C
:10A4480003F1390C03F1380E4FEACC009D4F384424
:10A4580044680838A04207D10DE0002AE16880F27C
:10A46800DF80884207D00C46636823F003035A1B39
:10A478000F2AF2DDF446DFF850823C69444500F0CB
:10A48800BC80636823F00309A9EB05030F2B00F3D5
:10A498004581002BC7E9048880F22F81B9F5007F38
:10A4A800D7F804E080F0C98001234FEAD9014FEAC8
:10A4B8005919194403FA09F357F831204EEA030EE3
:10A4C80007EBC103083BA260E360C7F804E047F864
:10A4D8003140D46001204FEAAC039840704532D82F
:10A4E80010EA0E0F07D12CF0030C400010EA0E0FF3
:10A4F8000CF1040CF9D007EBCC0AD646E146DEF89D
:10A508000C300BE059681C4621F003014A1B0F2A46
:10A51800DB6800F3BF80002A80F2E2809E45F1D11B
:10A5280009F1010919F0030F0EF1080EE7D11FE137
:10A538000C23336000246CE74FF400704FF0400C9C
:10A548004FF03F0E82E7BC68636823F00309A94512
:10A5580003D3A9EB05030F2B52DC5C4B08201B68C7
:10A5680003F1100804EB0903009305F03DFB584A7A
:10A5780083461368A844013305D008F1FF388044A6
:10A58800434203EA08084146304605F007FBB0F1AC
:10A59800FF3F82464E4A00F0DC8004EB0903834209
:10A5A80000F2D5804B4B0BF1FF31186840448446CC
:10A5B800186040F0FB801AEA010F40F0F780D7F8E6
:10A5C80008A0C84448F00102CAF804205446424B87
:10A5D8001968814238BF1860404B1968814238BFFA
:10A5E800186022F00308A845A8EB050301D30F2B38
:10A5F80006DC304600F09EF99CE7D7F804E069E7EE
:10A60800621943F0010345F0010565603046BA6000
:10A618000834536000F08EF9204603B0BDE8F08F8F
:10A62800A2683046D16023448A60EBE6DC68A34226
:10A638007FF4DFAE0CF1020C1DE7B9F5206F4FEA8D
:10A6480059227DD3142A00F2118102F15C03DB0048
:10A658005B32F918FB580839994203D1ECE09B6842
:10A66800994204D05A6822F003024A45F7D8D968BB
:10A67800C4E902318C60DC602CE7142B6CD9542BB4
:10A6880000F2FD802B0B03F16F0C03F16E0E4FEA05
:10A69800CC00DBE6D4F808C03046661945F0010561
:10A6A8006560CCF80C30C3F808C042F00103C7E974
:10A6B8000466C6E902887360625000F03BF908340A
:10A6C800A7E600BF6802002070020020801D00205D
:10A6D8005C020020501D00207C1D0020781D0020F9
:10A6E80021444A68304642F001024A6054F8082F73
:10A6F800D3609A6000F01EF98BE6A144D9F80430C3
:10A70800304643F00103C9F8043000F013F9083467
:10A718007FE64FEAD50C05F1080362E6621943F0BB
:10A72800010145F0010565603046C7E90422C2E928
:10A738000288516044F8093000F0FCF8083468E6F3
:10A748004FEA991202F13903DB00383281E7BC4243
:10A7580024D0BC68626844E703F15C0C03F15B0E2B
:10A768004FEACC0072E65AF80839534540F0D880D1
:10A778001CF0030F0CF1FF3CF5D17B6823EA0003C2
:10A788007B60400098423FF6DEAE18B9DBE6400039
:10A7980009F104091842FAD0CC46ACE6614B0BF13A
:10A7A800FF31186808EB000CC3F800C010680130CE
:10A7B80070D004EB0902AAEB020262441A601AF094
:10A7C8000702CDE9002340D0C2F108029244D044E8
:10A7D80008EA01005A44121A02EA010B59463046A7
:10A7E80005F0DCF9421C019B71D0A0EB0A0000EBDC
:10A7F8000B08186848F001025844BC42C7F808A082
:10A808001860CAF804203FF4E1AEB9F10F0F44D93B
:10A818004FF0050C6168A9F10C0222F0070201F063
:10A828000101114361600F2A04EB0201C1E901CC67
:10A8380055D8DAF80420C9E60120921000FA02F28D
:10A848004EEA020EC7F804E012E70AEB08020A40D3
:10A85800ABEB020202EA010B5946304605F09EF9BD
:10A86800431C019BC1D1DDF800B0C2E7542A18D8B7
:10A878004FEA193202F16F03DB006E32E9E6B3F5F5
:10A88800AA7F18D8EB0B03F1780C03F1770E4FEA87
:10A89800CC00DBE5C2F800A091E70123CAF8043038
:10A8A800A7E6B2F5AA7F25D84FEAD93202F1780394
:10A8B800DB007732CDE640F25452934225D8AB0CF8
:10A8C80003F17D0C03F17C0E4FEACC00BEE5009A43
:10A8D8004FF0000B083A9044A8EB0A0889E7304685
:10A8E80004F108010093FFF767FC009BD7F808A064
:10A8F80018689EE740F254539A420DD84FEA99429D
:10A9080002F17D03DB007C32A3E64FF47E704FF04A
:10A918007F0C4FF07E0E99E54FF47E737E2298E609
:10A928007B682EE7501D00200148FFF7A7BB00BF3A
:10A93800401D00200148FFF7A3BB00BF401D0020B9
:10A948002DE9F04FDDB00C4691460D910F938346EB
:10A9580005F0FAF8036818461A93FFF793FB0822E4
:10A96800189000212CA8FFF7B3FAA389180603D57D
:10A978002369002B00F01587002300249E46CDE9AB
:10A988003133002333AACDE91634DA4614464D464E
:10A99800CDE91BEE3092CDF864E0CDF880E0CDF83B
:10A9A80074E0CDF828E0CDF848E02F466E4BD3F898
:10A9B800E46005F0C3F80DF1B00C03463A46504682
:10A9C80028A9CDF800C0B047002800F09F80C0F249
:10A9D8009580289B252B01D00744E7E7B7EB0508AE
:10A9E800064640F0978000224FF0FF3393460993C4
:10A9F8007B787E1C8DF897200B9299460136A9F139
:10AA080020035A2B00F2B280DFE813F0F302B00003
:10AA1800B000EF02B000B000B000FD02B000B0001E
:10AA28006A003502B0002702D202B000CE025B00F5
:10AA38005B005B005B005B005B005B005B005B0036
:10AA4800B000B000B000B000B000B000B000280105
:10AA5800B000AA013E02280128012801B000B00078
:10AA6800B000B0003A02B000B000A802B000B000D8
:10AA7800B000D001B000BC02B000B0008A06B0003F
:10AA8800B000B000B000B000B000B000B0002801C5
:10AA9800B000AA0101022801280128012B020102A5
:10AAA8007400B0006402B0005502AF066E02740074
:10AAB800B000D0017200AC06B000B000B206B00021
:10AAC80072000022A9F1300316F8019B02EB820202
:10AAD80003EB4202A9F13003092BF5D90B928EE75B
:10AAE8000F9B53F8042B002A0B920F93C0F2B281EC
:10AAF800337882E733784BF0200B7EE70822002179
:10AB08002CA8FFF7E5F9012007444FE7B7EB050844
:10AB1800064610D0329BC4E9005843443293319B17
:10AB28000133072B319315DC08340A9B43440A93FD
:10AB3800002E7FF458AF329B002B41F05E810D9BB5
:10AB48009B8903F04003002B41F080830A985DB095
:10AB5800BDE8F08F50460D9930AA06F0B7FE0028E0
:10AB6800EDD133ACE1E700BF700600201096B9F1D3
:10AB7800000FE0D0012300228DF80C91069343AD1D
:10AB88008DF897200C93CDE913220E920992119219
:10AB98001BF0020302D00699023106911BF08408CB
:10ABA800329E05D10B9906980F1A002F00F39B804F
:10ABB8006AB101226260319A013601320DF19701C2
:10ABC800072A32963192216000F3D883083463B1A2
:10ABD80002236360319B0236013326AA072B329683
:10ABE8003193226000F3BF830834B8F1800F00F07E
:10ABF800BF82099B0C9A9F1A002F00F3F9821BF45D
:10AC0800807F40F01E820C9B25601E446360319B50
:10AC180032960133072B319300F33F8308341BF03E
:10AC2800040F05D00B9B069A9D1A002D00F3B383E1
:10AC3800DDE90A3206998A42ACBF9B185B180A9371
:10AC4800002E40F00883002331930E9B1BB1504621
:10AC58000E99FFF7B1FA33AC109DA6E60F9B10963C
:10AC6800073323F00703F3E802670F9327F0004345
:10AC78001F931E964FF0FF32DDE91E01B24BCDE95E
:10AC88001667F6F73BF9002840F0F484DDE91E0169
:10AC98004FF0FF32AC4BF6F713F9002840F0EA8486
:10ACA8000022002330463946F6F700F9002840F024
:10ACB800B2879DF8972000210320A44DA44B2BF0C8
:10ACC800800B0E910690B9F1470FD8BF1D46CDE90C
:10ACD800131109910C901191002A3FF459AF069B6A
:10ACE8000133069354E7102F319A41F30D82DFF8B0
:10ACF80064C2214630460D9C2E46CDF854C06546A8
:10AD0800219304E0103F102F01F1080116DD1023F4
:10AD180001321030072ACDE931200D604B60F1DD9A
:10AD28002146504630AA06F0D1FD002840F09B820B
:10AD3800DDE93120103F102F33A9E8DC35460C46F9
:10AD48000646219B013215993E44072ACDE9312652
:10AD58002160676000F381869DF89720083427E713
:10AD68000F9BB9F1430F109603F1040603D01BF0B3
:10AD7800100F00F00185082200212EA8FFF7A8F87F
:10AD88000F9A43AD2EAB29465046126806F06CFD6B
:10AD9800034601330C9001F054820C9B23EAE373C1
:10ADA800069300220F968DF89720ECE600230F9F5C
:10ADB800109657F8045B8DF89730002D00F0008549
:10ADC800B9F1530F00F094861BF01003119340F073
:10ADD8008F86099B002BC1F21B801A4628461199C1
:10ADE80004F010FF0E90002801F081820E9B11994B
:10ADF8005B1B0C9323EAE3734FF07309CDE913113E
:10AE08009DF897200F97099106930E9164E71BF020
:10AE1800200F10963ED00F9B073323F007031846E8
:10AE2800596850F8083B0A460F900029C0F2CA83B7
:10AE380009990029C0F2888253EA02012BF08007A1
:10AE480040F08382099A002A40F08482BB460C9223
:10AE58005CAD64E10B9B5B420B9333784BF0040BC6
:10AE6800CBE53378682B03BF73784BF4007B01364E
:10AE78004BF0400BC1E52B238DF897303378BCE5B8
:10AE880033784BF0080BB8E54BF0100B1BF0200F94
:10AE98001096C0D10F9A1BF0100F52F8043B0F9276
:10AEA80040F0C2831BF0400F00F0BA8343F3C03276
:10AEB80011461BB2B9E71BF0200F109600F0C583AE
:10AEC8000F9B0A9A1B681A60D2175A600F9B0433AB
:10AED8000F93C1E633786C2B03BF73784BF0200BCC
:10AEE80001364BF0100B88E547F630030F9AADF8A2
:10AEF800983052F8043B02210F924FF07809002253
:10AF0800154810964BF0020719900020099D8DF8FE
:10AF18009700002DC0F2EC8053EA020027F0800B66
:10AF280040F0E580002D40F0D285002940F05383A1
:10AF380017F001030C9300F0718330230DF26F15A5
:10AF48008DF86F31EBE000BFFFFFEF7F141F0108A2
:10AF5800101F010860530108201F010810964BF0CC
:10AF6800100B1BF0200200F012830F9B073323F015
:10AF7800070319465A6851F8083B0F9100212BF432
:10AF88008067C2E710964BF0100717F0200200F018
:10AF98000B830F9B0121073323F0070318465A68D8
:10AFA80050F8083B0F90B0E733784BF0800B24E55E
:10AFB800314611F8019BB9F12A0F01F02882A9F155
:10AFC8003003092B98BF002201F2A28011F8019BDF
:10AFD80002EB820203EB4202A9F13003092BF5D9F7
:10AFE80042EAE2730E46099309E533784BF0010B08
:10AFF80003E59DF897203378002A7FF4FEAC2022E1
:10B008008DF89720F9E4504604F09EFD43681846F1
:10B018001D93FFF737F820900746504604F094FD3B
:10B0280083681B93002F3FF463AD1B9A3378002A83
:10B038003FF4E3AC1278002A3FF4DFAC4BF4806BAA
:10B04800DBE4B9F1650F40F33781DDE91601002231
:10B058000023F5F721FF002800F0D8810123636061
:10B06800319B934A01330136072B32963193226084
:10B0780000F332850834279B129A934280F2C982E2
:10B08800189B1A9A1E44C4E90023319B3296013357
:10B09800072B319300F37A830834129B5D1E002D31
:10B0A8007FF7BDAD102D319B40F3EB80DFF80492A4
:10B0B8001027DDF83480CDF8549004E00834103DB2
:10B0C800102D40F3E08001331036072BC4E90097B8
:10B0D800CDE93136F2DD4146504630AA06F0F6FB9E
:10B0E800002840F0C080DDE9313633ACE7E75F4641
:10B0F800012900F02A8102295CAD1ED1199803F0BC
:10B108000F01415C1B0943EA0273120905F8011D8E
:10B1180053EA0201F3D1BB465CAB5B1B0C93099A63
:10B128000C9900238A42B8BF0A46CDE91333069228
:10B138000E939DF897201193CEE503F00701DB08E5
:10B1480043EA4273D208303153EA0206284605F82A
:10B15800011DF2D1FB07DED53029DCD030230238BF
:10B1680005F8013C5CAB1B1ABB4605460C93D6E7B9
:10B178000B9B069A9F1A002F7FF73BAD102F319B30
:10B1880041F35B804B48224631464FF01008064693
:10B198000D9C159004E0103F102F02F1080214DDF9
:10B1A80001331031072BC2E90068CDE93131F2DDF6
:10B1B8002146504630AA06F089FB002853D1DDE924
:10B1C8003131103F102F33AAEADC14460E46013302
:10B1D800159A3E44072BCDE931362260676000F3AB
:10B1E800C084099B0C9A08349F1A002F7FF707AD7B
:10B1F800304A102F319B159221DD32464FF010084E
:10B208002E460D9D04E0103F102F04F1080414DDB4
:10B21800013328491032072BC4E90018CDE931322F
:10B22800F1DD2946504630AA06F050FBD8B9DDE9D1
:10B238003132103F102F33ACEADC35461646013365
:10B24800159A3E44072BCDE931362260676000F33A
:10B2580092810834D3E450460D9930AA06F036FBA3
:10B2680000283FF4F0ACD3460E9B002B3FF467ACAC
:10B2780058460E99FEF7A0FF0D9B9B8903F04003EB
:10B2880061E40C4A1592159A01332E44072B22606B
:10B298006560CDE931367FF7C1AC50460D9930AACB
:10B2A80006F014FB0028DED1329E33ACB7E400BFB1
:10B2B800501F010850530108129B319F012B06F1C2
:10B2C800010607F1010704F1080940F31081012381
:10B2D800072FCDE931762560636000F38081189BE4
:10B2E80001371A9A1E44072FC9E90023CDE93176A0
:10B2F80000F3828109F10809129B0022DDE9160199
:10B308005C1E0023F5F7C8FD002840F009810137CD
:10B3180001352644072FCDE93176C9F80050C9F820
:10B32800044000F3F08009F108091C9B01371E4412
:10B33800C9F80430072F2AABCDE93176C9F80030B7
:10B34800ABDC09F108046AE45F460A2B72F10001DC
:10B3580080F0258330338DF86F310123BB460C9381
:10B368000DF26F15DBE650460D9930AA06F0AEFADD
:10B3780000287FF478AF329E33AC36E450460D99FE
:10B3880030AA159306F0A2FA00287FF46CAF329E1B
:10B39800159B33AC1BE4102D319B40F33187DFF84C
:10B3A800CC821027DDF83490CDF8548004E0103DAD
:10B3B800102D04F1080415DD01331036072BC4E9FC
:10B3C8000087CDE93136F2DD4946504630AA06F00D
:10B3D8007DFA00287FF447AFDDE93136103D102DA6
:10B3E80033ACE9DC0133159A2E44072BC4E9002558
:10B3F800CDE931367FF71CAC50460D9930AA06F0DE
:10B4080065FA00287FF42FAF329E11E427990029AE
:10B4180040F33383DDE911839845A8BF9846B8F116
:10B42800000F0ADD319B46440133072BC4E900585D
:10B438003296319300F33E860834119FB8F1000F1D
:10B44800A8BFA7EB0807002F00F3CB81DDF84490D5
:10B458001BF4806FA94440F0EA81279B129A93421B
:10B46800C0F271821BF0010F40F06D82129AAF1882
:10B47800A7EB0907D51AAF42A8BF2F46002F0BDD4F
:10B48800319B3E440133072BC4F800906760329625
:10B49800319300F385860834002FA8BFED1B002DDB
:10B4A8007FF7BDAB102D319B7FF7EBAEDFF8C09176
:10B4B8001027DDF83480CDF8549004E00834103DAE
:10B4C800102D7FF7E0AE01331036072BC4E9009743
:10B4D800CDE93136F2DD4146504630AA06F0F6F99C
:10B4E80000287FF4C0AEDDE9313633ACE7E71BF066
:10B4F800010F7FF4ECAE0123072FCDE931762560EB
:10B5080063607FF712AF50460D9930AA06F0DEF956
:10B5180000287FF4A8AEDDE931760DF1CC0904E707
:10B52800129B012B7FF701AF112B40F37F87504B04
:10B53800CDF824B010259B46DDF83480159305E03E
:10B5480009F10809103C102C40F33C8301371036F0
:10B55800072FC9E900B5CDE93176F1DD41465046FE
:10B5680030AA06F0B3F900287FF47DAEDDE9317624
:10B578000DF1CC09E6E750460D9930AA06F0A6F978
:10B5880000287FF470AE329E33ACFFF738BB0F99BA
:10B598001BF0100051F8043B55D11BF040054ED06C
:10B5A80002460F919BB2E9E40F9917F0100051F889
:10B5B800043B41D117F040053AD00F9102460121D2
:10B5C8009BB2A2E45B425F464FF02D004FF00101B1
:10B5D80062EB42029AE4099B5CAD0C939FE55046EE
:10B5E8000D9930AA06F072F900287FF43CAEDDE927
:10B5F80031760DF1CC0972E650460D9930AA06F065
:10B6080065F900287FF42FAEDDE931760DF1CC091C
:10B6180072E61BF0010F3FF402AB31E55CAD7EE54D
:10B628001BF4007F40F04F83DA171146FFF7FDBB8C
:10B6380017F4007240F052830F91012165E41BF466
:10B64800007240F046830F9198E41BF0100F40F011
:10B6580094821BF0400F40F0CA831BF4007F00F077
:10B668008C820F9B0A9A1B681A702FE4605301089A
:10B6780050530108DDE9160102460B46F5F73EFC7A
:10B68800002840F01C86B9F1610F00F01F85B9F160
:10B69800410F00F04A85099B013300F0EF8329F040
:10B6A8002003472B00F0E1850E90DDE91612002AF1
:10B6B80013464BF48078C0F2E68400231593DDE945
:10B6C8001623CDE92223A9F14103252B00F20E838D
:10B6D800DFE813F018040C030C030C03D803A504CB
:10B6E8000C030C030C030C030C030C030C030C03DA
:10B6F8000C030C030C030C030C030C030C030C03CA
:10B708000C030C030C030C030C030C030C030C03B9
:10B718000C030C0318040C030C030C03D803A50436
:10B72800A64B109619931BF0200200F01A810F9B6C
:10B73800073323F0070319465A6851F8083B0F915D
:10B748001BF0010F09D053EA020106D030218DF811
:10B7580099904BF0020B8DF8981002212BF480671A
:10B76800FFF7D3BB5F4610960FE41096FFF7F9BBBF
:10B77800934B10961993D6E70F9B43AD1B688DF832
:10B788000C31012306930C93FFF70BBB50460D9920
:10B7980030AA06F09BF800287FF465AD329E33ACE2
:10B7A8007BE440215846FEF70BFE0D9B186018619C
:10B7B800002800F03F8640230D9A5361FFF7DCB85C
:10B7C800099B2946062B28BF06232A4609950E956C
:10B7D800CDE913117B4D06930F970C931191FFF749
:10B7E8007BBA102F319B40F31D86774932464FF0C4
:10B7F80010090E46DDF83480159104E00834103F36
:10B80800102F40F3EE8101331032072BC4E9006991
:10B81800CDE93132F2DD4146504630AA06F056F8FD
:10B8280000287FF420ADDDE9313233ACE7E7129B25
:10B838002246EB180993139B4C46002B3146DDF842
:10B848005080CDF844B0DDF86C90209EDDF834B01F
:10B85800149531DDB8F1000F40F3338108F1FF385A
:10B8680031981D9B013031440728C2E900363291D6
:10B87800319000F389800832099B99F800001F1B5A
:10B888008742A8BF0746002F0CDD319839440130A4
:10B898000728C2E900473291319000F3558199F8A1
:10B8A80000000832002FB4BF0546C51B002D14DC6C
:10B8B8000444139B002BCDDCB8F1000FCEDCCDF88F
:10B8C8006C90A146149D129B1446EB1899450E46A0
:10B8D80028BF9946DDF844B0BFE5102D31983A4BA2
:10B8E80023DD0C9410272C461D4604E0103C102C38
:10B8F80002F1080216DD0130334B10310728C2E986
:10B908000037CDE93101F1DD5946504630AA05F03E
:10B91800DDFF00287FF4A7ACDDE93101103C102CD5
:10B9280033AAE8DC2B4625460C9C0130294407281D
:10B93800CDE931011360556000F3AD8399F800003B
:10B9480008320444B5E7189A1A991644C4E9001253
:10B95800319A32960132072A319200F3C8830834AB
:10B9680084E50F991BF0100051F8043B0AD11BF035
:10B97800400503D002460F919BB2E1E61BF400722A
:10B9880040F09D810F91DBE65946504630AA05F0FC
:10B998009DFF00287FF467AC329933AA6CE707F45F
:10B9A80080610C970E944FF0000E0F46DFF81CB024
:10B9B8001B9C0DF5B87CCDF8189010E0341F0108D9
:10B9C800201F0108481F010850530108CDCCCCCCDA
:10B9D8000A2B72F1000237D343463246AC46991817
:10B9E80041F10001ABFB010626F0030000EB9600D5
:10B9F8004FF0CC36091A581A06FB00F662F1000916
:10BA0800A0FB0B800BFB09660644052008F0010922
:10BA1800A9FB000940184FEA5808303048EAC678B0
:10BA28000EF1010E0CF1FF350CF8010C7608002F11
:10BA3800CED021788E45CBD1BEF1FF0FC8D00A2BCE
:10BA480072F1000280F0DA801B94DDF818900C9FE8
:10BA58000E9CCDF848E0FFF75EBB50460D9930AA22
:10BA6800159305F033FF00287FF4FDAB9DF8972070
:10BA7800329E159B33ACFFF79BB801236360319B63
:10BA8800994A01330136072B32963193226000F32D
:10BA9800FE800834002976D1129A0BF00103134373
:10BAA8003FF4BDA8189B1A9A1E44C4E90023319B91
:10BAB80032960133072B319300F3D38104F1080246
:10BAC80072E0139B09F1FF39013B1393C8E6012982
:10BAD8005F467FF410AB3DE450460D9930AA05F05F
:10BAE800F5FE00287FF4BFAB329E33ACFFF7C3BA34
:10BAF8000DF1B8080822002140462995FEF7E8F91B
:10BB0800099B002BC0F28C8000260697CDF8309058
:10BB1800374699460FE04346504643A905F0A4FE30
:10BB2800421C06F10406384400F0BD83484506DC93
:10BB380000F0FE830746299B9A59002AEBD1DDF8CD
:10BB480030900C97069F79E05946504630AA05F088
:10BB5800BDFE00287FF487AB99F80000329933AA1C
:10BB6800A0E650460D9930AA05F0B0FE00287FF4F3
:10BB78007AAB329E33ACFFF73CB80F9B0A9A1B682E
:10BB88001A60FFF7A3B9189B1A9A1E44C4E9002348
:10BB9800319B32960133072B319300F3628104F114
:10BBA80008020029C0F20B83129901330E44072BB7
:10BBB800CDE93136156051603FF76FAB02F10804EB
:10BBC800FFF72DB8DDF824B00137159B2644072F61
:10BBD800CDE93176C9F80030C9F804407FF7A3AB46
:10BBE80091E416460133159A3E44072BCDE93136C8
:10BBF8002260676000F32981083427E4209B1D999F
:10BC0800ED1A1A46284603F063FF637803B101343E
:10BC18004FF0000EE0E62D228DF89720FFF74BB885
:10BC2800002350461946CDF8008029AA05F042FEA7
:10BC3800034601330C9000F0368329950C9B002BAA
:10BC480031D0632B00F3F780002343AD0E93082215
:10BC580000214046FEF73CF90C9E294633465046E3
:10BC6800CDF8008029AA05F025FE864240F0F2832F
:10BC780000230C9ACDE9133322EAE271AB549DF804
:10BC880097200F97069109931193FFF725B850460F
:10BC98000D9930AA05F01AFE00287FF4E4AA279926
:10BCA800329E33ACF6E60C9B9DF89720CDE9133312
:10BCB8000F970693099311930E93FFF70DB82A4631
:10BCC8000F91DBB23CE543F3C01211465BB2FFF7BC
:10BCD800ACB82A460F91DBB2FFF750B90F912A464C
:10BCE8000121DBB2FFF711B9501F0108099B50462B
:10BCF8000193022300932EAB049329AB039327AB44
:10BD08000293DDE9222304F0DFF81BF0010F05465A
:10BD180040F007822E9B1B1A1293279B1193119BAD
:10BD2800D91C03DB099A9A4280F28E81119BA9F1F2
:10BD38000209013B002127935FFA89F2002B8DF855
:10BD4800A820B6BF2D222B22119B8DF8A920B8BFA1
:10BD5800C3F10103092B40F392820DF1BF073A4664
:10BD6800DFF8D0C21E461046ACFB0321C90801EB20
:10BD78008102A3EB42023032632E00F8012C0B46FD
:10BD880000F1FF32EEDC303302F8013C831EBB4287
:10BD980080F03A830DF1A90213F8011BBB4202F8A7
:10BDA800011FF9D15CAB181AA0F1AD031C93129BCB
:10BDB8001C9A012B1A440C9240F370820C9B189A1F
:10BDC80013440C932BF4806343F4807B00230C9A78
:10BDD800149322EAE272069213931193159B002B97
:10BDE80040F021819DF897200993FEF775BF0F9BBE
:10BDF8000A9A1B681A80FFF769B80D9C50462146BD
:10BE080030AA05F063FDA38903F04003FEF79BBE4B
:10BE18002846FEF737F9119B20EAE0714FF07309C5
:10BE2800CDE913339DF897200F970C90099306914D
:10BE38000E93FEF751BF5046591CFEF7C1FA05464E
:10BE4800002800F0FF820E9001E750460D9930AAB5
:10BE580005F03CFD00287FF406AA329E33ACFFF7BC
:10BE6800F5BA50460D9930AA05F030FD00287FF448
:10BE7800FAA9DDE93136279933AA92E606230E900E
:10BE8800099312E40223099A0132069200932EAB19
:10BE9800069E049329AB039327AB01960293504661
:10BEA800DDE9222304F010F829F02007462F054683
:10BEB80018BF4527064405D12B78302B00F0378171
:10BEC800279B1E440022DDE922010023F4F7E4FF4A
:10BED800002840F022812E9BB34206D230215A1C02
:10BEE8002E9219702E9B9E42F9D8279A11925B1BAD
:10BEF800472F12933FF413AF462F00F02681119B72
:10BF0800013B17E727AADDE9220103F0C7FE00225B
:10BF18004FF07F53F4F758FD02460B46CDE9062350
:10BF280000220023F4F7B8FF08B101232793099BE7
:10BF3800414A591E414BCDE911B4B9F1610F08BF0F
:10BF48001A462E46D346CDF8309013958946DDE93A
:10BF580006459246099207E000220023F4F79CFF69
:10BF6800002840F0D181B9460022354B20462946A9
:10BF7800F4F72AFD0D460446F4F7D6FF8046F4F799
:10BF880035FB02460B4620462946F4F7E1F91AF834
:10BF98000830B9F1FF3F324604460D4609F1FF3734
:10BFA80006F8013BD8D11746264B0022CDE90645B5
:10BFB800DA46DDF83090129CDDF844B0139DF4F7B2
:10BFC80093FF002800F0128209992E9716F8012C89
:10BFD800C97B3346914209D1302003F8010C2E9BCE
:10BFE8005A1E2E9213F8012C9142F6D0392A0BBF13
:10BFF800099A0132927AD2B203F8012C33465B1BBC
:10C008001293279BB9F1610F119303F1FF33279323
:10C0180000F0C28150224FF0410901218EE6099BB0
:10C028000693032332E72D2200238DF897200993E6
:10C03800FEF755BECDCCCCCC341F0108201F01081B
:10C04800000030400000E03FDDE91123934200F397
:10C05800DB801BF0010F119B00F04781189A1344F5
:10C068000C931BF4806F00F07A81119B4FF06709E5
:10C07800002B7DDC0C9B23EAE37306930023C34665
:10C08800CDE91333AAE622912D2103F1004315913E
:10C098002393FFF718BB5946504630AA05F016FC03
:10C0A80000287FF4E0A899F80000329933AA0444E4
:10C0B800FFF7FFBB50460D9930AA05F007FC002892
:10C0C8007FF4D1A8329E33ACFFF7B7B978238DF847
:10C0D800993030238DF89830099B4BF0020B632B75
:10C0E80000F3B980002343AD0E93FFF7DEBA504644
:10C0F8000D9930AA05F0EAFB00287FF4B4A8279B25
:10C10800329E33ACFFF7B2B9AE491591FEF71ABEAD
:10C1180000230E460993FEF772BC279A3346119204
:10C12800E5E6099B4727C618CCE65823CFE7002247
:10C13800DDE922010023F4F7AFFE002800F0278193
:10C14800279B1E441193731B12931199099A0BF0A4
:10C158000103002943EA020340F32D81002B40F03C
:10C1680001814FF06609119B0C931BF4806F81D0FD
:10C178001B990B78FF2B00F061810026119A30463D
:10C1880004E001300131FF2B00F0D880934280F2A7
:10C19800D580D21A4B78002BF3D10B780136F2E711
:10C1A80050460D9930AA05F091FB00287FF45BA852
:10C1B800279D129B329E33AC5D1BFFF76DB94F4232
:10C1C80010312CDADFF800821024CDF8548003E017
:10C1D8000832103F102F24DD01331036072BC2E937
:10C1E8000084CDE93136F3DD50460D9930AA05F0CB
:10C1F8006DFB00287FF437A8DDE9313633AAE8E77C
:10C20800704A1592FFF7EEB8129B189A9A18119B6C
:10C218000C92002B40F3AE804FF06709A5E76A49FE
:10C228001591013315993E44072BCDE9313611603C
:10C23800576000F3B3800832B6E4634A1592FEF7FC
:10C24800C6BF0D9A938943F0400393814FF0FF33A3
:10C258000A93FEF77BBC5046591CFEF7B1F8054619
:10C268000028EED00E90FFF720BA099B002B7FF430
:10C278001BAA099B0E9301230993FFF716BA0029FD
:10C2880040F0828030228DF8AA200DF1AB023033C5
:10C2980002F8013B2AABD31A1C9388E51BF0010F67
:10C2A8003FF490AD8AE50022D3460D9B0E92B3F978
:10C2B8000C3043F040030D9A9381FEF7D5BF179BCE
:10C2C8000320002BB8BF2D224FF00003A8BF9DF814
:10C2D800972019460E933D4D3D4BB8BF8DF89720DA
:10C2E8002BF0800B0690FEF7EEBC0C93B9E6099B89
:10C2F8004FF07309CDE913009DF897200F97069327
:10C308000C930990FEF7E8BC49460029DA46DDF8A7
:10C318003090129CDDF844B0139DFFF66FAE4B1CB5
:10C3280030223146334401F8012B9942FBD166E6AD
:10C33800099BDDF83090069F0C937FE4CDE9130646
:10C348001B911192DDE91332209913440C9AC346CC
:10C3580001FB03230C9323EAE37306933EE54FF0B6
:10C36800670987E61346189A4FF0660913440B4489
:10C378000C93FAE6C3F101031A4422EAE2734FF080
:10C3880067090C92069379E60DF1AA027FE7069BEE
:10C39800C3F10103279394E570223EE650460D99B8
:10C3A80030AA05F093FA00287EF45DAFDDE9313656
:10C3B80033AAFFF7F9BB6BB901234FF0660906935F
:10C3C8000C935BE660530108505301081C1F0108D9
:10C3D800181F0108189B4FF0660903F1010B099B10
:10C3E8005B440C9323EAE373069347E60022DDE9F6
:10C3F80006011C4BF4F750FD00283FF4FFAD18F080
:10C40800010F3FF4FBADDFE502231C93CFE40F9A45
:10C4180073780E4652F8041B0F9241EAE1720992B2
:10C42800FEF7EBBA104A1592FFF7DCBB0E4B1593DB
:10C43800FFF7CABB0C23CBF8003007E70023CDE990
:10C4480013337FE70D9BD346B3F90C300E9043F0BE
:10C45800400330E70D9BD346B3F90C3043F040035B
:10C4680029E700BF0000E03F505301082DE9F04FD5
:10C47800DDB0914609911C4683460F9303F064FB97
:10C48800036818461993FDF7FDFD0822189000214E
:10C498002CA8FDF71DFDBBF1000F04D0DBF83430EC
:10C4A800002B01F03480099B5A6EB3F90C30D50784
:10C4B80002D4980540F16986990407D4099943F490
:10C4C80000534A6E8B8122F400524A661A0740F1E3
:10C4D800C880099A1269002A00F0C38003F01A0282
:10C4E8000A2A00F0CD80002300249E46CDE931338E
:10C4F800002333AACDE91634DA4614464D46CDE971
:10C508001BEE3092CDF868E0CDF880E0CDF874E00D
:10C51800CDF82CE0CDF848E02F468B4BD3F8E460FB
:10C5280003F00CFB0DF1B00C03463A46504628A91F
:10C53800CDF800C0B047002800F0C180C0F2B78035
:10C54800289B252B01D00744E7E7B7EB05080646EB
:10C5580040F0B98000224FF0FF3393460A937B786E
:10C568007E1C8DF897200C9299460136A9F120037C
:10C578005A2B00F2EB80DFE813F0F702E900E9003C
:10C58800F302E900E900E900D502E900E9006A00E0
:10C598006602E90062026F02E9006B025B005B0061
:10C5A8005B005B005B005B005B005B005B00E9001D
:10C5B800E900E900E900E900E900E9006101E900B2
:10C5C800F1013503610161016101E900E900E90058
:10C5D800E9003103E900E9000103E900E900E900A5
:10C5E8000A02E9001F03E900E900C806E900E900BA
:10C5F800E900E900E900E900E900E9006101E90072
:10C60800F1013B0261016101610115033B02ED018A
:10C61800E9004D03E900BB02C3068C02ED01E90005
:10C628000A027200C506E900E900E906E90072009D
:10C638000022A9F1300316F8019B02EB820203EBFA
:10C648004202A9F13003092BF5D90C928EE70F9B12
:10C6580053F8042B002A0C920F93C0F2ED81337823
:10C6680082E7099D5846294603F0E4F8002841F07E
:10C678009D83B5F90C3003F01A020A2A7FF433AF10
:10C688000999B1F90E20002AFFF62DAF4A6ED50799
:10C6980002D4980541F1E28023464A465846099952
:10C6A80001F0DCFC0B900B985DB0BDE8F08F082220
:10C6B80000212CA8FDF70CFC012007442DE7B7EB5F
:10C6C8000508064610D0329BC4E90058434432930B
:10C6D800319B0133072B319310DC08340B9B434407
:10C6E8000B93002E7FF436AF329B002B41F08F80E6
:10C6F8000022099B3192B3F90C3019E05046099990
:10C7080030AA01F027FD80B933ACE7E75046099914
:10C7180030AA01F01FFD002800F08580D3460E9B4B
:10C728001BB158460E99FDF747FD099BB3F90C302C
:10C73800099A526ED10740F103815B0601F14283E9
:10C748000B985DB0BDE8F08F700600201096B9F127
:10C75800000FC9D0012300228DF80C91069343AD38
:10C768008DF897200D93CDE913220E920A9211921B
:10C778001BF0020302D00699023106911BF08408CF
:10C78800329E05D10C9906980F1A002F00F39B8052
:10C798006AB101226260319A013601320DF19701C6
:10C7A800072A32963192216000F3BE83083463B1C0
:10C7B80002236360319B0236013326AA072B329687
:10C7C8003193226000F3BD830834B8F1800F00F084
:10C7D800C2820A9B0D9A9F1A002F00F3FD821BF458
:10C7E800807F40F021820D9B25601E446360319B51
:10C7F80032960133072B319300F32F8308341BF053
:10C80800040F05D00C9B069A9D1A002D00F3A483F3
:10C81800DDE90B3206998A42ACBF9B185B180B9373
:10C82800002E7FF473AF002331930E9B1BB150464B
:10C838000E99FDF7C1FC33AC109D6DE60F9B109669
:10C84800073323F00703F3E802670F9327F0004349
:10C858001F931E964FF0FF32DDE91E01AC4BCDE968
:10C868001667F4F74BFB002840F0F484DDE91E015D
:10C878004FF0FF32A64BF4F723FB002840F0EA8480
:10C888000022002330463946F4F710FB002841F017
:10C89800F1809DF89720002103209E4D9E4B2BF0A0
:10C8A800800B0E910690B9F1470FD8BF1D46CDE910
:10C8B80013110A910D901191002A3FF459AF069B6C
:10C8C8000133069354E7102F319A41F3F481DFF8CE
:10C8D8004CC221463046099C2E46CDF854C06546C8
:10C8E800219304E0103F102F01F1080116DD1023F9
:10C8F80001321030072ACDE931200D604B60F1DD9F
:10C908002146504630AA01F025FC00287FF406AFE6
:10C91800DDE93120103F102F33A9E8DC35460C46FD
:10C928000646219B013215993E44072ACDE9312656
:10C938002160676000F3DB859DF89720083427E7BE
:10C948009A053FF5FAAE099CA06DFDF799FBB4F97D
:10C958000C30F2E633784BF0200B05E60F9BB9F16B
:10C96800430F109603F1040600F01C851BF0100F0E
:10C9780040F018850F9B43AD1B688DF80C310123DF
:10C9880006930D9300220F968DF89720EBE600236F
:10C998000F9F109657F8045B8DF89730002D00F024
:10C9A800F084B9F1530F00F0C8851BF01003119300
:10C9B80040F0C3850A9B002BC0F216871A4628460A
:10C9C800119903F01FF90E90002801F0A5820E9B23
:10C9D80011995B1B0D9323EAE3734FF07309CDE9BB
:10C9E80013119DF897200F970A9106930E9163E70C
:10C9F8001BF0200F109600F0FC800F9B073323F0EC
:10CA080007031846596850F8083B0A460F90002952
:10CA1800C0F2FF830A990029C0F2728253EA020128
:10CA28002BF0800740F06D820A9A002A40F06E824F
:10CA3800BB460D925CAD65E10C9B5B420C93337871
:10CA48004BF0040B90E52B238DF8973033788BE56A
:10CA580033784BF0800B87E5314611F8019BB9F12B
:10CA68002A0F01F0CD82A9F13003092B98BF0022CB
:10CA780001F2298111F8019B02EB820203EB4202C9
:10CA8800A9F13003092BF5D942EAE2730E460A935D
:10CA98006CE547F630030F9AADF8983052F8043B2E
:10CAA80002210F924FF0780900221D4810964BF092
:10CAB80002071A9000200A9D8DF89700002DC0F2F9
:10CAC8000A8153EA020027F0800B40F00381002D11
:10CAD80040F02285002940F0998417F001030D9356
:10CAE80000F0858330230DF26F158DF86F3109E161
:10CAF8001BF0200F109600F095830F9B0B9A1B6874
:10CB08001A60D2175A600F9B04330F9394E600BF44
:10CB1800FFFFEF7F141F0108101F01088053010851
:10CB2800201F0108504603F00FF8436818461D936C
:10CB3800FDF7A8FA20900746504603F005F88368E9
:10CB48001B93002F3FF48BAD1B9A3378002A3FF4D8
:10CB58000BAD1278002A3FF407AD4BF4806B03E568
:10CB680033784BF0010BFFE49DF897203378002AC7
:10CB78007FF4FAAC20228DF89720F5E410964BF05C
:10CB8800100B1BF0200200F0E3820F9B073323F009
:10CB9800070319465A6851F8083B0F9100212BF4F6
:10CBA800806787E73378682B03BF73784BF4007B83
:10CBB80001364BF0400BD7E410964BF0100717F0F6
:10CBC800200200F0D4820F9B0121073323F00703D2
:10CBD80018465A6850F8083B0F906BE733784BF0CB
:10CBE800080BC1E44BF0100B1BF0200F10967FF4DC
:10CBF80004AF0F9A1BF0100F52F8043B0F9240F04D
:10CC080003831BF0400F00F0FB8243F3C032114650
:10CC18001BB2FCE633786C2B03BF73784BF0200B08
:10CC280001364BF0100B9FE4B9F1650F40F32081FA
:10CC3800DDE9160100220023F4F72EF9002800F0A0
:10CC4800C68101236360319BB54A01330136072B46
:10CC580032963193226000F364840834279B129A39
:10CC6800934280F29A82189B199A1E44C4E90023C1
:10CC7800319B32960133072B319300F377830834C5
:10CC8800129B5D1E002D7FF7BAAD102D319B40F32E
:10CC9800D880DFF890921027DDF82480CDF85490E2
:10CCA80004E00834103D102D40F3CD8001331036D8
:10CCB800072BC4E90097CDE93136F2DD41465046ED
:10CCC80030AA01F047FA00287FF428ADDDE93136B3
:10CCD80033ACE7E75F46012900F0138102295CAD18
:10CCE8001ED11A9803F00F01415C1B0943EA027335
:10CCF800120905F8011D53EA0201F3D1BB465CABEA
:10CD08005B1B0D930A9A0D9900238A42B8BF0A4605
:10CD1800CDE9133306920E939DF897201193CBE536
:10CD280003F00701DB0843EA4273D208303153EAC3
:10CD38000206284605F8011DF2D1FE07DED5302986
:10CD4800DCD03023023805F8013C5CAB1B1ABB462B
:10CD580005460D93D6E70C9B069A9F1A002F7FF77E
:10CD680038AD102F319B41F384806E4822463146FE
:10CD78004FF010080646099C159004E0103F102F4C
:10CD880002F1080215DD01331031072BC2E90068F2
:10CD9800CDE93131F2DD2146504630AA01F0DAF909
:10CDA80000287FF4BBACDDE93131103F102F33AAE6
:10CDB800E9DC14460E460133159A3E44072BCDE9AB
:10CDC80031362260676000F3C5820A9B0D9A0834E9
:10CDD8009F1A002F7FF703AD524A102F319B1592EF
:10CDE80023DD32464FF010082E46099D04E0103F1F
:10CDF800102F04F1080416DD01334A491032072BBD
:10CE0800C4E90018CDE93132F1DD2946504630AA8F
:10CE180001F0A0F900287FF481ACDDE93132103F40
:10CE2800102F33ACE8DC354616460133159A3E44DC
:10CE3800072BCDE931362260676000F37D81083425
:10CE4800CDE4384A1592159A01332E44072B2260F7
:10CE58006560CDE931367FF7D1AC5046099930AAE3
:10CE680001F078F900287FF459AC329E33ACC6E45F
:10CE7800129B319F012B06F1010607F1010704F10E
:10CE8800080940F315810123072FCDE93176256084
:10CE9800636000F3CC82189B0137199A1E44072F50
:10CEA800C9E90023CDE9317600F3B48209F1080914
:10CEB800129B0022DDE916015C1E0023F3F7ECFF4C
:10CEC800002840F00E81013701352644072FCDE9AF
:10CED8003176C9F80050C9F8044000F3F58009F12B
:10CEE80008091C9B01371E44C9F80430072F2AABD8
:10CEF800CDE93176C9F80030AFDC09F108047EE4E9
:10CF08005F460A2B72F1000180F09E8230338DF863
:10CF18006F310123BB460D930DF26F15F2E600BF8A
:10CF2800501F0108705301085046099930AA1593FB
:10CF380001F010F900287FF4F1AB329E159B33AC59
:10CF480035E45046099930AA01F004F900287FF425
:10CF5800E5AB329E33AC38E4102D319B40F3378774
:10CF6800DFF8E4821027DDF82490CDF8548004E03F
:10CF7800103D102D04F1080415DD01331036072B80
:10CF8800C4E90087CDE93136F2DD4946504630AA7A
:10CF980001F0E0F800287FF4C1ABDDE93136103D3F
:10CFA800102D33ACE9DC0133159A2E44072BC4E964
:10CFB8000025CDE931367FF72BAC5046099930AAC8
:10CFC80001F0C8F800287FF4A9AB329E20E4279925
:10CFD800002940F3E780DDE911839845A8BF98460A
:10CFE800B8F1000F0ADD319B46440133072BC4E931
:10CFF80000583296319300F345860834119FB8F1F2
:10D00800000FA8BFA7EB0807002F00F31E83DDF869
:10D0180044901BF4806FA94440F05185279B129AD5
:10D028009342C0F2D7811BF0010F40F0D381129ACE
:10D03800AF18A7EB0907D51AAF42A8BF2F46002F94
:10D048000BDD319B3E440133072BC4F80090676029
:10D058003296319300F37A860834002FA8BFED1B6F
:10D06800002D7FF7CCAB102D319B7FF7EAAEDFF8B0
:10D07800DC911027DDF82480CDF8549004E00834C2
:10D08800103D102D7FF7DFAE01331036072BC4E9B2
:10D098000097CDE93136F2DD4146504630AA01F01D
:10D0A80059F800287FF43AABDDE9313633ACE7E7CD
:10D0B8001BF0010F7FF4E7AE0123072FCDE931768E
:10D0C800256063607FF70DAF5046099930AA01F0DB
:10D0D80041F800287FF422ABDDE931760DF1CC0967
:10D0E800FFE6129B012B7FF7FCAE112B40F39B87C9
:10D0F800564BCDF828B010259B46DDF824801593B3
:10D1080005E009F10809103C102C40F3C4820137EE
:10D118001036072FC9E900B5CDE93176F1DD414672
:10D12800504630AA01F016F800287FF4F7AADDE986
:10D1380031760DF1CC09E6E75046099930AA01F09D
:10D1480009F800287FF4EAAA329E33ACFFF747BB00
:10D158000F9951F8043B0F911BF010017FF41EAD9D
:10D168001BF0400000F0A6820A469BB216E50F9914
:10D1780051F8043B0F9117F010013FD117F0400010
:10D1880037D00A469BB2012194E4099DA86DFCF7AB
:10D1980075FFB5F90C30FFF78FB91BF0010F3FF49D
:10D1A8002EAB60E501236360319B294A01330136C8
:10D1B800072B32963193226000F347850834002903
:10D1C80040F02482129A0BF0010313433FF417AB8B
:10D1D800189B199A1E44C4E90023319B32960133E7
:10D1E800072B319300F32D8304F108021FE25CAD95
:10D1F80088E517F400721CBF0246DBB2012159E42E
:10D208001BF4007F40F0EA82DA1711460029BFF6C6
:10D2180001AC5B425F464FF02D004FF0010162EB1D
:10D22800420248E41BF0100F40F0EA811BF0400F67
:10D2380040F0CE821BF4007F00F0E2810F9B0B9A36
:10D248001B681A705FE400BF80530108705301081F
:10D25800501F0108DDE9160102460B46F3F74EFEA2
:10D26800002840F04086B9F1610F00F00985B9F156
:10D27800410F00F0D6820A9B013300F0FE8529F0A9
:10D288002003472B00F0B7850E90DDE91612002A1F
:10D2980013464BF48078C0F2C48400231593DDE96B
:10D2A8001623CDE92223A9F14103252B00F20F8291
:10D2B800DFE813F01E030D020D020D02D902AB03C5
:10D2C8000D020D020D020D020D020D020D020D02DE
:10D2D8000D020D020D020D020D020D020D020D02CE
:10D2E8000D020D020D020D020D020D020D020D02BE
:10D2F8000D020D021E030D020D020D02D902AB0331
:10D3080010963EE45F46109659E4B94B10961A936E
:10D318001BF020026CD00F9B073323F0070319463C
:10D328005A6851F8083B0F911BF0010F09D053EAD6
:10D33800020106D030218DF899904BF0020B8DF840
:10D34800981002212BF48067FFF7B4BBA94B109605
:10D358001A93DDE75046099930AA00F0FBFE002831
:10D368007FF4DCA9329E33ACFFF733BA50460999F3
:10D3780030AA00F0EFFE00287FF4D0A9329E33AC2B
:10D388007EE40A9B2946062B28BF06232A460A95CF
:10D398000E95CDE91311984D06930F970D931191A2
:10D3A800FFF78ABA082200212EA8FCF791FD0F9AF0
:10D3B80043AD2EAB29465046126804F055FA034691
:10D3C80001330D9000F027860D9B23EAE373069343
:10D3D800FFF7D8BA189A19991644C4E90012319A75
:10D3E80032960132072A319200F3588408341EE637
:10D3F8000F9951F8043B0F911BF0100194D11BF0C9
:10D40800400000F05E810A469BB28DE70A9B5CAD46
:10D418000D9377E45046099930AA00F09BFE002846
:10D428007FF47CA9DDE931760DF1CC0940E5504661
:10D43800099930AA00F08EFE00287FF46FA9DDE973
:10D4480031760DF1CC0926E507F48061CDE90D743C
:10D458004FF0000E0F46DFF8A4B11B9C0DF5B87C09
:10D46800CDF8189006E00A2B72F1000237D3434634
:10D478003246AC46991841F10001ABFB010626F093
:10D48800030000EB96004FF0CC36091A581A06FB39
:10D4980000F662F10009A0FB0B800BFB096606444D
:10D4A800052008F00109A9FB000940184FEA5808AF
:10D4B800303048EAC6780EF1010E0CF1FF350CF851
:10D4C800010C7608002FCED021788E45CBD1BEF145
:10D4D800FF0FC8D00A2B72F1000280F0BE821B94A5
:10D4E800DDF818900D9F0E9CCDF848E006E45046F4
:10D4F800099930AA159300F02DFE00287FF40EA993
:10D508009DF89720329E159B33ACFFF741B95846DA
:10D51800FCF7EEFAFEF7C7BF01295F467FF4DEABE2
:10D52800F4E45046099930AA00F014FE00287FF46C
:10D53800F5A8329E33ACFFF791BB0DF1B80808226D
:10D54800002140462995FCF7C3FC0A9B002BC0F23A
:10D55800758200260697CDF834B037469B460FE013
:10D568004346504643A904F07FF9431C06F10406DC
:10D57800384400F08C84584506DC00F0AD8407463A
:10D58800299B9A59002AEBD1DDF834B00D97069FF4
:10D598000D9B002B00F04D83632B40F31C845046F9
:10D5A800591CFCF70DFF0546002800F04B850E902E
:10D5B800082200214046FCF78BFC0D9E2946334685
:10D5C8005046CDF8008029AA04F074F9864240F04C
:10D5D800328500230D9ACDE9133322EAE271AB5468
:10D5E8009DF897200F9706910A931193FFF764B956
:10D5F800341F0108201F0108481F0108CDCCCCCCDE
:10D608000F9B0B9A1B681A60FFF77DBA189B199A33
:10D618001E44C4E90023319B32960133072B319312
:10D6280000F30F8104F108020029C0F29E831299C9
:10D6380001330E44072BCDE93136156051603FF7B1
:10D648000CAC02F10804FFF7DAB8102F319B40F355
:10D65800C184A54932464FF010090E46DDF82480F2
:10D66800159104E00834103F102F40F3D98101339D
:10D678001032072BC4E90069CDE93132F2DD4146A9
:10D68800504630AA00F066FD00287FF447A8DDE97F
:10D69800313233ACE7E7DDF828B00137159B264473
:10D6A800072FCDE93176C9F80030C9F804407FF773
:10D6B80016AC09E51BF400721CBF0246DBB2FFF78B
:10D6C8006DBA1BF400721CBF0246DBB22CE60A9B43
:10D6D80050460193022300932EAB049329AB039386
:10D6E80027AB0293DDE9222302F0EEFB1BF0010FCA
:10D6F800054640F0E4822E9B1B1A1293279B119338
:10D70800119BDA1C03DB0A9A9A4280F2B881119BBA
:10D71800A9F10209013B002127935FFA89F2002B46
:10D728008DF8A820B6BF2D222B22119B8DF8A92099
:10D73800B8BFC3F10103092B40F375830DF1BF078F
:10D748003A46DFF8A8C11E461046ACFB0321C908BB
:10D7580001EB8102A3EB42023032632E00F8012C68
:10D768000B4600F1FF32EEDC303302F8013C831E39
:10D77800BB4280F01D840DF1A90213F8011BBB42C6
:10D7880002F8011FF9D15CAB181AA0F1AD031C9384
:10D79800129B1C9A012B1A440D9240F373830D9B24
:10D7A800189A13440D932BF4806343F4807B002371
:10D7B8000D9A149322EAE272069213931193159B21
:10D7C800002B40F026819DF897200A93FFF774B844
:10D7D8000F9B0B9A1B681A80FFF795B943F3C01289
:10D7E80011465BB2FFF713B92846FCF74BFC119BB7
:10D7F80020EAE0714FF07309CDE913339DF89720C3
:10D808000F970D900A9306910E93FFF755B850465F
:10D81800099930AA00F09EFC00283EF469AFFEF793
:10D8280084BF58238DF8993030238DF898300A9B9F
:10D838004BF0020B632B00F31183002343AD0E93CF
:10D8480023E55046099930AA00F084FC00287EF4AC
:10D8580065AFDDE93136279933AAE5E6886DFCF72F
:10D868000FFCFEF719BF02230A9A013206920093B1
:10D878002EAB069E049329AB039327AB0196029324
:10D888005046DDE9222302F01FFB29F02007462F2E
:10D89800054618BF4527064405D12B78302B00F0E4
:10D8A8001782279B1E440022DDE922010023F3F79B
:10D8B800F3FA002840F046822E9BB34206D230216C
:10D8C8005A1C2E9219702E9B9E42F9D8279A1192B3
:10D8D8005B1B472F12933FF413AF462F00F00682CD
:10D8E800119B013B17E700BF70530108CDCCCCCC8E
:10D8F80027AADDE9220102F0D1F900224FF07F5377
:10D90800F3F762F802460B46CDE90623002200230E
:10D91800F3F7C2FA08B1012327930A9BB54A591EA7
:10D92800B54BCDE91194B9F1610F08BF1A462E46DF
:10D93800CDF834B01395D346DDE9064589469246BD
:10D948000A9207E000220023F3F7A6FA002840F025
:10D95800FF82B9460022A94B20462946F3F734F83E
:10D968000D460446F3F7E0FA8046F2F73FFE02461A
:10D978000B4620462946F2F7EBFC1AF80830B9F1B5
:10D98800FF3F324604460D4609F1FF3706F8013BD2
:10D99800D8D117469A4B0022CDE90645DA46DDF87C
:10D9A8004490129CDDF834B0139DF3F79DFA0028DB
:10D9B80000F002830A992E9716F8012CC97B33468A
:10D9C8008A4209D1302003F8010C2E9B5A1E2E9250
:10D9D80013F8012C8A42F6D0392A0BBF0A9A013271
:10D9E800927AD2B203F8012C33465B1B1293279B21
:10D9F800B9F1610F119303F1FF33279300F0BC8253
:10DA080050224FF04109012189E60A9B069303231E
:10DA18002DE72D2200238DF897200A93FEF74FBF9C
:10DA280016460133159A3E44072BCDE9313622605C
:10DA3800676000F307820834FFF7E9BA002350460D
:10DA48001946CDF8008029AA03F034FF03460133B4
:10DA58000D9000F01C8229959AE5209B1D99ED1ADE
:10DA68001A46284602F034F8637803B101344FF0BF
:10DA7800000EFCE42D228DF89720FEF70CBFDDE99F
:10DA88001123934200F3AC811BF0010F119B00F0AE
:10DA98005082189A13440D931BF4806F00F039825A
:10DAA800119B4FF06709002B00F334810D9B23EA8B
:10DAB800E37306930023C346CDE913337FE6129B35
:10DAC8002246EB180A93139B4C46002B3146DDF88F
:10DAD8005080CDF844B0DDF86C90209EDDF824B07D
:10DAE80014952EDDB8F1000F7DDD08F1FF3831986F
:10DAF8001D9B013031440728C2E90036329131902C
:10DB080066DC08320A9B99F800001F1B8742A8BFF1
:10DB18000746002F0BDD3198394401300728C2E948
:10DB28000047329131906FDC99F800000832002FDD
:10DB3800B4BF0546C51B002D15DC0444139B002B00
:10DB4800D0DCB8F1000FD0DCCDF86C90A146149D64
:10DB5800129B1446EB1899450E4628BF9946DDF8E6
:10DB680044B0FFF75BBA102D3198264B23DD0D9496
:10DB780010272C461D4604E0103C102C02F1080228
:10DB880016DD01301F4B10310728C2E90037CDE9F7
:10DB98003101F1DD5946504630AA00F0DBFA002881
:10DBA8007EF4BCADDDE93101103C102C33AAE8DC71
:10DBB8002B4625460D9C013029440728CDE9310123
:10DBC800136055604EDC99F8000008320444B5E74C
:10DBD8005946504630AA00F0BDFA00287EF49EADA2
:10DBE800329933AA8EE7139B09F1FF39013B13934E
:10DBF8007DE700BF341F0108201F010800003040E6
:10DC08000000E03F705301085946504630AA00F022
:10DC1800A1FA00287EF482AD99F80000329933AA5F
:10DC280085E722912D2103F1004315912393FFF7F6
:10DC38003ABB0D9B9DF89720CDE913330F970693B8
:10DC48000A9311930E93FEF737BE5046099930AAEE
:10DC580000F080FA00287EF461AD2799329E33AC3B
:10DC6800FFF7ADBA5946504630AA00F073FA0028BB
:10DC78007EF454AD99F80000329933AA04445DE764
:10DC88007823CFE55046099930AA00F063FA0028B6
:10DC98007EF444AD329E33ACFFF7B0B950460999D3
:10DCA80030AA00F057FA00287EF438AD279B329E40
:10DCB80033ACFFF7BCB9B1491591FEF733BE0A9BE7
:10DCC8004727C618EFE500230E460A93FEF74EBC19
:10DCD8000022DDE922010023F3F7DEF8002800F036
:10DCE8005581279B1E441193731B129311990A9A0D
:10DCF8000BF00103002943EA020340F36E81002B75
:10DD080040F0D1804FF06609119B0D931BF4806F92
:10DD18003FF4CCAE1B990B78FF2B00F088810026CE
:10DD2800119A304604E001300131FF2B00F0C38026
:10DD3800934280F2C080D21A4B78002BF3D10B7833
:10DD48000136F2E7279A33461192C1E55046099900
:10DD580030AA00F0FFF900287EF4E0AC279D129B62
:10DD6800329E33AC5D1BFFF778B94F4210314CDA65
:10DD7800DFF80C821024CDF8548003E00832103FFD
:10DD8800102F44DD01331036072BC2E90084CDE99A
:10DD98003136F3DD5046099930AA00F0DBF9002846
:10DDA8007EF4BCACDDE9313633AAE8E7099B5B6E4B
:10DDB800DF0707D4099B9B899E0503D4099B986DAF
:10DDC800FCF75EF94FF0FF330B93FEF7B9BC6B4AD3
:10DDD8001592FFF7E8B8002343AD0E93FFF7E8BBB1
:10DDE800129B189A9A18119B0D92002B40F3A3804E
:10DDF8004FF067098AE70A9B002B7FF445AA0A9B24
:10DE08000E9301230A93FFF740BA5D491591013338
:10DE180015993E44072BCDE931361160576000F360
:10DE2800BA80083203E4002940F08F8030228DF850
:10DE3800AA200DF1AB02303302F8013B2AABD31A0A
:10DE48001C93A5E45046099930AA00F083F90028EC
:10DE58007EF464AC329E33ACFFF7D9B85046591CF7
:10DE6800FCF7AEFA0546002800F0D5800E90FFF7C3
:10DE78000CBA434A1592FEF79EBF06230E900A93EA
:10DE8800FFF703BA1BF0010F3FF48DAC87E40022C3
:10DE9800D346099B0E92B3F90C3043F04003099A1C
:10DEA8009381FEF73CBC1346189A4FF06609134459
:10DEB8000B440D932AE7CDE913061B911192DDE976
:10DEC8001332209913440D9AC34601FB03230D9383
:10DED80023EAE373069372E40A9BDDF834B0069FE5
:10DEE8000D93FFF755BB179B0320002BB8BF2D22BE
:10DEF8004FF00003A8BF9DF8972019460E93214DB7
:10DF0800214BB8BF8DF897202BF0800B0690FEF7B9
:10DF1800CABC4FF06709C9E50A9B4FF07309CDE900
:10DF280013009DF897200F9706930D930A90FEF71C
:10DF3800C3BC0D93B0E5C3F101031A4422EAE273AE
:10DF48004FF067090D920693B4E50DF1AA0272E746
:10DF580049460029DA46129CDDF84490DDF834B0D1
:10DF6800139DFFF641AD4B1C30223146334401F876
:10DF7800012B8B42FBD138E5702244E58053010820
:10DF8800705301081C1F0108181F0108069BC3F1E4
:10DF98000103279386E45046099930AA00F0DAF87D
:10DFA80000287EF4BBABDDE9313633AAFFF73FBB6F
:10DFB80002231C93FFF7ECBB0022DDE90601254B89
:10DFC800F2F76AFF00283FF40FAD18F0010F3FF495
:10DFD8000BADEFE4204A159223E52BB901234FF04E
:10DFE800660906930D9365E5189B4FF0660903F1E2
:10DFF800010B0A9B5B440D9323EAE373069359E5EF
:10E008000F9A73780E4652F8041B0F9241EAE17298
:10E018000A92FEF7A9BA099AB2F90C3043F0400304
:10E028009381FEF785BB0C4B1593FFF736BB002396
:10E03800CDE9133343E7099BD346B3F90C3043F0DA
:10E0480040032CE7099BD346B3F90C300E9043F0FC
:10E05800400324E70000E03F70530108F0B54FF497
:10E0680080640026ADF26C4D1AADCDE905461F4619
:10E0780006460095049515468B8916A823F00203D9
:10E08800ADF80C304B6E02941993CB890C46ADF861
:10E098000E30CB6907934B6A0993FBF7EBFF2A46CF
:10E0A8003B4669463046FEF7E1F9051E07DB69463F
:10E0B800304601F081F9002818BF4FF0FF35BDF850
:10E0C8000C305B0603D5A38943F04003A38116985F
:10E0D800FBF7D2FF28460DF26C4DF0BD2DE9F84F45
:10E0E8004B6E90469C042ED5936812684BB30D4630
:10E0F800064602F1080959E9022A5FEA9A0716D08A
:10E108000024A2F1040B01E0A7420ED02A463046B3
:10E118005BF8041F01F02EFC431C04F10104F3D149
:10E128000023C8E90133BDE8F88FD8F808302AF091
:10E13800030AA3EB0A03C8F8083009F10809002B01
:10E14800D9D10020ECE701F061F90023C8E90133D7
:10E15800BDE8F88F10B4946814B110BCFFF7BEBFC7
:10E168002046546010BC704784462DE9F04F0E4697
:10E178001546E146C7B016AF0822002138461C46AE
:10E18800CDE906560B93FBF7A3FEB9F1000F04D0B7
:10E19800D9F83430002B00F0D086079A536EB2F9C4
:10E1A8000C20DE0702D4950540F1A485900407D41D
:10E1B800079942F400524B6E8A8123F400534B6650
:10E1C800110740F1BD80079B1B69002B00F0B88048
:10E1D80002F01A030A2B00F0C28000231DAA9246FF
:10E1E800CDE91B33CDE91033DFF844B21A920E9310
:10E1F80008930F93069DDBF8E44001F09FFC2A4644
:10E20800034614A948460097A047002800F0C68096
:10E21800C0F2BC80149B252B01D00544EBE7069B7C
:10E228000446EE1A40F0BE8000234FF0FF326978B2
:10E2380005926C1C8DF84B30099303930134A1F1BE
:10E2480020035A2B00F2F680DFE813F01303F400E2
:10E25800F4000D03F400F400F400ED02F400F400FF
:10E268006A003F03F40003022303F4001D035B006C
:10E278005B005B005B005B005B005B005B005B00BE
:10E28800F400F400F400F400F400F400F400F400E6
:10E29800F400B6014302F400F400F400F400F400C2
:10E2A800F400F400F400F400F4000902F400F400AF
:10E2B800F4008F01F4005C02F400F400F205F400AD
:10E2C800F400F400F400F400F400F400F400F400A6
:10E2D800F400B601DB01F400F400F400AA02DB014B
:10E2E8007400F400E402F400D5021506B3027400C9
:10E2F800F4008F017200EF05F400F4001906F40031
:10E3080072000022A1F1300314F8011B02EB820213
:10E3180003EB4202A1F13003092BF5D909928EE7EC
:10E328000B9B53F8042B002A09920B93C0F28E81A1
:10E33800217883E7039B217843F0200303937DE74B
:10E34800079D4846294601F075FA002840F0D48612
:10E35800B5F90C2002F01A030A2B7FF43EAF079997
:10E36800B1F90E30002BFFF638AF4B6EDE0702D442
:10E37800950540F18686DDE906212346484600F0EA
:10E38800E7FE0890089847B0BDE8F08F0822002102
:10E398003846FBF79DFD012005442CE7069B044603
:10E3A800EE1A12D0069B1C9ACAE900361B9B32440F
:10E3B8000133072B1C921B9311DC0AF1080A089BF6
:10E3C80033440893002C7FF42FAF1C9B002B40F0A4
:10E3D80074860022079B1B92B3F90C301CE0002ABC
:10E3E80000F04984484607991AAAFFF777FE80B9D2
:10E3F8000DF1740AE3E7484607991AAAFFF76EFE7B
:10E40800002800F09D800C9B1BB148460C99FBF737
:10E41800D3FE079BB3F90C30079A526ED10740F12F
:10E428009A805B0600F17486089847B0BDE8F08FC3
:10E438007006002006940029C7D000238DF84B30C1
:10E4480001238DF8B41004932DAC0A9300260C9682
:10E458000596039BDDE91B1213F0840301F1010CFF
:10E4680060460D9305D1099B049D5D1B002D00F3AB
:10E478004F839DF84B3083B101230132CAF8043031
:10E4880007280DF14B03CDE91B02CAF8003000F351
:10E49800098301460AF1080A0130D6B10223023283
:10E4A800CAF80430072813ABCDE91B02CAF80030BC
:10E4B80040F31183002A00F0FD83484607991AAA01
:10E4C800FFF70CFE00289ED1DDE91B120DF1740A3E
:10E4D800481C0D9B802B00F03B82059B0A9D5D1B11
:10E4E800002D00F38F820A9B07281A44CDE91B02EE
:10E4F800CAF80040CAF8043040F32782002A00F026
:10E508005083484607991AAAFFF7E8FD00287FF4C8
:10E518007AAF1C9A0DF1740A039B580705D5099B1D
:10E5280004995C1A002C00F34783DDE9083104984C
:10E538008142ACBF5B181B180893002A7FF45BAFBD
:10E5480000231B930C9B1BB119464846FBF734FE6E
:10E558000DF1740A4EE69A053FF563AF079CA06D6E
:10E56800FBF78EFDB4F90C305BE700230B9E069495
:10E5780056F8044B8DF84B30002C00F0F6845329E4
:10E5880000F09A84039B13F0100540F09584059BD6
:10E59800002BC0F27F851A462946204601F032FB3F
:10E5A8000C90002800F07285031B0A9323EAE3739A
:10E5B8000C95049300F036BD0B9B4329069403F198
:10E5C800040503D0039BDC0640F15D84082200218A
:10E5D80018A8FBF77DFC0B9A2DAC18AB21464846D2
:10E5E800126803F041F9034601330A9000F07C8574
:10E5F8000A9B23EAE373049300230B958DF84B30B1
:10E6080024E7039B069498066BD50B9B073323F0EE
:10E61800070318465A6850F8083B11460B90002A21
:10E62800C0F25881059A002AC0F26181039A22F04B
:10E638008002039253EA010240F05981059B002BA6
:10E6480040F0398504930A9346AC62E1099B5B422A
:10E658000993039B217843F004030393EEE5039B9E
:10E66800069443F0100111F0200200F007830B9B81
:10E67800073323F0070318465A6850F8083B0B90F5
:10E68800002021F480640394059C8DF84B0084429B
:10E6980063DB53EA020421F4906140F04C84039A4E
:10E6A8000391059B002B50D1002840F01A8312F0EB
:10E6B80001020A9200F01A8330238DF817319DF871
:10E6C8004B3004920DF21714002B40F027810C9365
:10E6D80029E1039B069443F010030393039B9806D8
:10E6E80093D403990B9AC90652F8043B00F17D8331
:10E6F80003994E0640F1438443F3C0310B921BB299
:10E708000A468CE7039B069443F0100212F020019E
:10E7180000F0C3820B9B073323F0070318465968A0
:10E7280050F8083B0B9000208DF84B000598002806
:10E73800C0F2FA8222F08000039053EA010040F010
:10E74800D680059B0120002BAED0012800F0B384B1
:10E75800002302281A4600F0C48146AC03F00701E2
:10E76800DB0843EA4273D208303153EA02052046F7
:10E7780004F8011DF2D1039BDD0740F1C081302967
:10E7880000F0BD813023059A023804F8013C46ABFD
:10E798001B1A9A42B8BF1A4604460A930492B8E074
:10E7A8002178039B682900F0CD8343F0400303934D
:10E7B80044E5039B0B9A43F00203039347F63003A7
:10E7C800ADF84C3052F8043BB4490B920022069441
:10E7D8000F9100218DF84B1005990029C0F2818115
:10E7E800039C53EA020024F0800140F0798122461C
:10E7F8000220039155E7039B06949C0640F1FE8294
:10E808000B9B089A1B681A60D2175A600B9B04333B
:10E818000B93EFE42178039B6C2900F09A8343F073
:10E82800100303930AE5484601F08EF94368184639
:10E838001193FBF727FC10900546484601F084F930
:10E8480083680E93002D3FF473AD0E9B2178002B47
:10E858003FF4F4AC1B78002B3FF4F0AC039B43F47B
:10E8680080630393EAE4039B217843F00103039355
:10E87800E4E49DF84B302178002B7FF4DFAC2023B3
:10E888008DF84B30DAE4039B217843F0800303933F
:10E89800D4E4204610F8011B2A2900F04584A1F190
:10E8A8003003092B98BF002200F2FD8310F8011BEA
:10E8B80002EB820203EB4202A1F13003092BF5D9E6
:10E8C80042EAE27304460593B9E42B2321788DF8D4
:10E8D8004B30B3E42D228DF84B20059A5B4261EB57
:10E8E8004101002A03DB039A22F0800203920A2BDB
:10E8F80071F1000280F01E823033DBB28DF81731DF
:10E90800059B0DF21714012BB8BF012304930123B3
:10E918000A939DF84B30002B3FF4D9AE00230C939B
:10E92800049B01330493039B13F002063FF491AD5B
:10E93800049B0226023304938BE501230A9A1D9453
:10E948001B931E921C920DF1740A0AF1080AE3E562
:10E95800099B049D5D1B002D7FF7BFAD102D40F373
:10E96800DC83DFF83C81D44643461026A046DDF818
:10E978001CA01C4606E0881C19460CF1080C103D2A
:10E98800102D1ADD4B1C1032072BCCE90046CDE9BF
:10E998001B32F0DD002A7BD0514648461AAAFFF701
:10E9A8009DFB00287FF42FADDDE91B12103D102DD3
:10E9B8000DF1740C01F10100E4DC2346E246444603
:10E9C80098462A440728CDE91B02CAF80080CAF8ED
:10E9D800045040F39781002A00F030834846079995
:10E9E8001AAAFFF77BFB00287FF40DADDDE91B12A7
:10E9F800059B0A9D0DF1740A5D1B002D01F10100B4
:10EA08007FF771AD102DDFF898802EDDD4461026E3
:10EA1800AA462546079C08E0881C19460CF1080CF4
:10EA2800AAF1100ABAF1100F1CDD4B1C1C48103259
:10EA3800072BCCE90006CDE91B32EDDD1AB32146E0
:10EA480048461AAAFFF74AFB00287FF4DCACDDE948
:10EA58001B12AAF1100ABAF1100F0DF1740C01F192
:10EA68000100E2DC2C465546E2462A440728CDE957
:10EA78001B02CAF80080CAF8045000F3EB800AF1C0
:10EA8800080A01302FE5012011460DF1740CC7E783
:10EA9800012011460DF1740C71E700BF201F010819
:10EAA800905301086AB1484607991AAAFFF716FB5E
:10EAB80000287FF4A8ACDDE91B120DF1740A481C8C
:10EAC800EBE4002E00F0AB810222012013AB1D9372
:10EAD8000DF1740A1E9201460AF1080A0130F8E4A1
:10EAE80003910F9846AC03F00F01415C1B0943EA00
:10EAF8000273120904F8011D53EA0201F3D1059AC1
:10EB080046AB1B1B9A42B8BF1A460A93049200E709
:10EB1800102D40F3CD82DFF8DC82D6461023A246C2
:10EB28004446DDF81C8008E001F1020C01460EF1B4
:10EB3800080E103D102D1BDD481C10320728CEE9A9
:10EB48000043CDE91B02EFDD2AB3414648461AAA25
:10EB5800FFF7C4FA00287FF456ACDDE91B12103D1C
:10EB6800102D4FF010030DF1740E01F1010CE3DCD0
:10EB7800A04660465446F2462A440728CDE91B02BF
:10EB8800CAF80080CAF8045000F3998001460AF1D7
:10EB9800080A01306DE411464FF0010C0DF1740EB6
:10EBA800C7E7039B1B925C074BD5099B04995C1A2A
:10EBB800002C46DD0DF1740A102C1B9940F3878256
:10EBC800DFF8308210254646DDF81C8006E0881CF8
:10EBD80019460AF1080A103C102C19DD4B1C10329A
:10EBE800072BCAE90065CDE91B32F0DD22B34146A7
:10EBF80048461AAAFFF772FA00287FF404ACDDE948
:10EC08001B12103C102C0DF1740A01F10100E5DC17
:10EC1800B04622440728CAE90084CDE91B027FF7E1
:10EC280084AC72B1484607991AAAFFF757FA002828
:10EC38007FF4E9AB1C9A78E4012011460DF1740ABF
:10EC4800C9E70499DDE908328A42ACBF9B185B1812
:10EC5800089375E4002A3FF470AE484607991AAA4B
:10EC6800FFF73CFA00287FF4CEAB1B981C9A0DF1F5
:10EC7800740A013037E41B92FFF7BABB0B9811F006
:10EC8800100450F8043B40F0AE8011F0400500F04D
:10EC9800A68022460B909BB2F2E40B9812F0100467
:10ECA80050F8043B38D112F0400531D021460B9082
:10ECB8009BB238E5012011460DF1740A09E4002AD7
:10ECC80000F0EB80484607991AAAFFF707FA0028D0
:10ECD8007FF499ABDDE91B120DF1740A481CFFF7AC
:10ECE800C8BB059B46AC04930A9312E6059B46AC49
:10ECF80004930EE6079DA86DFBF7C0F9B5F90C2043
:10ED0800FFF754BA01460AF1080A0130FFF7E5BBDC
:10ED180012F4007140F098810B9000208DF84B00A0
:10ED280005980028BFF606AD0A2B039271F1000280
:10ED3800FFF4E2AD039A984602F480624FF0000CAB
:10ED480013462D4D0DF58C7ECDF810A0CDF82890EA
:10ED580007E0B8F10A0F71F100013BD3C84631460C
:10ED6800A64618EB010242F10002A5FB020626F0B6
:10ED7800030000EB96004FF0CC36121AB8EB0200F5
:10ED880006FB00F661F1000AA0FB059005FB0A6688
:10ED98000644052009F0010AAAFB000A80184FEA78
:10EDA8005909303049EAC6790CF1010C0EF1FF34EB
:10EDB8000EF8010C7608002BCBD00E9A127862451B
:10EDC800C7D1BCF1FF0FC4D0B8F10A0F71F100012F
:10EDD80080F0E180DDF810A0DDF828908FE611F4CE
:10EDE800007240F036810B904AE4D9170B920A461C
:10EDF80015E400BFA0530108CDCCCCCC039BD806AA
:10EE080000F1AE80039B590600F13181039B9A05FE
:10EE180040F1A6800B9B089A1B681A70F6E411460D
:10EE280001200DF1740AFFF754BB039A06946DE4B0
:10EE3800A94B06940F93039B13F0200264D00B9BFD
:10EE4800073323F0070318465A6850F8083B0B901D
:10EE5800039CE6070AD553EA020007D08DF84D1047
:10EE680044F00201039130218DF84C10039921F4EC
:10EE780080610391ADE403990694FFF7F4BB974BC7
:10EE880006940F93D7E70B9B2DAC1B688DF8B43015
:10EE9800012304930A93FFF7AFBB9DF84B30002B77
:10EEA80000F0DF8001200DF14B0302461D930DF1A8
:10EEB800740A1E90FFF7EDBA0822002118A81594CD
:10EEC800FBF706F8059B002B77DB0025CDF810A093
:10EED800A8469A460FE018AB48462DA902F0C4FC94
:10EEE800431C05F10405404400F0FE80504506DC53
:10EEF80000F016818046159B5A59002AEBD1DDF89F
:10EF080010A0CDF8288066E0039C0B9814F010043C
:10EF180050F8043B0DD1039A12F0400203D0224668
:10EF28000B909BB294E7039C14F4007440F0968015
:10EF380022460B908CE703910FE44846FAF7D8FD78
:10EF4800FFF72BB943F40073617803930134FFF79B
:10EF580075B943F02003617803930134FFF76EB964
:10EF68000B9B089A1B681A6050E4059B5C4C062BA7
:10EF780028BF0623CDE90A360493FFF767BA039939
:10EF88000B928D054CBF43F3C011D9170A4648BFF1
:10EF98005BB2FFF744BB0C93109B1199E41A1A4615
:10EFA800204600F095FD0E990C9B4A7812B10A464E
:10EFB80001320E924FF0000CD0E618AB00930023FC
:10EFC8004846194615AA02F075FC034601330A9013
:10EFD80000F08A8015940A9B0BB3632B4DDD4846DD
:10EFE800591CFBF7EDF9044600287DD00C90082247
:10EFF800002118A8FAF76CFF0A9D18AB0093214668
:10F008002B46484615AA02F055FC854240F09780E9
:10F0180000230A9AA35422EAE273049302E00A9BAB
:10F0280004930C939DF84B301BB100230B9605936A
:10F0380076E40B9605931E46FFF70BBA012011469E
:10F048000DF1740AFFF749BA29460B90DBB2FFF7B6
:10F058006ABB2A460B90DBB2FFF712BB0B90DBB200
:10F06800F6E6114601200DF1740AFFF716BA0B9B5C
:10F07800089A1B681A80FFF7C9BB00232DAC0C93B4
:10F08800B5E7886DFAF7FCFFFFF775B9059B0493A0
:10F098000A93C7E72046FAF7F5FF20EAE0730C95D4
:10F0A8000A900493BEE7002304460593FFF7C7B808
:10F0B800DFF8308060E5302320E4484607991AAA33
:10F0C800FFF70CF800283FF484A9FFF7A2B9DFF88E
:10F0D8001480481C9DE500BF341F0108201F01084B
:10F0E800481F0108A0530108079AB2F90C3043F0F1
:10F0F80040039381FFF790B9079B5B6EDB0707D44A
:10F10800079B9B899F0503D4079B986DFAF7B8FF67
:10F118004FF0FF330893FFF787B9DFF8308050E4EA
:10F12800DDE904A30A9356E70B9B617853F8042B97
:10F1380004460B9342EAE2730593FFF77FB8079AF8
:10F14800938943F040039381FFF75DB99053010819
:10F15800F0B54FF480640026ADF26C4D1AADCDE9E0
:10F1680005461F4606460095049515468B8916A840
:10F1780023F00203ADF80C304B6E02941993CB893F
:10F188000C46ADF80E30CB6907934B6A0993FAF732
:10F1980071FF2A463B4669463046FEF7E5FF051EE5
:10F1A80007DB6946304600F007F9002818BF4FF022
:10F1B800FF35BDF80C305B0603D5A38943F0400347
:10F1C800A3811698FAF758FF28460DF26C4DF0BD4A
:10F1D80070B500293FD006460C4610B1436B002B92
:10F1E8003CD0636EB4F90C20DD0732D4900538D5D5
:10F1F8002146304600F04CF8E36A054633B1304604
:10F20800E16998470028B8BF4FF0FF35A3891A066F
:10F2180039D4216B41B104F14003994202D0304600
:10F22800FAF7CAFF00232363616C21B13046FAF76D
:10F23800C3FF00236364FAF779FC0022636EA2819E
:10F24800DB071CD5A06DFAF717FFFAF775FC2846FF
:10F2580070BD002ACCD10025284670BDFAF748FCBD
:10F26800BFE7A06DFAF70AFFB4F90C30002BBFD145
:10F27800636ED907EFD4A06DFAF702FFEBE7A06D34
:10F28800FAF7FEFEDEE730462169FAF795FFC0E798
:10F29800B1F90C20F8B516070C46074648D449685A
:10F2A80042F400630029A3815FDDA56A002D3DD0EB
:10F2B800002112F480523E683960E16961D101236E
:10F2C8003846A847451C02466AD0B4F90C30A56AEE
:10F2D800E169580705D56368D21A236B0BB1E36B54
:10F2E800D21A00233846A847411C4CD13968B4F9D2
:10F2F8000C301D293FD82F4ACA40D2073BD50022DF
:10F3080062602269DD04226023F40062A28101D5D3
:10F31800002943D0216B3E6041B104F1400399427A
:10F3280002D03846FAF748FF002323630020F8BDCF
:10F338000E69002EFAD0920718BF00230D6808BF87
:10F348004B690E60AD1B8B600CE02B463246D4F83F
:10F3580024C03846E169E047B0F1000CA5EB0C0584
:10F36800664406DD002DF0DCE0E7E16B00299CDC5B
:10F37800DCE7B4F90C3043F040034FF0FF30A381D1
:10F38800F8BD226DA5E70022B4F90C30626022694D
:10F39800226023F40062DB04A281BBD52065B9E7B3
:10F3A8003B68002B91D01D2B01D0162BE1D13E607C
:10F3B800BCE700BF0100402038B505460C4608B13F
:10F3C800436B03B3B4F90C0088B1636EDB0701D457
:10F3D80081050FD528462146FFF75AFF636E05467B
:10F3E800DA0702D4A3899B0508D5284638BD054607
:10F3F800284638BDA06DFAF741FEEBE7A06DFAF795
:10F408003FFE284638BDFAF773FBDBE79368002B0D
:10F4180000F0F0802DE9F04FB1F90CC090461CF0D7
:10F42800080F81460C4683B02BD00B694BB31CF0F8
:10F438000207D8F8006032D04FF0000A5546D4F8D9
:10F4480024B0E169AB4FC5B1BD422B46524628BF37
:10F458003B464846D847002840F3C280D8F80830D1
:10F4680082441B1A2D1AC8F80830002B00F0AE8011
:10F47800D4F824B0E169002DE6D1D6E900A5083614
:10F48800E1E72146484600F0D5F9002840F0AD8074
:10F49800B4F90CC0D8F800601CF00207CCD11CF0FD
:10F4A800010A63D157462368A16818468B46002F86
:10F4B80058D01CF4007F00F0B180B9420A4600F22F
:10F4C800DD801CF4906F2FD0216962695D1A02EB10
:10F4D800420202EBD2726B1C52103B44934292BF21
:10F4E80093469B461A461CF4806F00F0E68011464E
:10F4F8004846FAF765FF002800F0F5802A4621699A
:10F508000190F1F7EBF9A289019B22F4906242F095
:10F518008002A2815819C4F814B0ABEB05053A462D
:10F52800BB462361A56020603D46002751460192F5
:10F5380000F050FAA1682368019AA1EB0B011A4464
:10F54800A1602260D8F80830AA445B1BC8F80830CC
:10F55800002B3BD02368A16818468B46B4F90CC031
:10F56800002FA6D1D6E900A708369EE73846BB4645
:10F578003D46002D40D0002845D03A46D4E904C382
:10F588002068AA4228BF2A466045A16804D901EB31
:10F59800030A524500F38280934272DC5A46484679
:10F5A800E169D4F824C0E047B0F1000A18DDB7EBF0
:10F5B8000A070FD00120D8F80830D344A3EB0A0378
:10F5C800A5EB0A05C8F80830002BD2D1002003B0FB
:10F5D800BDE8F08F21464846FFF7EEFE0028EAD046
:10F5E800B4F90C3043F04003A3814FF0FF3003B06F
:10F5F800BDE8F08F00207047756833460836002D47
:10F60800FAD0D3F800B02A460A21584600F0FAFA90
:10F61800002865D00130A0EB0B07AEE722699A42BB
:10F6280014D36569BD4211D86FF00043BB4228BFAF
:10F638003B4693FBF5F3524605FB03F34846656AE0
:10F64800E169A847051ECBDD7F1B7BE7B94228BFD0
:10F6580039460D46184651462A4600F0BBF9A168BE
:10F668002368491B2B44A16023600029ECD1214663
:10F678004846FFF7A1FE0028E6D0B1E7BB463A4668
:10F6880052E75946019200F0A5F9019AA3689246FB
:10F698009B1AA36023681344236088E7594652469F
:10F6A80000F098F923682146534448462360FFF741
:10F6B80083FE00283FF47BAF92E7484601F020FF25
:10F6C800034600287FF426AF48462169FAF774FDFF
:10F6D8000C22B4F90C30C9F8002023F0800381E72C
:10F6E8006A1C17464AE70C22B4F90C30C9F8002006
:10F6F80078E700BF00FCFF7F2DE9F041B1F90C303D
:10F708000C46990796B008D5012204F14303C4E9D1
:10F718000432236016B0BDE8F081B4F90E10064635
:10F72800002926DB6A4600F013FA00281FDB019D3A
:10F738004FF4806805F47045A5F50055B5FA85F5D0
:10F748004FF400676D0941463046FAF739FEE8B1D3
:10F75800B4F90C30C4F8148043F0800320602061B1
:10F76800A3813DBB3B43A38116B0BDE8F081B4F94A
:10F778000C3013F0800519D04FF0400800254146A1
:10F7880030462F46FAF71CFE0028E1D1B4F90C30B8
:10F798009A05BFD4012123F0030304F1430243F087
:10F7A8000203C4E90421A3812260B3E74FF480680F
:10F7B8002F46C8E73046B4F90E1000F0DDF910B94D
:10F7C800B4F90C30CEE7A38923F0030343F0010317
:10F7D8001BB2C7E770B50C46B1F90E1015460029E3
:10F7E8001E4696B014DB6A4600F0B2F900280FDB1B
:10F7F80001994FF4806301F47041A1F50051B1FA09
:10F8080081F14FF40060490931602B6016B070BD7A
:10F81800A18911F0800106D00021402308463160FB
:10F828002B6016B070BD4FF48063084631602B60C2
:10F8380016B070BD38B52F4B05461B680C4613B182
:10F848005A6B002A4BD0B4F90C3018071CD5226922
:10F8580022B313F0010107D000206169A06049427A
:10F86800A1613AB1002038BD980758BF6169A1600D
:10F87800002AF7D1190658BF1046F4D543F04003C3
:10F88800A3814FF0FF3038BDD9062CD55A0712D4C2
:10F89800226943F00803A381002ADAD103F4207116
:10F8A800B1F5007FD5D021462846FFF725FFB4F9EA
:10F8B8000C302269CDE7216B51B104F1400291422D
:10F8C80004D02846FAF778FCB4F90C3000222263F9
:10F8D8000021226923F02403C4E90021D9E718464E
:10F8E800FAF706F9AFE7092243F040032A60A3813B
:10F8F800C7E700BF3401002070B582B006460D4648
:10F90800144600F01BF9012802D16B1EFE2B26D9E4
:10F9180004F15C032A46304601A901F0A5FF431C07
:10F9280020D078B1A3689DF80410013B002BA36098
:10F9380004DAA269934208DB0A2906D023685A1C14
:10F9480022601970284602B070BD2246304602F087
:10F9580045F80130F6D14FF0FF3002B070BD8DF898
:10F968000450DFE7A3894FF0FF3043F04003A38141
:10F97800F3E700BF30B51446526E0546D007B4F918
:10F988000C3083B001D49A051CD5980406D4626E55
:10F9980043F4005342F40052A3816266224628468B
:10F9A800FFF7AAFF636E0546DA0702D4A3899B0511
:10F9B80002D5284603B030BDA06DFAF761FB284692
:10F9C80003B030BDA06D0191FAF758FBB4F90C30C3
:10F9D8000199DAE788420ED98B1883420BD900EBDC
:10F9E800020C002A6DD0624613F801CD994202F844
:10F9F80001CDF9D170470F2A0FD8034602F1FF3C19
:10FA0800002A5ED00CF1010C013B8C4411F8012B4B
:10FA1800614503F8012FF9D1704740EA01039B07BC
:10FA280050D1A2F1100370B501F1200C23F00F059D
:10FA380001F1100E00F11004AC441B095EF8105CD3
:10FA48000EF1100E44F8105C5EF81C5C103444F89B
:10FA58001C5C5EF8185C44F8185C5EF8145CE645BB
:10FA680044F8145CEAD1013312F00C0F01EB0311D6
:10FA780002F00F0400EB031328D08E46043C24F058
:10FA880003064FEA940C1E441C1F5EF8045B44F8FE
:10FA9800045FB442F9D10CF1010402F0030203EB54
:10FAA800840301EB840102F1FF3C4AB10CF1010C23
:10FAB800013B8C4411F8012B614503F8012FF9D162
:10FAC80070BD7047034602F1FF3C9BE72246EAE718
:10FAD80040EA01039B0710B524D1032A22D98E4698
:10FAE8008446DEF800407146A4F1013323EA04039A
:10FAF80013F0803F0EF1040E15D1043A032A4CF896
:10FB0800044BEED8714601F1FF3E52B163461EF830
:10FB1800011F541E03F8011B41B122469C46002ACE
:10FB2800F4D110BD844601F1FF3EEEE79444002C69
:10FB3800F7D003F8011B6345FBD110BD014B93F8C7
:10FB480028017047700600200048704760070020B1
:10FB580070B50026074D0446084611462E60F1F799
:10FB680059FC431C00D070BD2B68002BFBD02360D0
:10FB780070BD00BF3C1D0020002238B5064D04466C
:10FB880008462A60F1F7F4FB431C00D038BD2B6807
:10FB9800002BFBD0236038BD3C1D0020002238B567
:10FBA800064D044608462A60F1F7F2FD431C00D0D2
:10FBB80038BD2B68002BFBD0236038BD3C1D0020CE
:10FBC80038B5074D074C2C1BA41005D0013C55F83F
:10FBD800043D9847002CF9D1BDE8384002F096B8AA
:10FBE800C8550108C4550108082802D14FF48050AF
:10FBF800704708B5FAF710FA162203464FF0FF309F
:10FC08001A6008BD5FFA81FC810744D00346511E83
:10FC180022B909E09A0709D0013905D318460278B4
:10FC280001336245F6D17047002070471846032912
:10FC38000CD80029F8D00346014401E08B42F3D0E8
:10FC4800184613F8012B6245F8D1704710B50CEB34
:10FC58000C24024604EB044402E00439032915D9B4
:10FC6800104652F8043B6340A3F1013E2EEA030319
:10FC780013F0803FF1D00346014401E08B4208D0E5
:10FC8800184613F8012B6245F8D110BD104600291B
:10FC9800F1D1002010BD1146C9E700BFF8B5002713
:10FCA800DFF858C021F00043634504460D4617604D
:10FCB80021D8844653EA0C0C1DD0DFF844C0164600
:10FCC80001EA0C0C0A46BCF1000F09D100220D4BC9
:10FCD800F0F77AFE6FF0350704460A4621F0004334
:10FCE8001B156FF31E52A3F2FE333B4442F07F55BF
:10FCF800336045F4001520462946F8BDFFFFEF7F25
:10FD08000000F07F000050432DE9F8431B4D0646E4
:10FD1800286898460F469146FAF7B0F9184B1C68C0
:10FD28001CB3286865681F2D22DC4EB96B1C023590
:10FD3800636044F82570FAF7A3F90020BDE8F8835A
:10FD4800012304EB8501C1F88890D4F88821AB40E1
:10FD58001A43022EC4F88821C1F80881E6D1D4F8E4
:10FD68008C211A43C4F88C21E0E7064C1C60D8E7C4
:10FD7800FAF786F94FF0FF30E0E700BF580200209D
:10FD88004C1D0020841D00202DE9F04F03690C69EB
:10FD980085B0A342C0F291808146013C01F114056F
:10FDA80009F1140855F8243058F824C001339C454B
:10FDB800BCFBF3F64FEA840005EB840708EB8402EA
:10FDC80043D34FF0000CAA46CDE90105C646634669
:10FDD80065469346CDF80C805AF8040BDEF80020EF
:10FDE8001FFA80FC06FB0C554FEA10484FEA154CE9
:10FDF80006FB08CCADB290B2401B18441FFA8CF336
:10FE0800C3EB204303EB124380B240EA034057455B
:10FE18004EF8040B4FEA1C454FEA2343DCD2DDE9D8
:10FE28000105DDF80C8058F8003073B9ABF1040215
:10FE3800904504D307E0904504F1FF3403D252F80B
:10FE48000439002BF7D0C9F81040484601F01EFAD3
:10FE580000282EDB4146002255F8040BD1F800C0DB
:10FE68001FFA80FE1FFA8CF3A3EB0E031344020C57
:10FE7800C2EB234202EB1C429BB243EA0243AF426D
:10FE880041F8043B4FEA2242E6D258F8242008EB16
:10FE980084036AB9043B434504D807E0984504F154
:10FEA800FF3403D253F80429002AF7D0C9F81040C8
:10FEB8000136304605B0BDE8F08F002005B0BDE83A
:10FEC800F08F00BF000000002DE9F04F16461F46D6
:10FED800816B9DB0CDE90667299D039049B1012347
:10FEE800C26B044693408B604A6000F073FF0023A6
:10FEF800A363B7F10009B4BF012300232B60784B3B
:10FF0800BCBF29F00049CDF81C9033EA090300F082
:10FF1800AD80DDE906341846214600220023CDE9EC
:10FF28000401F0F7B9FF804668B10123289A1360ED
:10FF38002A9B13B16B4B2A9A13606B4B0893089852
:10FF48001DB0BDE8F08F1AAB01931BAB009303986B
:10FF5800DDE9042301F076FA5FEA1955824640F09C
:10FF68009B80DDE91A85454405F23243202B40F396
:10FF78008B83C3F1400309FA03F905F2124326FA09
:10FF880003F349EA0300F0F721FB0123013D119334
:10FF9800A1F1F8710022554BF0F7DAF94AA3D3E939
:10FFA8000023F0F711FD4AA3D3E90023F0F7D2F9B3
:10FFB800064628460F46F0F719FB47A3D3E9002366
:10FFC800F0F702FD02460B4630463946F0F7C2F913
:10FFD80006460F46F0F7A8FF0022044609900023C2
:10FFE80030463946F0F762FF002840F02383099C29
:08FFF800A8EB050808F1FF3336
:020000040801F1
:10000000162C0A9300F28F81DDE904013A4B03EBD1
:10001000C403D3E90023F0F74DFF002872D0631E1C
:1000200009930023109308F1FF33002BC0F2828163
:1000300000230B93099B002B6ADA099B0B9A0E9302
:10004000D21A5B420F9300230993269B0B92092B34
:1000500068D8052B40F321830025043B2693269B7B
:10006000023B032B00F23F86DFE813F070046D04BF
:100070006404480442F20F73289AC9F3130959EA39
:10008000060913601CD12A9B002B00F04C861B4BE9
:10009000089308332A9A089813601DB0BDE8F08FC2
:1000A000DDE90412C2F31303084643F07F51CDF893
:1000B0004480A5F2FF35DDF8688041F440116DE71A
:1000C0002A9B002B40F0F5830D4B08933BE700BFC4
:1000D00061436F63A787D23FB3C8608B288AC63F4E
:1000E000FB799F501344D33F0000F07F511F01085C
:1000F000501F01080000F83FE85301089C1F010849
:10010000A81F0108B8F1000F40F3A88410900B90CD
:10011000DDE9092313440A9300230F93269B0E92D3
:10012000092B96D9002301254FF0FF3B26932793F7
:100130000C950021039BCDF860B0D963039800F0C3
:1001400027FE0890002800F0D785039B089ABBF192
:100150000E0F9A6300F21981002D00F016810E999E
:10016000002940F34984B44B01F00F0203EBC203B2
:10017000C8054FEA2115D3E9006740F10A84DDE99B
:100180000401AE4B4FF00309D3E90823F0F74AFD11
:10019000CDE9120105F00F058DB1DFF8A082E90766
:1001A00009D5D8E9002330463946F0F711FC064658
:1001B0000F4609F101096D1008F10808EFD1DDE9DA
:1001C00012013B463246F0F72DFD07468846109B4C
:1001D00043B1002238464146994BF0F76BFE0028A8
:1001E00040F010854846F0F705FA3A464346F0F7E6
:1001F000EFFB0022934BF0F7B1F80446A1F15075E4
:10020000BBF1000F00F0AA800E9BCDF848B0199307
:1002100041463846F0F78CFE1299874BCDE91445DC
:1002200003EBC10353E902340546CDE91634F0F778
:10023000E1F90B46024641463846F0F78DF8089F33
:100240000C9B30357E1CECB2804689463546002B2F
:1002500000F06E84DDE9162300207B49F0F7E2FC14
:10026000DDE91423F0F778F83C7042464B4604462B
:100270000D46F0F73DFE002840F0BB84CDF850A0BD
:10028000CDF858B00027AB46A246129D2AE00137B0
:10029000AF4280F201855046594600226B4BF0F781
:1002A00097FB0022694B82468B4640464946F0F751
:1002B0008FFB89468046F0F73BFE0446F0F79AF93B
:1002C00002460B4640464946F0F746F8303452465F
:1002D0005B4606F8014B80468946F0F7EBFD0028A7
:1002E00040F0D78442464B4600205549F0F734F899
:1002F00052465B46F0F7DEFD0028C8D0199B374612
:10030000DDF850A0089A03F1010802E0974200F0DE
:100310009F843E4617F8013D392BF7D00133DBB2FD
:1003200045463B7079E10123109308F1FF33002B20
:10033000BFF67EAEC8F101030B9300230A9379E662
:100340004846F0F757F93A464346F0F741FB00229A
:100350003C4BF0F703F80446A1F1507538460022F3
:100360003B4B4146EFF7F8FF22462B4606460F4629
:10037000F0F7BEFD002840F07A8430463946224628
:1003800005F10043F0F796FD28BB1B9B002BC0F244
:1003900091800E9A0E2A00F38D80274B0E9A03EB64
:1003A000C203D3E90034CDE90634279B002B19DAC8
:1003B000BBF1000F16DC0ED1DDE906010022244B53
:1003C000F0F706FB02460B46DDE90401F0F77CFD81
:1003D000002800F04C8400231F46089E0493279BAE
:1003E000DD432DE2089B5D1CDDE90678DDE90401B3
:1003F0003A464346F0F716FCF0F79AFD0646F0F74A
:10040000F9F83A464346F0F7E3FA02460B46DDE9CF
:100410000401EFF7A1FF089A06F13003BBF1010FC9
:100420002F46137000F025830125CDF810A0A846B3
:10043000DDE9069A2CE000BFE8530108C05301082B
:100440000000F03F00001C400000E03F000024409E
:10045000000014404A46534620462946F0F7E2FB86
:10046000F0F766FD0646F0F7C5F84A465346F0F742
:10047000AFFA08F101080B46024629462046EFF77D
:100480006BFF06F13003D84507F8013B00F0EF821F
:100490000022834BF0F79CFA0022002304460D460D
:1004A000F0F7FEFC0028D5D00E9D3E46DDF810A0EA
:1004B0000135B2E00C9A002A40F0D68000231F4696
:1004C0000F9E0B9D0C9365B10A9900290B4608DD20
:1004D000A942A8BF2B460B9AED1AD21ACB1A0B923F
:1004E0000A930F9B53B10C9B13B1002E40F0FC827A
:1004F00051460F9A039800F0FDFD824601210398B2
:1005000000F018FD099B0490002B40F0BD81269B54
:10051000012B40F3D38101200A9A104410F01F00F0
:1005200000F09980C0F12003042B40F3E2810B9B83
:10053000C0F11C00034402440B9305440A920B9B38
:10054000002B05DD51461A46039800F02DFE824629
:100550000A9B002B05DDDDE903011A4600F024FEAD
:100560000490109B002B40F07481BBF1000F40F30E
:100570004B810C9B002B40F0A2800E9D0135012683
:10058000DDE90394DDF8208007E0514600230A22CC
:10059000484600F02DFC8246013621465046FFF7C2
:1005A000F7FBB34500F1300008F8010BEDDCBBF1BF
:1005B000000FCCBF5E46012681460024089B03EB5A
:1005C000060B51460122039800F0EEFD0499824685
:1005D00000F060FE002840F3F081089A02E09345A5
:1005E00000F005821BF8013C5E46392B0BF1FF3B06
:1005F000F5D001338BF80030DDE90381404600F08F
:10060000EDFB57B12CB1BC4203D02146404600F06F
:10061000E5FB3946039800F0E1FB5146039800F0F2
:10062000DDFB00233370289B1D602A9B002B3FF4C9
:100630008AAC08981E601DB0BDE8F08F2046EFF729
:10064000D9FF32463B46F0F72BFC00287FF4D3ACB1
:10065000631E0993CFE41C230B9A1D441A440B928A
:100660000A9A1A440A926AE7269A012A40F3B0814C
:100670000F9B0BF1FF36B342C0F26B81BBF1000F51
:10068000A3EB060680F2F7820B9BA3EB0B056EE152
:10069000C3F1200306FA03F079E40125DFE400BF8B
:1006A00000002440394600230A22039800F0A0FBF2
:1006B000189B0746002B40F307839B460E96002DA0
:1006C00005DD39462A46039800F06EFD0746099B72
:1006D000002B40F0ED81B846089B1E46013B03EB22
:1006E0000B04069B03F00103CDE90A43039C049924
:1006F0005046FFF74DFB39468346504600F0CAFD91
:10070000049905464246204600F0E4FDC3680146D0
:100710000BF13009ABBB0990504600F0BBFD0999C5
:100720000990204600F05AFB099A002A54D1269BD2
:100730001BB90B9B002B00F0B582002D3FDBB346AD
:100740000A9B0BF8019B9E4200F0C9815146002391
:100750000A22204600F04CFB4745824639464FF0BE
:1007600000034FF00A02204630D000F041FB414622
:1007700000230A220746204600F03AFB5E468046E8
:10078000B5E7039800F02AFB002D06DB069B03F07B
:100790000102269B1D432A4329D151460122039879
:1007A00000F002FD0499824600F074FD002840F339
:1007B000F880B9F1390F00F050820BF131090E9D2C
:1007C0003C460135474606F8019B15E700F010FB53
:1007D0005E46074680468AE7002DC0F29B82269B34
:1007E0001D430B9B1D4300F09582002AA7DDB9F144
:1007F000390F00F032820E9D09F101033C460135AC
:10080000474606F8013BF7E6269B022B7FF7B1AE81
:10081000BBF1000F40F029815B4605220499039843
:1008200000F0E6FA01460490504600F033FD00283F
:1008300040F31B8131230E9D089E013506F8013BD4
:10084000DDE9030100F0CAFA0135002F7FF4E1AEC3
:10085000E3E65046049900F01DFD0028BFF685AE82
:10086000514600230A2203980E9C00F0C1FA0C9B0B
:100870008246661E002B7FF415AF189B002B40F3B9
:1008800018829B460E9D7AE601461A46039800F0B0
:1008900031FC269B0490012B6FDD00230993049A01
:1008A000136902EB8303186900F0F4FAC0F1200029
:1008B00032E69B4B08930333FFF7ECBB069B002B00
:1008C0007FF429AEDDE90612C2F31303002B7FF497
:1008D00022AE944B134033B10B9B01330B930A9B15
:1008E00001330A930123099A0993002A3FF413AEB6
:1008F000D5E73FF424AEC0F13C03ADE601230C93F1
:10090000279B0E9A134403F1010B5E46012EB8BFDC
:1009100001261893172E40F30182012204235B0065
:1009200003F11400B042114602F10102F7D9039B12
:10093000D96303E401230C93279B002B38DD9B46EE
:100940001E461893E6E700230C93D9E700230C9387
:10095000F2E70F9B0F96F31A0026099A1A440A9B96
:1009600009925B440A930B9B1D465B440B93012148
:10097000039800F0DFFA0746A5E5069B002B8CD113
:10098000DDE90601C1F313030A46002BA1D009904B
:1009900085E7DDE904344FF00209CDE91234FFF7B1
:1009A000FBBB7FF40CAF19F0010F7FF402AF06E739
:1009B00001239B462793FFF7BCBB03D119F0010F1E
:1009C0007FF40BAE5E461BF8013D302BFAD013E6E8
:1009D000119A002A00F09F8003F233430A9A0F9E77
:1009E0001A440A920B9A15461A440B92BFE7312318
:1009F000089A01351370FFE500F0FE80DDE904017F
:100A00000E9A494B554205F00F0203EBC203D3E99E
:100A10000023EFF7DDFF2D11CDE9120100F05D811C
:100A200000234FF0020907468846404EEA070AD5E0
:100A3000D6E9002338464146EFF7CAFF01230746AF
:100A4000884609F101096D1006F10806EED1002B68
:100A50007FF4BDABDDE91278FFF7B9BBC8F1010344
:100A60000A900B931090FFF753BB089EB7E4DDF894
:100A700010A002460B46EFF771FC03460C46DDE979
:100A800006010E9D1A46CDE9043401352346A846D9
:100A9000F0F710FA40B9DDE90423DDE90601F0F7CB
:100AA000FFF918B1F30701D5089A32E43E46B4E5E0
:100AB0000398796800F06CF90546002800F023815E
:100AC0003B6907F10C0102339A000C30EFF70AFF83
:100AD00001222946039800F067FB8046FCE50E9D45
:100AE0003C46013547466CE5039C39463246204674
:100AF00000F000FB074652463946204600F048FA0F
:100B000051468246204600F069F90F9B9B1B0F93CC
:100B10003FF4F4ACECE41A9BC3F136035EE700BF8C
:100B2000A81F01080000F07FE8530108C053010826
:100B3000DDE91623DDE91401EFF74AFF089BCDE953
:100B40000C011C70129B012B00F0C580129F089BAA
:100B500011961F4400227C4B40464946EFF738FF70
:100B60000D460446F0F7E4F98146EFF743FD0246EF
:100B70000B4620462946EFF7EFFB09F1300906F84E
:100B8000019BBE4280468946E4D1119D0022DDE9E9
:100B90000C016E4BEFF7E2FB02460B46404649461E
:100BA000F0F7A6F900286ED1DDE90C230020674993
:100BB000EFF7D2FB02460B4640464946F0F77AF97A
:100BC00080B91B9B002BFFF679AC0E9B0E2B3FF7D9
:100BD00075AC5F4B0E9A03EBC203D3E90034CDE949
:100BE000063401E417F8013C3E46302B07F1FF378D
:100BF000F8D0199D013510E54FF00209DDE90478C0
:100C0000FFF7E5BABBF1000F3FF49AAB189C002C3C
:100C10007FF7BBAB0E9B3846013B41460022199340
:100C2000494BEFF7D5FE02468846174609F1010009
:100C3000EFF7E0FC3A464346EFF7CAFE0022454B89
:100C4000EFF78CFB1294A1F150750446FFF7E0BA60
:100C5000312308F10108FFF763BBB34639230E9D2A
:100C60003C46089A474601350BF8013BBAE400239D
:100C70001F460493DEE50A9B5B440A930B9B1D46CB
:100C80005B440B9373E6199B089A03F10108FFF785
:100C900040BBDDF850A0ACE7DDF850A0DDF858B05F
:100CA000FFF773BBB9F1390FD7D0002D3FF785ADF2
:100CB00085E5269B022B03DC0E9DDDF860B05EE42B
:100CC000DDF860B00E96A3E5269B022BF8DCDDF87C
:100CD00060B00E96F3E4374658E74FF00209DDE9BD
:100CE0001278FFF774BA0025039B29461846DD6386
:100CF00000F04EF80890D0B9002240F2AF11164B28
:100D0000164800F0C5FE024640F2EF21124B134890
:100D100000F0BEFE002A3FF740AD50E50021039BE6
:100D2000D963FFF70BBA0E4B0893FFF70CB9039B7F
:100D3000089A4FF0FF3B9A6301232795CDF860B0E6
:100D40000C93FFF722BB00BF000024400000E03FEF
:100D5000E853010800001C40AC1F0108C01F010837
:100D60009C1F010882B049B15AB16BB113780B6076
:100D70001278101E18BF012002B0704701A9002A86
:100D8000F3D1104602B070476FF00100F4E700BFE6
:100D900038B5436C05460C464BB153F8240080B17E
:100DA000026843F824200023C0E9033338BD212220
:100DB000042100F08DFE034668640028EDD1002078
:100DC00038BD0121284601FA04F56A1D920000F0A1
:100DD0007FFE0028F3D0C0E90145E4E731B1436C60
:100DE0004A6853F82200086043F82210704700BF99
:100DF0002DE9F0414FF0000E0E461C460D690746E6
:100E000001F1140001680EF1010E8BB202FB0343E5
:100E1000090C4FEA134C02FB01CC9BB203EB0C43D1
:100E2000754540F8043B4FEA1C44EBDC3CB1B36829
:100E3000AB4207DD06EB850301355C613561304669
:100E4000BDE8F081716838460131FFF7A1FF8046A7
:100E5000A8B1326906F10C01023292000C30EFF7B2
:100E600041FD7B6C726853F82210316043F82260B8
:100E7000464606EB850301355C613561DFE70246D6
:100E8000BA21024B024800F003FE00BFAC1F01086C
:100E90001C200108B0F5803F03463ABF1020834074
:100EA0000020B3F1807F3CBF1B020830B3F1805FAC
:100EB0003CBF1B010430B3F1804F03D3002B06DB92
:100EC000013070479B0003D45B0003D4202070479F
:100ED00002307047033070470368014613F0070281
:100EE00009D0DA0721D498074BBF5B089B08012083
:100EF00002200B60704798B2A0B11046DAB20AB96E
:100F000008301B0A1A0704BF1B0904309A0704BFE4
:100F10009B080230DA0703D45B0800F1010006D019
:100F20000B6070471020C340E8E700207047202086
:100F3000704700BF38B5436C04460D464BB1586846
:100F4000B0B102685A60002201234561C0E9032361
:100F500038BD2122042100F0BBFD03466064002857
:100F6000EDD1002240F24511074B084800F090FDFA
:100F70001C220121204600F0ABFD0028F1D0012207
:100F80000223C0E90123DEE7AC1F01081C20010891
:100F90002DE9F04FD1F8108015690E46A84592460C
:100FA00085B005DB2A46534645468A4690461E468E
:100FB000DAF80830DAF8041005EB0804A342B8BFE9
:100FC0000131FFF7E5FE002800F0898000F11407E9
:100FD00007EB840E774505D23B46002243F8042BED
:100FE0009E45FBD8143606EB88080AF114094645DD
:100FF00009EB850566D2A5EB0A03153B23F0030335
:101000000AF1150A043355452CBF9B464FF0040BDB
:10101000CDF808E08246AE46039405E0090C2AD1DB
:10102000B04507F104074AD956F8041B8DB2002DCC
:10103000F4D0CC463C46002301965CF8040B2168B2
:1010400086B28AB205FB0622000C090C05FB0011D2
:101050001A4401EB124192B242EA0142E64544F8D9
:10106000042B4FEA1143E8D8019E47F80B3056F89D
:10107000041C090CD4D000223B6848461D463C465F
:10108000944602889BB201FB02C202EB154243EA7E
:10109000024344F8043B50F8043B25684FEA134CE4
:1010A000ABB201FB0C33704503EB12434FEA134C18
:1010B000E7D3B04547F80B3007F10407B4D8DDE9B2
:1010C00002E45046002C02DC05E0013C03D05EF84F
:1010D000043D002BF9D0046105B0BDE8F08F024655
:1010E0004FF4B171014B024800F0D2FCAC1F010873
:1010F0001C20010812F003032DE9F04114460746B5
:101100002CD10E46A4101CD03D6C85B3E3074FF0E4
:10111000000806D4641014D02868A8B10546E30777
:10112000F8D52A4631463846FFF732FF36B17B6C98
:10113000716853F82120326043F82160641006463C
:10114000EAD13046BDE8F0812A4629463846FFF705
:101150001FFF28600546C0F80080E0E70F4A013B0A
:1011600052F823200023FFF743FE0646CAE7012179
:101170003846FFF70DFE054640B140F271230122CB
:10118000C0E90423002338640360BFE7024640F24D
:101190004511034B034800F07BFC00BFB05301082E
:1011A000AC1F01081C2001082DE9F0470C462769F7
:1011B000A36807EB62177D1C9D429046064649686E
:1011C0004FEA621904DD5B009D4201F10101FADC86
:1011D0003046FFF7DDFD002851D0B9F1000F00F1D6
:1011E00014010FDD0B464FF0000C09F105024FEA28
:1011F000820E00EB820243F804CB9342FBD1AEF1A6
:1012000014031944226904F1140318F01F0803EBB6
:10121000820C2CD08E464FF0000AC8F120091A68C3
:1012200002FA08F242EA0A024EF8042B53F8042BA1
:101230009C4522FA09FAF2D8ACEB0403153B23F0E3
:101240000303043304F11502944538BF042341F825
:1012500003A0BAF1000F00D13D46736C62680561CE
:1012600053F82210216043F82240BDE8F08704398A
:1012700053F8042B9C4541F8042FF9D8ECE70246BB
:101280004FF4EF71014B024800F002FCAC1F010863
:101290001C20010884460B690069C01A15D10CF1A5
:1012A000140C14310CEB830210B401EB830301E046
:1012B000944508D252F8044D53F8041D8C42F7D0DF
:1012C00004D24FF0FF3010BC70477047012010BCB3
:1012D000704700BF2DE9F04F14460A69236988461C
:1012E000D21A002A83B040F0888001F1140604F17C
:1012F000140202EB830206EB830301E09E427FD2DD
:1013000053F8045D52F8041D8D42F7D076D323467E
:101310000025444698466168FFF73AFD002800F032
:10132000898000F1140949464FF0000C2769D8F86C
:10133000106004F1140B08F1140EC56004F11002E2
:101340000EEB86060BEB870ACDF804B05EF8044B73
:1013500052F8045F1FFA84FBABB2A3EB0B03240C1F
:101360006344C4EB154404EB23449BB243EA0443B7
:10137000764541F8043B4FEA244CE7D808F11501C3
:101380008E4234BF00210121A6EB0806153EB608A7
:10139000002906F101024FEA820208BF0422DDF8AB
:1013A00004B00BEB0204A2454A4434D91546214649
:1013B000E04651F8046BB3B263444FEA164E0EEBAD
:1013C000234E06EB08039BB243EA0E438A454FEADD
:1013D0002E4C45F8043BEBD80AF1FF3AAAEB040A7D
:1013E0002AF0030A524423B952F8043D013F002B6E
:1013F000FAD0076103B0BDE8F08F88DA01258AE7EB
:101400000021FFF7C5FC70B101220023C0E90423CD
:1014100003B0BDE8F08F00294FEA860608BF00261A
:1014200009EB0602DFE7024640F23721054B06488A
:1014300000F02EFB024640F24521024B024800F02C
:1014400027FB00BFAC1F01081C200108F0B50121DB
:1014500083B016461F46FFF79BFC0546002847D081
:10146000C7F30A54C7F313030CB143F48013002EDF
:10147000019314D101A8FFF72FFD0122019B203019
:101480006B612A6114B3089BA4F2334404441C60CA
:10149000099BC0F135001860284603B0F0BD6846CE
:1014A0000096FFF719FD019B00B30099C0F12002DF
:1014B00003FA02F2C34001930A43002B6A610CBF96
:1014C00001220222AB612A61002CDCD105EB8201F2
:1014D000A0F23243086908990B60FFF7DBFC099B17
:1014E000C0EB42101860284603B0F0BD009AE4E754
:1014F000024640F20F31024B024800F0C9FA00BF29
:10150000AC1F01081C2001082DE9F84F16460029E0
:1015100000F096800C46804606F10B05F9F708FAB4
:1015200054F8041C162DA4F1080921F0030758D81B
:101530001025AE4258D8AF4260DABF4B09EB070C1A
:101540009A68DCF80400624500F0908020F0010306
:1015500063445B68DB0768D420F003003B189D42BE
:1015600047DDCB0712D454F8083CA9EB030BDBF89A
:10157000043023F00302104400EB070A554540F302
:10158000F68007EB020A554540F3CC8031464046D1
:10159000F8F71AFF0646002800F0218154F8043CB1
:1015A000A0F1080223F001034B44934200F0B48001
:1015B0003A1F242A00F2D780132A00F2A2800346A1
:1015C0002246116819605168596092689A602146F4
:1015D0004046F8F7F5FD4046F9F7B0F93046BDE86A
:1015E000F88F35F00705A4D50C23C8F80030002685
:1015F00018E01F46DCE90223D3609A60D9F8043072
:101600007A1B0F2A03F0010309EB07001DD83B43A7
:10161000C9F80430436843F0010343604046F9F7DA
:101620008DF926463046BDE8F88FC907AED454F888
:10163000083CA9EB030BDBF8043023F00302A0E71E
:101640001146BDE8F84FF8F7BFBE2B4309EB050183
:1016500042F00102C9F804304A604368083143F09F
:10166000010343604046F8F7ABFDD7E720F00300E5
:10167000C21905F1100C624580F29280CA0785D428
:1016800054F8082CA9EB020BDBF8042022F003022B
:10169000104400EB070AD4453FF773AF5E46DBF812
:1016A0000C1056F8080F3A1F242AC160886000F217
:1016B000B080132A40F2AB8021681B2ACBF80810B7
:1016C0006168CBF80C1000F2AA8008340BF110020C
:1016D0002168116061685160A1689160AAEB050200
:1016E0000BEB050142F0010299604A60DBF804301F
:1016F000404603F001032B43CBF80430F9F71EF901
:1017000090E723681B2A0360636843603DD804F1B7
:10171000080200F1080354E750F8043C23F00303E7
:101720001F446BE75E463A1FDBF80C3056F8081F83
:10173000242ACB60996023D8132A1FD923681B2A37
:10174000CBF808306368CBF80C303CD808340BF188
:10175000100322681A6062685A60A2689A60344670
:101760005746D9464AE72146FEF738F92FE7DCE924
:1017700002135E46CB603A1F9960D5E73346E8E72F
:1017800021463046FEF72AF9E9E7A368242A836058
:10179000E368C36027D004F1100200F1100310E7E2
:1017A000521B09EB050142F0010299604A6054F8AE
:1017B000043C404603F001032B4344F8043CF9F792
:1017C000BDF826462EE7A368242ACBF81030E3683C
:1017D000CBF8143010D010340BF11803B9E74046A1
:1017E000F9F7ACF803E7236904F1180203616369B0
:1017F000436100F11803E4E623691834CBF818308C
:1018000054F8043CCBF81C300BF12003A1E732461E
:101810005EE721463046FEF7E1F8074B5EE7A16838
:10182000242ACBF81010E168CBF8141006D010343D
:101830000BF118024CE700BF68020020226918343F
:10184000CBF8182054F8042CCBF81C200BF1200204
:101850003EE700BF034649B1FF2A02D801200A70C3
:1018600070478A224FF0FF301A6070470846704771
:1018700070B5054684B05BB11C460F4BD3F8E060F1
:10188000234669B12846B047431C0FD004B070BD51
:10189000094B00F58274D3F8E06023460029F1D1AA
:1018A0000A46284601A9B047431CEFD100228A23EB
:1018B00022602B6004B070BD7006002010B51C467D
:1018C00082B0049B009401934FF0FF3300F0ACF919
:1018D00002B010BD2DE9F04F936883B092461768AF
:1018E0000190002B76D04FF0000B0C465D468B68C4
:1018F0000A6848E0B4F90CC01CF4906F2FD0D4E90A
:101900000403A2EB000803EB430202EBD27208F1DE
:10191000010152102944914292BF914689460A46DC
:101920001CF4806F39D011460198F8F74DFD06463A
:1019300000283DD042462169EEF7D4FFA28922F467
:10194000906242F08002A28106EB0800A9EB080237
:101950002661A8462E46A2602060C4F81490324644
:101960005946FEF73BF8DAF80810A3682268A3EBA3
:1019700008033244491BA3602260CAF8081049B327
:10198000D7E900B5083798461046002DF8D09D429B
:101990001E46AFD2A8462E46E1E701460198FFF762
:1019A000B3FD06460028CFD101982169F8F708FC5D
:1019B0000C21A389019D43F0400329600022A381EB
:1019C0004FF0FF300023CAF80820CAF8043003B0F3
:1019D000BDE8F08F00200023CAF8043003B0BDE852
:1019E000F08F00BFF8B506460D46144610B1436BA4
:1019F000002B4AD0B4F90C20A3691007A3601BD5B3
:101A00002369CBB1EDB291042F4621D522686169DB
:101A1000D31A994228DD0133A1680139A160511C14
:101A20002160157062699A4226D0A389DB0701D52F
:101A30000A2D21D03846F8BD21463046FDF7FEFE7E
:101A400000BBB4F90C20EDB291042F462369DDD41C
:101A500042F40052A281626E616922F40052626611
:101A60002268D31A9942D6DC21463046FDF7A8FCFD
:101A700040B901232268CFE721463046FDF7A0FC9C
:101A80000028D7D04FF0FF37D4E7F8F735F8B1E7A3
:101A9000144600B51A460A4B0D461B6885B0DE6831
:101AA00003464CB10749019130460749029400951D
:101AB00000F0CCF800F0DEF804490C46F3E700BF74
:101AC000340100207820010888200108301D010819
:101AD00038B5A1FB021454BBF8F776FC054650B3A9
:101AE00050F8042C22F00302043A242A10D8132AB6
:101AF00013D91B2AC0E9004416D9242AC0E902449C
:101B00000ABFC0E9044400F1100200F1180205E028
:101B10002146F8F7E1F9284638BD02460023284659
:101B2000C2E90033936038BD00F10802F6E7F8F728
:101B300077FA0C2303600025284638BD2DE9F04FC5
:101B400089B08646DDE9137A1E46002F53D015680A
:101B5000002955D0129B002B62D0741E2EB3002694
:101B6000CDE900E1DDF848B0043D029103920AE0BE
:101B7000019BF3B92868002831D0DC4552D2013CE2
:101B8000631C664611D0D7E9009855F8042F3B46F0
:101B90000098DAF8E0C005A9E047421C34D000EB19
:101BA000060CDC45E4D9C7E90098304609B0BDE829
:101BB000F08F00280CDD029B05A918445A1E00F185
:101BC000FF3E11F8013B02F8013F7245F9D1029046
:101BD000039B28681A6804321A600028CDD1019945
:101BE000039A01B110600CF1FF36002230463A60D2
:101BF00009B0BDE8F08F156800F586770029A9D1F6
